:1040000000800010E97304001D7404005B54040078
:104010005F5404006354040067540400000000006F
:1040200000000000000000000000000027740400F1
:104030006B54040000000000EDC500002D74040066
:10404000CDBA00009DC5000069C2000029BA000079
:10405000397404006F54040073540400775404004E
:104060007B54040043740400457404004774040046
:10407000497404004B7404004D7404004F74040030
:104080005174040053740400557404005774040000
:10409000597404005B7404005D7404005F740400D0
:1040A000CDA7010063740400657404006774040004
:1040B000359601006B7404006D7404006F74040085
:1040C00071740400737404007574040010B5054C19
:1040D000237833B9044B13B10448AFF300800123B4
:1040E000237010BD5802001000000000F43D0600CF
:1040F00008B5064B1BB106480649AFF300800648D9
:10410000036813B1054B03B1984708BD00000000D8
:10411000F43D06005C020010580200100000000090
:10412000024B1A6801321A60704700BF7402001017
:10413000014B1868704700BF74020010042808D8AB
:10414000064B53F8203023B122B91A6822EA010144
:10415000196070471A68114319607047E826050016
:10416000042804D8024B53F8203003B199617047FA
:10417000E8260500042804D8024B53F8203003B188
:10418000D9617047E8260500F0B404461AB300264A
:10419000237D9B0608D44FF0FF3300E0C3B1207DA0
:1041A000013B8006FAD59BB192B101F110050B4697
:1041B00000E072B113F8010B013A2070AB4203EB3F
:1041C0000600C1EB0000F4D11AB119460646DFE73C
:1041D0003046F0BC70471046FBE700BF2DE9F04FBA
:1041E000A64B8DB0984207900A9100F08281A44BB3
:1041F0000798984200F04A81A24B079A9A4200F031
:104200007D81A14B0798984200F06D8107980023AB
:10421000072202720372037DD90704D503461A7878
:104220001A7DD207FBD40799802381F830300A46E3
:10423000137D9B06FCD5079A934B0026104682F807
:1042400030609842566016731662027D00F0F2806C
:1042500007988A4B0A9A9842D2F8009008BF062025
:1042600000F0FD80864B0799994200F03A81854B1A
:104270000799994200F0F28000220023CDE908233B
:104280000B9600230493059300220023CDE902231B
:10429000DDE908AB4FF0FF30CDF818904FF0010882
:1042A0000190069F00263A4600235046594645F0A5
:1042B00099FEB0F1004F0B4688BF4B1C03F1FF3154
:1042C000024688BF4242B1F5803F4F440BD201986D
:1042D000824208D218460021CDE90201EAB1CDF8A8
:1042E00010800596019201364645DCD3019969B1EB
:1042F000069ADDE9080108F101081AEB000A4A44B0
:104300004BEB010BB8F1100F0692CAD1DDE9022385
:1043100013431FD0059EDDF81080029C06EB0801B8
:10432000A1FB04230B9C2009039C00FB08F001FB6C
:104330000433002145F056FE484534BFC0EB090068
:10434000C9EB0000642303FB00F3B3FBF9F9B9F1F7
:10435000020F2DD94A4B079C9C4266D0079C237BB9
:1043600003F0C0030A9C6279012A43D003D3022AD6
:104370003DD143F002030A9C22794AB1032A3CD082
:10438000042A78D0022A14BF43F0080343F018032C
:104390000A9CA279079C012A394A08BF43F004030A
:1043A000944218BF079CDBB223730DB0BDE8F08FB9
:1043B000334B079C02980399020A9C4242EA01622D
:1043C0001ED0079C9DF80830217BD2B241F08001BD
:1043D000217322712370227B06F00F0343EA081336
:1043E000DBB202F07F02227384F82830B6E743F094
:1043F0000303C0E743F00103BDE743F02803C7E729
:10440000217B9DF80830079CD2B241F080012173D6
:1044100022712370227B4FEA0813DBB206F00F06ED
:10442000334302F07F022273A362154B1B7B03F020
:10443000C00397E780F8246000220023CDE9082319
:104440000A9B3220D3F80090099600F07BF90B907C
:104450000B99000909070990089112E73020002202
:104460000023CDE9082300F06DF903090B90000744
:104470000993089005E743F0380389E700C000403E
:10448000000001400080094000C0094001211020C7
:1044900000F07AF90799002307220A720B720B7D4C
:1044A000DD0704D5079B1A781A7DD407FBD416497B
:1044B000802381F830300A7D134B9006FBD5002213
:1044C00083F830205A601A731A621A7483F84C20E9
:1044D00083F8542083F850200A991A7ED1F800906E
:1044E0001B7D0820BFE74FF00070012100F04CF960
:1044F0008CE60820012100F047F987E64FF0807034
:10450000012100F041F981E600000140124B984280
:104510000ED0124B0021984290F8302080F83010D5
:1045200013D00F4B984213D00E4B984209D07047CE
:10453000002390F83020194680F83030102000F029
:1045400023B94FF0007000F01FB9082000F01CB92B
:104550004FF0807000F018B90000014000C000402A
:104560000080094000C0094000234FF41651032287
:104570000160427103718371704700BF0170704721
:10458000012B70B405460E46144619D0DAB1037DEE
:1045900003F0200303F0FF0083B11023002000E0AC
:1045A00064B1325C013B2A7004F1FF3400F1010078
:1045B000F6D11CB12A7D10239206F2D470BC70474C
:1045C00070BCFFF7E1BD1046F8E700BF012BF0B467
:1045D00019D0002A30D0037D13F001032ED08C189F
:1045E0004B1C002502E0027DD20709D50278A342C8
:1045F000D2B203F8012C05F1010503F10103F2D158
:104600002846F0BC7047BAB10025067DF4070AD4ED
:104610004FF0FF3301E0002BF2D0047D013BE607B1
:10462000F9D5002BECD00678F6B24E550135AA42EA
:10463000EBD12846F0BC70471546E1E71D46DFE7A1
:10464000062996BF0B4B002153F82110012A0A4B73
:104650000BD0984242680CBF40F28F3340F20733D0
:10466000134023EA010343607047436819434160E4
:10467000704700BF0027050000000140007DC0B268
:10468000704700BF806840F2CF331840704700BFCA
:10469000CB78022B96BF0B4AC123D35C4A78012A00
:1046A0000A7808BF43F00403012A8A7808BF43F060
:1046B0000203012A08BF43F0080303F0CF0303728B
:1046C000704700BFFC260500002201238270C270E3
:1046D00003704370704700BF012905D0002390F894
:1046E000302080F83030704790F8303043F080034D
:1046F00080F83030704700BF1F2811D920380322BE
:10470000824001FA00F00E4BD3F8AC1121EA02020C
:10471000C3F8AC21D3F8AC211043C3F8AC01704707
:10472000032282408140064BD3F8A80120EA02020E
:10473000C3F8A821D3F8A8211143C3F8A8117047E2
:1047400000C00F400E4A1F2892BFD2F8A821D2F80D
:10475000AC21203822FA00F00A4B10F003001B684D
:104760000AD0022802D8B3FBF0F07047032803D127
:104770000820B3FBF0F070470420B3FBF0F0704763
:1047800000C00F409801001001290AD041B9094A20
:10479000094BD2F8C4100B4023EA0003C2F8C4301E
:1047A0007047044A044BD2F8C41003400B43C2F8CC
:1047B000C430704700C00F40DEF7EFEF38B5044655
:1047C000F8B1012821D1214A214B126889089508A6
:1047D000A3FB0505AD0C05FB01F5FE2D24D85508FE
:1047E000A3FB0505AD0C05FB01F5FE2D25D8A3FBAC
:1047F0000205AD0C05FB01F5FE2D4FF000000BD8B6
:1048000038BD21F00301FE2901D8002038BD4FF04A
:1048100080435960012038BD2146FFF76DFF4FF0FE
:10482000804320465D6038BD00200146FFF764FFED
:104830004FF0804320465D6038BD00200221FFF725
:104840005BFF4FF0804320465D6038BD980100104B
:1048500083DE1B4338B5054600200C460146FFF7B2
:104860004BFF4FF080431A69012C22F003021A61BA
:104870001A6945EA02051D6103D11A7842F0020265
:104880001A7038BD10B54FF080442369014603F01B
:104890000300FFF793FF237843F00103237072B600
:1048A0004FF08043AA21552219721A7262B610BDC8
:1048B0004FF080431A7802F0FB021A70704700BF75
:1048C00072B64FF08043AA21552219721A7262B64D
:1048D000704700BF30B4427803210F2A88BF103AD6
:1048E0004FEA420201FA02F18478037804FA02F2F4
:1048F0004FEA430388BF01339B0003F1804303F574
:1049000030331C6824EA01011960196803240A4342
:104910001A604278C1780F2A88BF103A4FEA4202E3
:1049200004FA02F401FA02F10378154A4FEA43034C
:1049300088BF013352F8235025EA040442F823408B
:1049400052F82340214342F8231002790378012AC8
:1049500041780BD030BC012202FA01F1094A52F829
:10496000230020EA010142F8231070478A4030BC3E
:10497000044850F823100A4340F82320704700BF32
:1049800040C0024068C002407F2810B40ED981B9EF
:104990000E4B01E0802915D033F8022F8CB28242F1
:1049A00001F10101F6D104F1800080B25DF8044B01
:1049B0007047FF2806D8064B803833F810005DF8A2
:1049C000044B704700205DF8044B7047FA2805003F
:1049D000FC28050061280AD00749002201E0834233
:1049E00006D031F8023F0132002BF8D17047002287
:1049F000024B33F8120070471C270500FC29050004
:104A0000F8B51E4E012303704370B36900251C499D
:104A10001C4A8370C570044613680868E3606060D0
:104A200025746574A574E57425756575A575E575BA
:104A300025766576A576E57680277169B269258148
:104A4000678104F11C0048F054FFB2692946A018A0
:104A50001C30C2F1100248F070FF2946402204F1D8
:104A60002C0048F06AFF29463A4604F16C0048F0F1
:104A700064FF054B1868C4F8EC00F8BD000008207E
:104A8000CC000010800A0010DC2B05002DE9F0415D
:104A9000214E82B034684FF035082046FFF7B0FF52
:104AA0001E4B4FF0010C186ADD69C4F8F500986AD6
:104AB000032704233621322284F8F08084F8F1C0E1
:104AC00084F8F27084F8F31084F8F920C4F8FB003D
:104AD00084F8F43084F8FA30E5B1284649F087FAD2
:104AE00004F20113C7B24FF00C0E84F8000184F8F1
:104AF000FFE029463A46184648F0FBFEC419214615
:104B0000FF2301F8013B3068091A02B0BDE8F0410B
:104B100001F034BDFF34F2E77C0A001000000820E9
:104B200070B51C4D2C682046FFF76AFF1A4B3520E4
:104B3000DA693721012384F8F00084F8F31084F84F
:104B4000F13084F8F230C2B10426032006210C2291
:104B500084F8F53084F8F46084F8F60084F8F710EF
:104B600084F8F820F9342146FF2301F8013B286836
:104B7000BDE87040091A01F001BD0322062184F846
:104B8000F53084F8F42084F8F62084F8F710F8342F
:104B9000E9E700BF7C0A0010000008202DE9F04181
:104BA0002F4B1C682378022B02D00020BDE8F08137
:104BB000201D2C49042248F08DFE06460028F4D121
:104BC000294D04F11C00AA69696948F083FE024678
:104BD00010B13046BDE8F081244904F1F0030988A2
:104BE000206919448B42A862144623D205F1240897
:104BF00005F1200C05F1340705F130062C350DE0E8
:104C0000032A28D0062A22D0012A02D1D3F8020092
:104C100028605A780232134499420BD91A78332A01
:104C200010D0EDD9362A08D0FF2A03D0352AF0D18A
:104C30009C78EEE72046BDE8F081D3F80200CCF87E
:104C40000000E6E7D3F80200C8F80000E1E7D3F877
:104C500002003060DDE7D3F802003860D9E700BF1A
:104C60007C0A0010CC00001000000820960A0010FA
:104C700030B50D4C83B04FF6FF736061A161002524
:104C800001A84FF48641E261A570ADF80430ADF89B
:104C9000063000F007FD606010B14FF48843838058
:104CA0000023238003B030BD0000082070B57F4C86
:104CB0002388B3F59A7F00F0BC802FD940F24D12C3
:104CC000934200F0A480B3F5A77F5BD340F2591262
:104CD000934209D0B3F5B57F28D17548218A01F0F8
:104CE000D3FC40F259132380724B1B789B0705D4E9
:104CF0006F4801F0D7FC002800F0C2806B4D05F131
:104D0000080001F0CFFC002800F0BC802B8AB3F52E
:104D10007A7F40F2BF8000232B8070BDB3F58E7F79
:104D200012D0B3F5957F04D0002B77D000232380D9
:104D300070BDA378022B00F0B2805D48218A01F09B
:104D4000A3FC4FF48E7323805A4D2B789E0713D506
:104D5000564E06F1080001F0A5FC00286BD0338AFE
:104D600041F26F7293429CBF5B003382FFF7D8FE23
:104D70004FF49573238070BD4D4801F093FC0028DB
:104D8000E6D170BD40F243129342CFD1A378032BFA
:104D900025D0484D4648218A01F076FC4FF49A739D
:104DA00023802B78990704D4414801F07BFC00282C
:104DB00067D03E4E06F1080001F074FC30B1338A32
:104DC000B3F57A7F48D90023338070BD2B789A07DA
:104DD00046D5FFF7E3FE052842D10323B3703348DD
:104DE00013F010FA606A00BA44F024FA0022324B41
:104DF00044F096FA314B002244F092FA44F052FD0E
:104E000001462B4801F040FC40F24D132380274D12
:104E100005F1080001F046FC30BB70BD284B0120B5
:104E20001A68642102441A60A0702182FFF778FE9C
:104E300083E7204DB5E72B78980799D5FFF7AEFEAD
:104E4000022895D1B0701E4B64211A68218201326C
:104E50001A60FFF71BFE9DE764333382FFF716FEEF
:104E600040F24313238070BD164813F055F9144BDC
:104E700064211A68298201321A60FFF707FE2CE7C5
:104E800070BD70BDFFF78AFE05280AD04FF4B573D8
:104E9000238070BD64332B82FFF7F8FDF6E7054DE4
:104EA000D1E7094813F038F99CE700BF000008205B
:104EB00008000820940A00100000E03F000059405C
:104EC000CC000010E02B0500F42B0500034B9B7871
:104ED00013B9034A13805380704700BF00000820B5
:104EE000800A00102DE9F0073B4B3C4EB3F81CC084
:104EF000B3F81E803A4D33460122002705E0092908
:104F000003F10C0317D017460A461888511CC9B282
:104F10000028F4D05C88002CF1D06045EFD14445E6
:104F2000EDD1304A304C1068918822782F7058604B
:104F300019819A7224E0294B0122002701E01746CB
:104F40000A461888511CC9B21C4610B95888002856
:104F50003CD0092903F10C03F1D1082A2A70224B15
:104F600011D093F800C0214923460A4652F8060D95
:104F70000968928843F8041B60609A8084F80AC02C
:104F8000BDE8F00770470027DFF864A0DFF8649001
:104F9000124A93F800C0B8463B46917ADCB2C1EBA6
:104FA0000C01B94203F10103C4BFA046CFB2082BE4
:104FB00002F10C02F1D108EB48048AF8007089F87C
:104FC000008085F8008006EB8404CCE7064B2F7048
:104FD00093F800C0C7E700BF9800082038000820F9
:104FE00078020010AE0008207B020010B4000820F8
:104FF000790200107A020010F0B4154A154D1678A7
:10500000154B0136F6B216700027012205E02A7012
:10501000CAB2092A03F10C0318D05C881888511C05
:10502000204380B20028F2D0987A301A7728EEDD3B
:10503000184600F8017B01302A70CAB25F70092A55
:1050400000F8017B077003F10C03E6D1F0BC704758
:105050007B02001078020010380008202DE9F84F7C
:10506000304C2388292B12D92F4D0026AB8A26805D
:10507000B3F5807F04D0B3F5007F0CD0BDE8F88F86
:105080002A4FEA8C3B889A4212D0BDE8F88F002361
:105090002380BDE8F88F254BE98C1A889142F4D122
:1050A0002A8D5B889A42F0D1BDE8F84FFFF71ABF0E
:1050B0002A8D7B889A42E8D1FFF714FF0223294604
:1050C0006B7551F8168F1A4BB1F804C01A689B889B
:1050D000C5F82080A5F824C0C5F81620B5F824B07E
:1050E0008B80D5F820A0B5F81C90B5F81E80B7F8D5
:1050F00000C07F88082006216B81C5F806204FF08C
:105100002A03A5F804B0C5F800A02E75A5F82690CE
:10511000A5F82880A5F81CC0EF8328736973238045
:10512000BDE8F88F960A001098000820800A001049
:105130008C0200102DE9F84F504E4FF6FF73F28BA2
:1051400095B29D424FD0DFF858814D4BB8F8000022
:105150001988684008423BD04A4B4B4F1D885B88FA
:105160003D807B80DFF83CA1B7F80290474B0124DB
:105170004FF0000C05E0092A03F10C030DD0A44602
:1051800014461988621CA942D2B21846F3D1598834
:105190004945F0D18AF800C003E0082C8AF80040A5
:1051A0002AD0034653F8040F9B883060B380384AF6
:1051B000384B15681F88948837480E37002108221D
:1051C000C6F8065084801F8071733273BDE8F88F73
:1051D000318CB8F802005B8848401842BCD12A4F95
:1051E0003A807980BEE7338CAB42ACD12B4B186848
:1051F0009B883060B380DAE7FF2106221F4848F021
:105200009CFB234B244A798898881F68B8F8009043
:10521000002302F1300B3473DFF88CA0B8F8028061
:10522000F584347406250424C6F80670C6F8167092
:1052300090809082174A4FF02A0C318586F82030F2
:10524000012186F8213086F8223086F8233086F84E
:10525000243086F82530B574F474CAF800B0A6F886
:105260001C90A6F81E80A2F800C03375B373737447
:105270007175F1737573BDE8F88F00BF9800082051
:10528000780A0010880A00107C02001038000820FC
:105290008C020010960A00109E000820082C0500C1
:1052A000800A0010780200107C0A001010B590F8F7
:1052B00020300446062B0ED00B4A238A1268606801
:1052C000518A8B4298BF194601F058F9062384F899
:1052D0002030012010BD054B1B7803F0040303F0C0
:1052E000FF00002BE8D110BD740A0010940A0010D2
:1052F00090F82030062B01D000207047104B1B780F
:1053000013F0010319D00F4A038A1268528A93429C
:1053100009D842680021134443600123018280F8C8
:1053200020301846704741689B1A03820A440123C3
:10533000426080F82030184670471846704700BF1A
:10534000940A0010740A0010024B1878C0F3400051
:10535000704700BF940A001038B543880446A3B1D3
:10536000D52B0ED12046FFF7C3FF05462046FFF799
:105370009DFF284010F0FF0006D0228A6AB984F809
:10538000202000236380022038BD4AB192B20282FD
:10539000416080F82030002AF1D0D5236380E1E716
:1053A0004280012038BD00BFF8B5458804460E464E
:1053B00017462DB1F42D14D0002363800220F8BDD0
:1053C00001B310468847114B20821B6884F8205097
:1053D00063600F4B1B785B0701D53846B047F42359
:1053E00063802046FFF784FF05462046FFF75EFFF7
:1053F000284010F0FF00E2D0238A002BE9D184F886
:105400002030D9E761800120F8BD00BF7C0A001080
:10541000940A0010C269038BD01A80B2704700BF93
:1054200070B5438882B00446002B2FD040F2211281
:10543000934226D1438A002B32D02B4A2B4B126841
:105440001B880220A260638284F82000228B002A3D
:1054500037D013B3A268636910781870638A228BFF
:10546000A6686569013B013A9BB292B201360135EB
:10547000814263822283A6606561E8D1A38B934257
:105480002DD000236380022002B070BD808BE268C3
:10549000638A20836261002BD8D140F2211363809C
:1054A00094F82030022B06D00191FFF74DFF0199AF
:1054B0000028E9D0C1E70323002084F8203002B09F
:1054C00070BD002BE9D0A06810F8015B013B9BB2D6
:1054D000A9426382A060D1D0002BF5D1DDE7002086
:1054E00084F820006080CFE77C0A0010960A001044
:1054F0000023C1604161C261028380F82030438291
:1055000003804380704700BF013A30B48D18A94230
:1055100014D20B461C785A78023302EB042292B262
:10552000104480B2824284BF013080B29D42F1D8E3
:10553000CB432B4423F0010302331944A94201D089
:1055400030BC70470B7830BC1B02184480B28342D9
:1055500084BF013080B2704738B50E4C0822637C9E
:10556000257C04F11A0103EB0525ADB2A5F10E006F
:1055700080B2FFF7C9FFA5F1140292B204F1220133
:10558000FFF7C2FF10B94FF6FF7038BD40BA80B2C6
:1055900038BD00BF9800082070B4C478134B0C4489
:1055A000E4B2DC7082780D0A2A44D2B29A7046784E
:1055B00095425E700078187003D90136F6B25E70BD
:1055C0008EB1C9B28C420CDA0132D2B29A70074B5A
:1055D0003AB95A780132D2B25A7012B91A780132F5
:1055E0001A7070BC704701301870EAE7900A00101A
:1055F00010B5084C014620680830FFF7CDFF064A79
:105600002368507814789178D2781C725872997205
:10561000DA7210BD740A0010900A001008B500205C
:1056200005491422FFF770FF10B94FF6FF7008BD4F
:1056300040BA80B208BD00BFA6000820FFF78CBFAB
:1056400030B4154B15490022154C04204FF48065E9
:1056500083F8B92183F8D92183F8F92183F8192235
:1056600083F8392283F8592208702580A3F8942101
:10567000A3F89621A3F89821A3F89A21A3F89C21D6
:10568000A3F89E21A3F86422A3F8A822A3F8EC2291
:10569000A3F8302330BC7047980008209402001013
:1056A000880200102DE9F0012A4C2B4EB4F8645208
:1056B0003288B4F8A872B4F8ECC2B4F8308301327E
:1056C00092B2B2F5FA4F1ED34FF480521023AB4280
:1056D000F5D0BB42F3D06345F1D04345EFD03280E3
:1056E0001E4A042695B1B4F8A8520127194C45B3B7
:1056F000B4F8EC520DB3B4F8304334B31670002054
:10570000BDE8F001704753BA9BB2E0E715702C4634
:1057100004EB0414124EA4003219F0D09380D1800F
:1057200048B1038833534388538040231372104693
:10573000BDE8F00170473051F7E7022425461570A7
:10574000E6E73D463C461570E2E703242546157022
:10575000DEE700BF980008208802001094020010C5
:10576000F8020820DFF850C02DE9F001DFF84C8086
:10577000BCF89461002388F80030AEB101231F46C5
:105780000CF5CA7100E02F4631F8024F5A1C1E4634
:10579000D5B2134634B1062AF5D188F80050BDE8D9
:1057A000F001704788F800700CEB4606A6F89401EB
:1057B000BDE8F001704700BF980008209402001077
:1057C0002DE9F04FBC4D042887B02B6821D0DFF8BD
:1057D0000CB3BA4EBA4F0BF13602032832603A606E
:1057E00070D0022800F0E680052800F087819BF841
:1057F0000E30452B00F02981B24812F08DFCDFF805
:10580000EC82B14C0023238088F8003007B0BDE85B
:10581000F08FDFF8D882AC4CAC4A1388002BF1D063
:1058200003F11C01AA4ADFF8B4B289B21268080A6F
:105830008BF810008BF81110167A08335BBA11251B
:105840000020ABF826308BF816608BF81750ABF8B9
:10585000280090889F4BABF82200D58818885B8879
:10586000ABF82450ABF81C30ABF81A001088934BFF
:10587000ABF81E0050880BF136022180ABF82000F7
:105880001A60954900230A884520013292B2140A11
:105890008BF813208BF812408BF80E008BF80F302A
:1058A0008BF815308BF81430ABF818300A80FFF7FE
:1058B000B5FEC043ABF81800002388F8003007B0ED
:1058C000BDE8F08F5A7E02F00F02032A97D11A8AA0
:1058D000DFF81882002A94D1082288F800207A4C38
:1058E000019312F09DFD794A019B98F8000000F0A9
:1058F000200101F0FF05002900F08F810021142014
:10590000DFF8D091597611808BF82F002822228061
:1059100050228BF82E201A7A06268BF82A205A7AE3
:10592000B9F802108BF82B209A7AB9F800508BF84E
:105930002C20D87A694A8BF82D00187B8BF826002A
:10594000587B8BF82700987B8BF82800D87B8BF846
:1059500017608BF829009888ABF82200D888ABF83C
:105960001A50ABF82400ABF81C101988ABF81E10C5
:105970005988ABF820105B7EDB0640F1478100239D
:1059800082F8313082F83030228800234021100A1A
:105990008BF811208BF810008BF816108BF835302F
:1059A0008BF83430ABF83230FFF7D6FDC043ABF89C
:1059B000320066E74A4AD1780131C9B2D17061B983
:1059C00091780131C9B2917039B951780131C9B2B8
:1059D000517011B9117801311170587E3A4C3B4A1F
:1059E00000F0FD050021052D2180118000F0A08030
:1059F00000285ED0198A002900F0F780997E4D1E9C
:105A00009D76002955D1D97E082900F0A281451E36
:105A1000012D40F29B8104299CBF4FF0030C0CFA2E
:105A200001FC00F00F0094BF5FFA8CFC4FF0300CCB
:105A30000131451ED97683F81AC0072D39D8DFE821
:105A400005F089A3A681388138811F4C9BF810A0EE
:105A50009BF81120238802EB0A2A9A4526DC9BF842
:105A600014301FFA8AFA9906A4F800A040D19BF8D6
:105A70001530002B3CD1DFF85C90B9F80030002BDA
:105A800040F0A280B9F80220002A40F09D800193E6
:105A9000FFF7C4FD4FF6FF718842019B00F02081A3
:105AA000104812F039FBDFF84480ABE60E4812F0E4
:105AB00033FBDFF83880A5E6740A00107C0A00107A
:105AC0008C0A0010102C0500960A0010840A0010A1
:105AD000980A0010800A0010820200109800082026
:105AE00084020010802C0500382C0500940A001058
:105AF000B34812F011FBDFF8F48283E6B14B1B6868
:105B00009B88002B3FF47BAEAF4AB04CDFF8DC82C1
:105B100000230BF12A0108201380316039602B60CB
:105B2000238088F800000292FFF7C0F8029A74E61A
:105B30009A7E0132D2B2782A9A76BAD15976DFF8B3
:105B4000AC825FE6DFF8A482DFF8A49211228BF822
:105B50002F20DBE6DFF8989212204FF0020E042788
:105B600001265A252C2160228BF82F008BF836E075
:105B70008BF837708BF838608BF8395021808BF8B0
:105B80002E20DFF86882C6E6DFF86492E5E7DFF8EA
:105B90005C82042188F800100292019312F040FC0C
:105BA000029A019B11883A683260002900F0A880AF
:105BB0001A8A002A00F0A4802832182122808BF84B
:105BC0002F10DFF82C92A3E69BF817208049112AAA
:105BD000CA8B34D093427FF46CAFBBF82010B9F875
:105BE000022091427FF465AF51E700F00F000328D7
:105BF000DFF8F8817FF406AE082188F800100292E1
:105C0000019312F00DFC029A019B6EE601215A23CA
:105C100082F8301082F83130B6E600F0100101F061
:105C2000FF0C002979D0012604201121DD761E8287
:105C300058761580DFF8B8918BF82F1066E64FF68E
:105C4000FF708242C6D1098C9142C3D1BBF824E0D7
:105C5000AAF11C035F49BBF822A0BBF81A80BBF86D
:105C60001CB02380DFF85C91CDF80CB001F1440347
:105C700001F5AA70059403E0443383427AD061466B
:105C800033F8402C9C46002AF6D07245F4D133F804
:105C90003E2C0AB15245EFD133F8442C002A4CD1A6
:105CA00033F842BCBBF1000F06D04245E4D133F8D3
:105CB000422C039CA242DFD1434AC9F80010DFF80E
:105CC0002C81454900230220138088F800003160B0
:105CD00039602B60059C0292FEF7E8FF029A9CE572
:105CE0009BF81710DFF8E88006294CD01129ADD0B9
:105CF000012954D0394812F00FFADFF8F08081E51D
:105D000098F8002097077FF57DAD2821102221808B
:105D10008BF82F20DFF8D890FAE511882A4D49B189
:105D2000C00747D5A3F810C0588A814288BF1080A9
:105D3000118819820022DA7635E74FF6FF74A24205
:105D4000B3D133F842BCA345AFD1B5E705297FF401
:105D500062AE0022DFF894805A76802288F8002014
:105D6000019312F05DFB14228BF82F20DFF8809056
:105D7000019BCBE51A48059CC9F800C0DFF86C8090
:105D800012F0CAF93EE50290FFF7E6FB029A904254
:105D900030D0144812F0C0F9DFF8508032E598F89E
:105DA0002220082A00F0AD800F4812F0B5F9DFF884
:105DB0003C8027E5188A0028B6D028800146B9E73C
:105DC000682C0500980A0010840A0010960A00103A
:105DD00098000820F8020820C2000820942C050032
:105DE000C82C0500EC2C0500B02C0500940A00100E
:105DF000800A0010B8F822C0B8F81A10B8F81C30A1
:105E0000B8F8240008F5E072CDF80CC004910593B1
:105E100008F5207CCDF800A012F8071CA2F12003A1
:105E200021B132F81C8C804500F08A802032624516
:105E3000F2D19BF82F30CC4903F03F03022B00F046
:105E4000C880DFF83C839BF82F20C74B52073FF5F3
:105E5000D9AC93F8295093F82DE093F82C7093F86F
:105E60002B6093F8262093F8280093F8271093F8D6
:105E70002AC00135DFF80CA3EDB283F829E083F8DE
:105E800028704FF0140E282783F82760502683F8D7
:105E90002D5083F82C0083F82B108AF8002083F80B
:105EA0002A2083F826C083F82FE0278083F82E600D
:105EB00065B90130C0B283F82C0038B90131C9B2DC
:105EC00083F82B1011B9013283F82A20BBF8223055
:105ED000BBF82460BBF81A50BBF81C00A34FB9F8FC
:105EE0000010B9F802203B80ABF82430ABF82260F8
:105EF000ABF81E50ABF82000ABF81A10ABF81C2022
:105F000042E5B8F824204FF6F6718A424FF00000BF
:105F10008CBF0932083288F82200A8F82420BBF888
:105F20001C10BBF81A20B9F80200ABF82010ABF82F
:105F30001C00ABF81E20ABF81A30DFF84482BBE43B
:105F400032F81A8CDDF80CA0D0457FF46FAF32F830
:105F5000208CDDF810A0D0457FF468AF32F81E8C9D
:105F6000DDF814A0D0457FF461AF9BF82F20DFF857
:105F70001082002012F0040FDDF800A02B6088F8DA
:105F80000000DFF8E4C140F051829CF82EC0AAF175
:105F900014004FEA1C1C4FEA8C0CCCEB0000DFF81D
:105FA000E4A101F00F0180B2022920808AF800C02C
:105FB00000F0F08010B9910700F0F180BBF826C026
:105FC00018896949844500F03C8210228BF82F2003
:105FD0009CE4B1F89461654ADFF8A8A100278642E5
:105FE00010808AF8007011D0012601F5CA718AF874
:105FF000006002E0072E2CD0334631F8027F5E1C91
:10600000B842F6B2F6D100238AF800309BF8B90105
:1060100020B30021564F0B4601260CE0062E5FFAF6
:1060200086FE00F0B48097F83900314620370136FB
:10603000002800F0A9800728F0D148010BEB000EE2
:1060400023B19EF8BAE1997E8E45E7D9484B0344C7
:10605000E4E7DFF82C818AF80030F4E60146DFF847
:1060600010C10CEB4113002B77D003210026042034
:10607000997619769E75DE76D875BBF824003D4971
:106080009880BBF822002B60D880BBF81A0091F8EA
:1060900000E01880BBF81CC04F788D78C9780120CB
:1060A00058761882A3F802C083F80CE05F739D73E2
:1060B000D9739BF82910D9729BF8281099729BF814
:1060C000271059729BF82610197202920193FFF75C
:1060D0008FFA9BF82E10029A01F0F0005028019BD5
:1060E0007FF73AAD0F092449053F0D78BF008AF8C4
:1060F00000603046B8422CDA0BEB000696F83650BA
:10610000B64635B3012D09D0022D0AD09EF837606E
:1061100006EB000EEEB15FFA8EF0EBE70130C0B295
:10612000E8E796F837C0BCF1040FEFD196F8387065
:1061300096F839608AF8000046EA0726B6F5AD7F82
:1061400034BF30464FF4AD700D701680588298827F
:1061500002E58AF800000D70FEE4084811F0DCFF4B
:10616000DFF81C80FFF74EBB98000820800200106B
:10617000380208208402001095020010002D05004E
:10618000940A0010940200108AF800E067E78AF889
:1061900000E068E702F03F0112297FF40BAFD2065E
:1061A00001D5198AD1B95A7E02F00F0101390729A8
:1061B0003FF628AB0FF2040C5CF821F04F640000AE
:1061C000E163000017630000D5620000B3620000C5
:1061D0009D620000CB5F00008162000003F10C00B3
:1061E0000193FFF7D9F9A74A9BF82A001178019B80
:1061F0000391DDF80CC0A4498445D4D192F801C0C4
:1062000091F82B00CDF814C08445CCD191F82C0026
:106210000490DDF810C090786045C4D191F82D103D
:10622000D2788A42BFD1039993F81BC0197305999C
:1062300098735973DA73BCF1000F19D1187E997EE7
:106240009A7D411AA1EBD201C9B20A44D0B2CAB2B6
:1062500012F0800F18BF4A42D97D18BFD2B2A1EB0D
:1062600091010A44D2B2987502EBD0001876DA7523
:10627000187E01210022987688F800101A8292E791
:1062800098F80010814ACE077FF5BCAA0021597604
:106290001023137012F0C4F8FFF7B4BA98F8002076
:1062A000D2077FF5AFAA0721002259769A76FFF729
:1062B000A9BA208818B10193FFF79AF9019B9BF8BE
:1062C0002F20D10700F1A3802288002A7FF47DAE21
:1062D000FFF798BA208818B10193FFF789F9019B5D
:1062E0009BF82F2012F0010200F0968098F8002011
:1062F000D50740F189800022072159769A761A82C3
:1063000001200193FFF774F9102288F8002012F0A1
:1063100087F8019B59E69BF82F10CD0724D5D006AE
:1063200022D41A8A002A7FF46DAA208801930130B2
:1063300080B2FFF75DF998F80020208842F0100144
:1063400088F80010019B514910B142F012020A7006
:10635000019312F065F8019B0120082100221882A8
:106360005976DA76FFF7F2BB89060BD59BF834C075
:106370009BF835003168258840EA0C200144281A32
:1063800031602080208858B1D20609D498F80020C6
:1063900042F0020288F800200193FFF729F9019BDF
:1063A0009BF830009BF83110394A01EB0021988AA4
:1063B00089B28142118000D801B91080118898F803
:1063C0000020598295073FF41DAA324A002111800E
:1063D0000292019312F024F8019B029AFFF785BA0A
:1063E00098F80020D20706D59BF82F10264A01F016
:1063F0003F01122952D0202388F8003012F010F803
:106400002B6800225A761EE506225A7678E7072185
:10641000002259769A7673E798F80010C8077FF53E
:1064200053AF05211A825976FFF7ECB958761A480E
:1064300011F072FE202388F8003011F0F1FFFFF711
:10644000E1B9088D598988427FF4BFADA7E698F875
:1064500000100E4AC9077FF5D5A920884FF0030E1A
:106460004025002183F819E01570198228B14221D6
:1064700011700193FFF7BCF8019B064A00211180BF
:10648000FFF7BDBB900A001098000820940A001086
:1064900080020010840A0010242D050092F82E209E
:1064A00002F0F001502939DD2F491209A2F1050E41
:1064B000087800224FEA8E0E8AF8002072454EDAE4
:1064C0000BEB020595F83600AC46002847D00128B2
:1064D00042D0022808D09CF8375005EB020C002D62
:1064E0003DD05FFA8CF2E9E795F83790B9F1040FE7
:1064F000F1D195F838E095F83950DFF874C045EAE5
:106500000E2EBEF5AD7F34BF75464FF4AD758AF8DB
:1065100000200870ACF800E05D829D829BF82800A6
:106520009BF829109BF826E09BF8275003229872CD
:10653000D9725A7683F808E05D7201200193FFF763
:1065400057F8019B094A00214220198221801180BD
:1065500088F80000FFF753BB0132D2B2AEE78AF8E9
:1065600000200870DAE700BF95020010840A0010CE
:106570008002001040BA80B2704700BF0A1E034676
:1065800009DD0548054900680A80834203D01946A1
:1065900092B247F0AEB970478C0A0010840A00101E
:1065A0002DE9F041334CE37D062B03D0BDE8F041EB
:1065B00011F090BF304D2B88B3F5C17FF6D3363B39
:1065C0009BB25F08B3EB470F07F128034FF00006BB
:1065D0004FEA1322CCBF07F10108B84622742B8082
:1065E000637484F8326084F83360FFF727F8C0439F
:1065F000608626766676FFF711F82B88C0430E3347
:1066000020832B8011F066FF1C4A08F128031068D4
:106610009BB24FEA132E4246C11984F810E02B803A
:10662000637447F066F939461548FEF7B5FF154B18
:1066300084F8326059789A781878DB7884F82710D3
:1066400084F8293084F8282084F8336084F8260000
:10665000FEF7F4FFC043608626766676FEF7DEFF1F
:106660002B88C0430E3320832B80BDE8F04111F00E
:1066700031BF00BF98000820960A00107C0A001065
:10668000BE000820900A001010B541600446FDF7D6
:106690004FFD206010BD00BF90E80C001344036064
:1066A000704700BF10B50446FDF742FD94E80C00AA
:1066B000801A984234BF0020012010BD70B4134EE0
:1066C00075682A78A2B103780D2B11D00A2B0FD050
:1066D0009A4214D1002306E0C25C0D2A08D00A2A8F
:1066E00006D094420BD10133DBB2EC5C002CF3D129
:1066F000B268F368012081E80C0070BC704736680E
:10670000002EDDD1304670BC704700BF5C2D050007
:1067100010B5064C20683DF07FFC054A0023106848
:10672000236046F021FA012010BD00BFA002001036
:106730009C0200100A4B10B50A460C461B6801214A
:1067400047F008F8A042034603D0FFF7E1FF00201E
:1067500010BD044A012011680B44136010BD00BF36
:106760009C0200109802001070B5038D40F22B15AA
:10677000AB4282B00446164600F0A380B3F5967F84
:106780001DD340F23112934200F08E80B3F5997F11
:1067900032D240F22D12934237D040F22F12934260
:1067A00025D100F12805654847F021FC63490246E0
:1067B0002846FEF7D1FDD0B9002002B070BD40F2EE
:1067C000231293425FD0B3F5927F59D337D040F272
:1067D000291293420BD104F12805594847F007FCD0
:1067E000574902462846FEF7B7FD0028E4D00023AB
:1067F0000220238502B070BD40F23312934211D0C3
:1068000040F235129342E6D0F1E700F128054D48F9
:1068100047F0EDFB4B4902462846FEF79DFD002858
:10682000E5D1C9E700F12805474847F0E0FB4649B4
:1068300002462846FEF790FD0028D8D1BCE700F1BB
:106840002805424847F0D3FB404902462846FEF758
:1068500083FD0028B0D0002EC9D004F1B4002E2151
:1068600047F018FC064600284CD03948314605222E
:1068700047F0E8FB002831D140F22B13238522E0BA
:10688000002BB4D102850846019147F0B0FB04F11A
:106890002805024601992846FEF75EFD00288BD0A8
:1068A0004FF492732385CCE700F12805294847F07F
:1068B0009EFB284902462846FEF74EFD002896D149
:1068C0007AE700F12805244847F091FB2249024667
:1068D0002846FEF741FD002889D16DE71F48314663
:1068E000042247F0AFFB18B940F22D1323858EE741
:1068F0001B483146042247F0A5FB38B940F22F135C
:10690000238550E740F22913238566E71548314671
:10691000042247F097FB18B940F231132385C5E7ED
:1069200031461148042247F08DFB18B940F2331369
:10693000238579E740F2351323854EE7A8800500CB
:106940009C7E0500C480050058800500907F0500EE
:10695000D87E0500208105008C800500E87E0500BA
:10696000E07E0500887F05005081050038B5038D65
:1069700004460BB340F20512934219D100F12805E9
:1069800028460F492246FEF70FFDA0B1B4F83C217E
:10699000D4F83431D4F830119B1A002B0A44C4F8CF
:1069A0003431C4F8302103DD40F205132385E7E7D5
:1069B00000232385022038BD00F12805F4E700BF3D
:1069C0000D6A000038B50E4B0E4D1B6804465A8AFE
:1069D0000121D0F83831286846F062FC002803DD38
:1069E000A4F83C0180B238BD074A2B681088917822
:1069F0001880002299700220A4F83C2138BD00BF05
:106A0000740A00107C0A0010F0ED05000A4B10B566
:106A10001A68D0F83431528A04469342D8BF9AB2E9
:106A2000064BA0F83C21D4F83011186846F061FFFD
:106A3000B4F83C0110BD00BF740A00107C0A0010BD
:106A400038B50C460546C1B1D1F8540185B112F0F4
:106A50001BF9092801DD002038BD2846D4F854412F
:106A600047F0AAFA0146204612F0F6F8012038BD98
:106A7000294612F0F1F8012038BD4FF0FF3038BD43
:106A80002DE9F047B74DB84E2B7837685906A2B0BC
:106A9000FC6900F18480002C00F0A88003F008025B
:106AA00002F0FF013AB322780132D2B2272A2270D3
:106AB00022D920232B70D4F838311BB1AB4B186886
:106AC00046F052F8D4F8400108B13DF0A5FAD4F8E8
:106AD00050313BB1D4F8540112F0F4F8D4F850011D
:106AE00012F010FA20463DF097FA33680022DA617E
:106AF00022B0BDE8F087217013F0300FDBD11A0609
:106B0000D9D494F82D31032B1BD0A28840F2EF1179
:106B10008A4200F0CF81B2F5F87FC0F0F08040F2F9
:106B20003E218A4267D040F24F218A4200F0AB8179
:106B300040F206218A4200F068810022A280032BE5
:106B4000D6D1B4F84C3040F25B12934200F034815D
:106B5000B3F5AE7FC0F08480B3F5B97F6ED040F25C
:106B6000358140F28112934200F0F982B3F5C17F82
:106B700080F0A68140F2731293426BD040F27D12F6
:106B8000934208D120467A490022FFF7EDFD002804
:106B9000AED010232B700023A4F84C30A8E74FF49C
:106BA000AE703DF033FA044600B300F150031946CD
:106BB000F86163221F460430FEF79AFC394604F15F
:106BC00028006322FEF794FC0023A4F84C30A4F8BC
:106BD0004E3084F82D312370C4F83831C4F8403178
:106BE000C4F85431C4F850312B7857E720232B7068
:106BF00022B0BDE8F087261D30460A21FEF710FCC2
:106C0000002840F0B48194F82D3198E7002304F572
:106C10009877C4F8383139463046FFF74FFD0028E1
:106C200040F0918339465348FFF748FD30465149BB
:106C300047F0B9F94FF4B973A4F84C3020464E49E7
:106C40000122FFF791FD00283FF452AF40F2731389
:106C5000A4F84C302046FFF789FE002899D147E779
:106C6000B3F5A77F1BD000F28D80B3F5A37F00F0B2
:106C7000B18240F2B08140F24712934200F09C8012
:106C8000B3F5A67F87D120463C490122FFF76CFD72
:106C900000283FF42DAF4FF4A773A4F84C30238D98
:106CA000CE2B05D0D42B15D033B30023238570E72A
:106CB000D4F8540111F0E8FF00287FF719AFD4F899
:106CC000540112F013F8C4F84001002800F0528378
:106CD000D4232385D4F84061304647F088F9314603
:106CE000024604F12800FEF737FB00283FF400AF0E
:106CF000D4F840013DF090F9CE232385D8E7002A4F
:106D000000F0DA80B2F5F07F7FF417AF261D304631
:106D10002021FEF785FB00283FF475AF04F15007F2
:106D200038461749032247F08DF9002840F0D180FA
:106D3000012384F82C3140F2EF13A3803046202148
:106D4000FEF76EFB00283FF45EAF94F850302F2B17
:106D500000F0CB8000231022A3802A7094F82D31FC
:106D6000EDE600BF940A0010740A00109C020010A7
:106D7000D87F05004C800500BC7E05003C810500E5
:106D80005881050040F25712934200F0CF81B3F5CD
:106D9000AC7FC0F04C8100F0D481B3F5AD7F7FF4BF
:106DA000FAAE2046CA490122FFF7DEFC00283FF474
:106DB0009FAE40F25B13238504F12800C5490422ED
:106DC000FEF7CAFA00287FF4E4AE91E640F26312BF
:106DD00093423FF43FAFB3F5B27FC0F0EB80B3F521
:106DE000B57F00F01081B3F5B67F7FF4D4AE01AE6D
:106DF000304647F0FCF83146024604F12800FEF721
:106E0000ABFA00287FF4C5AE72E6261D30460A2193
:106E1000FEF706FB00283FF4F6AE3046FEF7FAFA1E
:106E20000023204480F84F3094F850300D2B00F0B0
:106E3000E78104F150073846A749102247F002F9CC
:106E40008046002800F019823846A4490B2247F0FA
:106E5000F9F88046002800F01F823846A0490F222A
:106E600047F0F0F80746002800F0298294F82D3109
:106E7000012B55D0022B00F0E081042B7FF45DAE96
:106E800040F24F23A380B4F84E30D4F80C80E68A49
:106E9000002B00F0D98040F2C312934244D000236B
:106EA000A4F84E3000220323E28284F8242084F8E0
:106EB0002D3142E6261D41E74FF4F073A38025E70C
:106EC000B3F5C27F00F05C81B3F5C47F3FF4C2AE7E
:106ED00061E638468349042247F0B4F8002840F0C0
:106EE000EA80022384F82C3125E794F85130202BD6
:106EF00000F07F813046FEF78DFA0023204480F8B1
:106F00004F3004F1500104F1B4003C2247F0B0F8D6
:106F10000023012284F82D21C4F8443184F84C3137
:106F200040F20623A38071E794F84B31012B1AD06D
:106F30002B789B077FF567AE6B4B6C4A1E8801234D
:106F4000106884F84B31002E40F03681D4F844614B
:106F5000002E40F3D88140F2C313A4F84E3094F8C9
:106F60004B31012BE4D1002384F84B314BE6304602
:106F7000FEF750FA0023204480F84F303046D4F812
:106F80004471FEF747FA381AC4F84401D4F8501196
:106F900004F1500011F0EAFEB4F85831D4F844215D
:106FA0000133A4F85831022A00F30B82032384F83A
:106FB0002D31C2E5B3F5B17F7FF4EDAD20464C49EC
:106FC0000122FFF7D1FB00283FF492AD40F263139A
:106FD000A4F84C303EE6002B7FF4DDAD94F82C3164
:106FE000032B00F0F38004F1B406022B304600F0CE
:106FF0009081404946F0CDFF002840F094814FF445
:10700000B573A4F84C30204631490122FFF7ACFBA0
:1070100000283FF46DAD11F0E3F901AE0146832283
:10702000304647F025F84FF4B6732385E0E6B3F514
:10703000A97F7FF4B0AD204625490122FFF794FBDC
:1070400000287FF4A6AD53E5DFF8BC9004F1F00A08
:10705000D9F8000008B13CF0DFFF504646F0C7FF0A
:1070600005303CF0D3FF244B0746514640F8043B23
:10707000C9F8007046F097FF3846204946F016F8E8
:107080001F4B0746DFF880901860002800F0308121
:10709000002E00F0AB8040463146FFF74BFB002846
:1070A00000F0C680D4F844319E1BC4F8446101232B
:1070B00084F84B314CE738461249072246F0C2FFAC
:1070C00000287FF447AE032384F82C3133E600BF59
:1070D0003C810500A48105007880050074810500CD
:1070E00010810500F07E0500960A00107C0A001051
:1070F000BC7E0500B88105002F73642FA0810500B8
:107100009C020010F8800500A00200103046B8492B
:1071100046F03FFF002840F05D8194F84A31002B93
:1071200040F0538140F25713A4F84C302046B14947
:107130000122FFF719FB00283FF4DAAC4FF4AC73DF
:10714000238504F12800AC490822FEF705F9002840
:107150007FF41FADCCE440F28113A4F84C302046FC
:10716000A6490122FFF700FB00283FF4C1ACD4F888
:107170003831002B00F0F9804FF4C273A4F84C3082
:10718000238D002B00F0988040F2131293427FF47D
:107190008CAD04F12806304699492246FEF704F9E1
:1071A00000283FF4A5ACB4F83C71002F00F09980A2
:1071B00040F213132385EEE73146FFF7BBFAB8B36D
:1071C000D4F844319E1BC4F84461C1E64FF4A37364
:1071D000A4F84C3020468B490122FFF7C5FA00285D
:1071E0003FF486AC40F247132385E5E5D4F84461CB
:1071F0005DE704F1B40084493C2246F039FF87E69C
:1072000094F82C31032B1F463FF4D1AE012B3FF4F1
:10721000CDAE022B7FF42AAE04F1B400744946F0DF
:10722000B8FE002840F0C780042384F82D3127E6FB
:1072300084F84A01A4F84E0034E694F82C71022F29
:107240007FF4B4AE04F1B4073846704946F0A1FEAD
:10725000002800F0A58038466D4946F09AFE0028C7
:107260007FF4A4AEC4F85001D4F8442100239A421C
:10727000A4F858313FF797AE98E63046FEF7CAF8C3
:10728000204480F84E8004F1600045F001FC94F841
:107290002D31C4F84401EBE53046FEF7BBF820443D
:1072A00080F84E8004F15C0104F1F0003B2246F0CE
:1072B000DFFE94F82D31DBE504F1280678E730464F
:1072C000FEF7A8F8204480F84E7004F15F015148A1
:1072D000082246F0B7FE003018BF012084F84C01A8
:1072E000C4E5D4F8380145F03FFCC4F83871DCE45B
:1072F000D9F800003CF090FEC9F8007084F84A719B
:10730000A4F84E70CEE5FFF703FA012384F84A3162
:10731000C5E53E4946F03DFE002835D14FF4A67341
:10732000A4F84C30AFE430463B49042246F08AFED4
:1073300000287FF46BAC3046384945F0B7FEC4F8FE
:10734000380100283AD094F84C31002B3FF403AFB9
:10735000D4F8380120B145F007FC0023C4F83831D7
:1073600040F27D13A4F84C300CE44FF4C473A4F83D
:107370004C306FE4B4F85831013B9BB2A4F858315B
:10738000002B3FF492ACB7E43046214946F001FEB1
:1073900000287FF4BBAE4FF4A973A4F84C304AE642
:1073A00011F050FC2146C4F854011D4811F09AFD1B
:1073B000C4F8500158E784F82D7143E704F5987735
:1073C00030E440F23E23A38016E44FF4AD73A4F8FA
:1073D0004C30E6E404F598711248FFF76FF9304637
:1073E000104946F0E0FD4FF4B173A4F84C30E5E5E8
:1073F0006C810500E0800500AC8105003C81050042
:10740000C5690000F87E05006081050084810500E3
:107410009081050004810500C0810500D415060097
:10742000416A00004C8005004FF4A040FEF79AB975
:1074300000487047C881050000487047D8810500A2
:107440000249034A01608260704700BF30A6050010
:107450002833060010B50A4B0A4A044603F15401CA
:1074600003F14800C4F890002360C4F89410C4F8F5
:10747000982004F1940004F057FC204610BD00BF92
:1074800088A60500108A0500A0F19800FFF7E2BF6A
:10749000A0F19400FFF7DEBF10B5074B044603F1DF
:1074A000300103F148022360616040F8082F04F0C6
:1074B0003BFC204610BD00BFF0A30500A0F1080072
:1074C000FFF7EABF10B5044A044B0446026083602C
:1074D00004F0F2F8204610BD30A60500283306005F
:1074E00010B50B4B0B4A044603F1540103F148005D
:1074F0002360C4F89000C4F89410C4F8982004F1F4
:10750000940004F011FC204604F0D6F8204610BD8B
:1075100088A60500108A0500A0F19800E0E700BFEA
:10752000A0F19400DCE700BF10B5084B044603F15E
:10753000300103F148022360616040F8082F04F035
:10754000F3FB204604F0B8F8204610BDF0A3050078
:10755000A0F10800E8E700BF38B50E4B044603F180
:107560005C0503F1680103F1800284E82800A16052
:1075700040F89C2F04F0D8FB074B204603F14C0148
:1075800003F1580223606160A26012F0C9FD204639
:1075900038BD00BF708F050090A20500A0F19C00CF
:1075A000FFF7DABF10B5034B0446036005F0C0FCDB
:1075B000204610BD3084050010B5054B044603601D
:1075C00005F0B6FC204604F077F8204610BD00BF59
:1075D0003084050038B50F4B044603F15C0503F118
:1075E000680103F1800284E82800A16040F89C2F24
:1075F00004F09AFB084B204603F14C0103F15802BA
:1076000023606160A26012F08BFD204604F054F804
:10761000204638BD708F050090A20500A0F19C00A7
:10762000D8E700BF2DE9F043BA4CA5B004F10A0534
:10763000204601F00DFA20460021023401F010FA34
:10764000AC42F5D1A82040F00DFE044601F0ACFF9D
:10765000B14AB24B12686068A3FB02120368920C35
:107660009B68AF4998476A46AE4903A841F00CFCB5
:1076700003A861682DF0AEF9039BAB4FA3F10C009A
:10768000B84240F00882A94814F064F9D0F1010929
:1076900038BF4FF00009B9F1000F00F0F281A44D9E
:1076A0005421286803F0E8FE064627F0FBFC31462B
:1076B000204602F0E7FC0821286803F0DDFE0646BC
:1076C00029F028FF3146204602F0DCFC142128680E
:1076D00003F0D2FE064629F025FA3146204602F094
:1076E000D1FC1021286803F0C7FE06462CF0FCFEF2
:1076F0003146204602F0C6FC012040F0B3FD0646AC
:1077000023F0F2FB304603F0D7FF012040F0AAFD42
:10771000064615F0ADFE304603F0CEFF012040F0E6
:10772000A1FD06461AF05EFC304603F0C5FF482175
:10773000286803F0A1FE064623F01CFD31462046D2
:1077400002F0A0FC2C2040F08DFD06461BF0D6F880
:107750003146204602F096FC4FF48871286803F009
:107760008BFE06462AF032FF3146204602F08AFCA4
:107770003821286803F080FE804604F0E5FA6D4B5E
:10778000404640F81C3B00F0F5FA98F834300026EB
:1077900066F3041388F834304146C8F82460C8F80A
:1077A0002860C8F82C60204602F06CFC1021286884
:1077B00003F062FE027B002366F300020273436063
:1077C00083600660804604F0BFFA5B4B4146C8F810
:1077D0000030204602F056FC0421286803F04CFEDD
:1077E000804604F0B1FA554B4146C8F800302046B7
:1077F00002F048FC402040F035FD804610F092FC3D
:107800004146204602F03EFC1821286803F034FE71
:1078100080461AF08DFC4146204602F033FC2021C0
:10782000286803F029FE804615F084FA4146204678
:1078300002F028FC282040F015FD314680462BF050
:10784000F9FF4146204602F01DFC3D4807F06EF866
:1078500020463C4902F016FC20463B4902F012FC4F
:10786000324633464EF6D321606903F085FC31463B
:1078700004F040FA04F028FA002840F0F3800022D7
:10788000134644F20901606903F076FC002104F01C
:1078900031FA04F019FA002840F0D680002213468D
:1078A0004DF2BD11606903F067FC284904F02EFA1F
:1078B00004F064F92649054642F02EFB002869D001
:1078C000042040F0CFFC23490646284642F068F9E0
:1078D00042F068FB00220146304604F0D7F83146FA
:1078E000204602F0CFFB284641F0C6FC66680246FF
:1078F00035680B46AD6830461749A84720461749FA
:1079000002F0C0FB606903F0F7FB94F8A430DB07DA
:1079100046D425E0A40200109801001083DE1B432A
:10792000F08105000CE905005C0A001000C007208A
:10793000FC02001050C2050080D9050088A805008F
:1079400020C00720C8C007203CC2072000002041FB
:10795000CDCCCC3D002474492C820500BCC007204E
:10796000B9F1000F27D1524C2368DA68986992F870
:1079700070110DF01DF92368986A04F0BFFB2368AD
:10798000586A03F0E3FF2368D86808F0DFFF25B0EA
:10799000BDE8F0836068474903689B689847ADE796
:1079A0000121454801F05CF84448494601F058F887
:1079B000B9F1000FD7D04248424945F077FB06465F
:1079C0000028D0D06068404903683D4A9B689847CA
:1079D000DFF808818421324603A845F059FA24AD26
:1079E0003A4903AA38B3606803689B6898479DF8D2
:1079F0000C3003A93B2B6A464FF0000E02A8E9D0D9
:107A000045F88C8DCDF808E041F03EFA20462A4634
:107A1000012102F057FB029BA3F10C00B842D9D020
:107A200053F8042C511E002A43F8041CD2DC69468A
:107A300040F084FFCEE76068254903689B6898475B
:107A4000304645F091F88EE728684C2103F014FD8C
:107A50002049054606F070FDCDB1291D204602F0F3
:107A600011FB1BE7C021286803F006FD19490646F3
:107A700014F0CAFA6EB106F19401204602F002FB3E
:107A8000FDE66068144903689B68984707E6294645
:107A9000E4E73146F1E753F8042C511E002A43F87D
:107AA000041C3FF7F0AD01A940F048FFEBE500BF33
:107AB000E402001050820500A4020010AA02001087
:107AC00070820500D415060084820500AC82050092
:107AD000B482050020C007200C82050010030010AE
:107AE00070B5FFF79FFD0D4C0025264620686A1CE7
:107AF00090F8A43092B2DB0706D5C5F300310848F0
:107B0000154600F0ADFF306800210A4602F0DAFAAF
:107B100020680321002202F0D5FAE7E7E402001012
:107B2000A6020010F0B52B4B2B4C83B02B4E0093CC
:107B3000204601332A492B4A13F092FB04F1200519
:107B400032462949204640F0B2FB284607F01AF891
:107B500004F5D47732462846244940F0A8FB29464C
:107B6000384614F051FA32463846214904F1C0072C
:107B700040F09DFB29462246384612F043FE32462D
:107B800038461C4904F51A771B4D40F090FB2246FD
:107B900038461A4901F0D0F932463846184940F0C3
:107BA00086FB2846174900F047FFA81C164900F03D
:107BB00043FF281D154900F03FFFA81D144900F0A0
:107BC0003BFF144905F1080003B0BDE8F04000F0A8
:107BD00033BF00BF06C0092000C00720C800001046
:107BE00009C0092008C0092041740000597500002F
:107BF0005574000099740000A4020010D48205009E
:107C0000A575000032C0092033C0092034C0092006
:107C100035C009209CC0092010B44379002B2FD116
:107C200003790F2B19D802225B0002FA03F3504AA2
:107C30000124116C0B4313640379116CA34004FA03
:107C400003F321EA030313644379CBB903790F2BC0
:107C500003D800205DF8044B704702225B0002FA53
:107C600003F3434A0124516C0B4353640379516C71
:107C7000103BA34004FA03F321EA0303536443795E
:107C8000012B1DD0022B48D0032B5BD0042BE0D15D
:107C900003790F2BDDD95B0002229A40344B01247B
:107CA000596E0A435A660279596E103AA24004FA94
:107CB00002F221EA020200205A665DF8044B704786
:107CC00002790F2A14D80221520001FA02F228493F
:107CD0008C6C22438A6404798A6C6400A34022EA93
:107CE00003038B644379012BCCD102790F2AB0D9DD
:107CF0000223520003FA02F21D4B0124D96C0A43FD
:107D0000DA640279D96C103AA24004FA02F221EA4C
:107D10000202DA644379022BB6D102790F2A98D88D
:107D200052009340124A0124116D0B4313650379ED
:107D3000116DA34004FA03F321EA030313654379A9
:107D4000032BA3D103790F2B83D95B0002229A4026
:107D5000074B0124D96D0A43DA650279D96D103ACF
:107D6000A24004FA02F221EA0202DA6543798DE7C1
:107D700000C00240827910B402F0FE0220246FF3AA
:107D8000410200210471827101605DF8044B70476B
:107D900010B5837904469B0714D543793BB9037921
:107DA00001229A401B4B996E0A439A664379012B34
:107DB00012D0022B19D0032B21D0042B04D0204643
:107DC000FFF72AFF204610BD237901229A40114B6C
:107DD000996F0A439A67F2E721790E4A8B40D16E78
:107DE0000B43D3666379022BE5D1237901229A40B4
:107DF000084B196F0A431A676379032BDDD1237986
:107E000001229A40034B596F0A435A676379042B46
:107E1000D5D1D9E700C00240837930B49B071ED585
:107E20004379F3B1012B4BD0022B00F08B80032B55
:107E300072D0042B13D103790F2B10D95B000122D0
:107E40009A404A4B0224596E0A435A660279596E87
:107E5000103A520004FA02F221EA02025A6630BCD9
:107E6000704703790F2B16D801225B0002FA03F347
:107E70003E4A0224116C0B4313640379116C5B00BE
:107E800004FA03F321EA030313644379002BC9D1F5
:107E900003790F2BE3D901225B0002FA03F3334A83
:107EA0000224516C0B4353640379516C103B5B000B
:107EB00004FA03F321EA030353644379012BB3D19A
:107EC00002790F2A14D852009340284902248D6C5D
:107ED0002B438B6403798A6C5B0004FA03F322EA78
:107EE00003038B644379012B9ED102790F2AB6D903
:107EF0000123520003FA02F21C4B0224D96C0A43FC
:107F0000DA640279D96C103A520004FA02F221EADA
:107F10000202DA64437987E703790F2B9FD95B006C
:107F200001229A40114B0224D96D0A43DA65027985
:107F3000D96D103A520004FA02F221EA0202DA651F
:107F4000437976E702790F2A89D8520001219140BE
:107F5000064A146D214311650479116D6400A34034
:107F600021EA03031365437961E700BF00C00240C3
:107F7000837910B49B0716D54379BBB1012B34D05C
:107F8000022B5DD0032B4ED0042B0CD103790F2B89
:107F900009D9103B03225B0002FA03F32F4A516E0A
:107FA00021EA030353665DF8044B704703790F2BF6
:107FB0000ED803225B0002FA03F3284A116C21EA6F
:107FC000030313644379002BD8D103790F2BEAD92B
:107FD000103B03225B0002FA03F3204A516C21EAB2
:107FE000030353644379012BCAD103790F2B0ED8B5
:107FF00003225B0002FA03F3184A916C21EA03039F
:1080000093644379012BBBD103790F2BCBD9103B60
:1080100003225B0002FA03F3104AD16C21EA030346
:10802000D3644379ACE702790F2ABCD9103A5200E5
:1080300093400A49CC6D24EA0303CB654379A3E757
:1080400003790F2BAFD803225B0002FA03F3034A34
:10805000116D21EA03031365437993E700C00240E1
:10806000837910B49B0715D54379B3B1012B31D077
:10807000022B57D0032B49D0042B0BD103790F2BA4
:1080800008D9103B03225B0002FA03F32C4A516E1D
:108090000B4353665DF8044B704703790F2B0DD8E3
:1080A00003225B0002FA03F3254A116C0B431364AD
:1080B0004379002BDAD103790F2BEBD9103B032244
:1080C0005B0002FA03F31E4A516C0B43536443797D
:1080D000012BCDD103790F2B0DD803225B0002FABF
:1080E00003F3174A916C0B4393644379012BBFD17F
:1080F00003790F2BCED9103B03225B0002FA03F366
:108100000F4AD16C0B43D3644379B1E702790F2A4C
:10811000C0D9103A520093400949CC6D2343CB6536
:108120004379A9E703790F2BB4D803225B0002FA45
:1081300003F3034A116D0B43136543799AE700BFBC
:1081400000C002402DE9F0410F4686B004464A497E
:10815000384640F083FB38B9A37960F34103A3713B
:10816000204606B0BDE8F081444E01AD0FCE0FC5EC
:10817000A279D7F800803368002142F0020206AFEE
:1081800047F8181DA271694640460A222B6046F046
:1081900099FE009BC0B2434560710AD9042808D8F3
:1081A00006AA02EB800050F8142C22601A782E2ABE
:1081B0000FD0A27900230199202002F0FD0263F381
:1081C000000220712046A2716371216006B0BDE8F3
:1081D000F0815D1C0A2269462846009546F072FE31
:1081E000009AC0B295422071E3D21F28E1D8012342
:1081F00003FA00F02368196921EA00011961107877
:1082000088B9ADE76F2827D0762820D05E2828D0FF
:1082100002F06CF90028A3D0009A134601320092B4
:10822000587800289CD040280CD0EBD821281DD0AD
:108230002D28EDD1A3799B07EFD52046FFF7ECFC65
:10824000009AEAE72046FFF7E7FD009AE5E72046B7
:10825000FFF706FF009AE0E72046FFF799FD009A36
:10826000DBE72046FFF784FE009AD6E7A37943F0C8
:108270000103A371D1E700BFEC820500D88205009D
:1082800010B54379012B13D0022B27D0032B0DD12E
:108290000379192B49D01A2B08D108203FF0E2FFAF
:1082A0004A4904463EF01CFE204610BD002010BD89
:1082B0000379122B42D0142B49D0152B50D0172BF9
:1082C0002AD0182B55D01A2BF0D108203FF0CAFF26
:1082D0003F4904463EF004FE204610BD037993B1A9
:1082E000012B4FD0022B56D0032B5DD0042B64D032
:1082F000052BDBD108203FF0B5FF364904463EF0A0
:10830000EFFD204610BD08203FF0ACFF3249044687
:108310003EF0E6FD204610BD08203FF0A3FF2F49A8
:1083200004463EF0DDFD204610BD08203FF09AFFD8
:108330002B4904463EF0D4FD204610BD08203FF0F6
:1083400091FF284904463EF0CBFD204610BD082091
:108350003FF088FF244904463EF0C2FD204610BD90
:1083600008203FF07FFF214904463EF0B9FD20463A
:1083700010BD08203FF076FF1D4904463EF0B0FDD9
:10838000204610BD08203FF06DFF1A4904463EF01C
:10839000A7FD204610BD08203FF064FF16490446A3
:1083A0003EF09EFD204610BD08203FF05BFF1349C4
:1083B00004463EF095FD204610BD08203FF052FFD8
:1083C0000F4904463EF08CFD204610BD7AC00920BE
:1083D0003AC0092045C0092040C0092037C0092003
:1083E00079C0092032C0092034C0092035C00920D5
:1083F00038C0092041C0092042C0092043C00920DB
:1084000044C0092038B503468079C0F3400080B1EC
:108410001A79012191401A68106820EA010111605F
:10842000587910F0FD0F05D09A7900206FF34102C2
:108430009A7138BD19793EF067FC054660203FF01F
:1084400011FF294604463FF0F7F8204638BD00BF2B
:1084500038B5084B05280C461B680ADC80011D183E
:10846000A91D281D3E22C4F30B1445F04BFAA5F8B4
:10847000424038BDB002001038B5094B04464C20CC
:108480001C603FF0EFFE082205464FF47A7105F0BC
:10849000EFFC28462560034905F0A6FF204638BDBD
:1084A000B0020010518400000B68134A934205D0BB
:1084B000124A93420FD04FF0FF3070470B79172BC1
:1084C00012D0182B12D0192B12D00D481A2B18BF0E
:1084D0004FF0FF3070470B791E2B0BD009481F2B34
:1084E00018BF4FF0FF307047074870470748704784
:1084F000074870470748704700C0092020C009207E
:108500001AC009203FC0092017C0092018C009203F
:1085100019C009203EC0092038B50446FFF7C4FF42
:1085200005460146206805F0CFFD04EB801040228F
:108530000021043045F001FA2068012105F0FAFE1F
:1085400020682946012205F0CBFD2068294601223A
:10855000BDE8384005F010BF88422DE9F04781465C
:108560008A462BD0851CA94228D0074637F8026FCF
:10857000B9F800302C46B34205F1020810D837F89C
:10858000023C9E4207D2AA1E2380154632F8023DC5
:108590002C469E42F8D3D0452E800FD04546E5E7C5
:1085A000C9EB07035B1005D05A00C2EB080049462F
:1085B00045F0A8F9D045A9F80060EFD1BDE8F087F3
:1085C0002DE9F00102F1FF3808EBD8784FEA68088E
:1085D0004145B8BF0C464CDA651C6C0004F10046FE
:1085E000013E30F816C030F825602746B4450744F0
:1085F00000EB850504D9013C30F8146000EB44051C
:10860000444527F8026CE7DBD60705D4023A02EBB3
:10861000D272B4EB620F20D0621E02EBD2728C4297
:108620004FEA620215DD30F81260B34206D810E05E
:1086300030F815601446B34209D92A46551E05EB99
:10864000D575914220F814604FEA6505F0DB00EB28
:1086500042052B80BDE8F00170470134640004F14D
:108660000042013A30F81220013C2A8000EB440518
:10867000D2E700EB41050C46C6E700BF2DE9F84FF5
:108680000B1A212B8246934640F39380002A6BD02D
:1086900000F102099B103AF81320BAF802400BF1DE
:1086A000FF3B944231F8020C44D2824246D38442CA
:1086B00051D2BAF80050AAF8000021F8025CBAF8CA
:1086C0000260BAF80040A6420F464B461DD2023364
:1086D000984633F8026BA642FAD3A542A7F10203EB
:1086E00018D93B1F1F4633F80259A542FAD8B8459E
:1086F00013D2434623F8025B3E80B8F80260BAF812
:10870000004037F8025CA642E1D3A5429846A7F1A3
:108710000203E6D81F46B845EBD340465A46FFF75A
:10872000ADFFCAEB0803212B41DDBBF1000F1CD0CC
:108730004146AFE784420ED38242BAD3BAF8000072
:10874000AAF800202AF81300BAF8026031F8025C97
:10875000BAF80040B7E7BAF80060AAF80040AAF8F3
:10876000026031F8025CAEE788465E10B41E641009
:10877000651C0AEB450500E0013C504621463246A7
:1087800035F8023DFFF71CFF002CF5D1BAF80020A8
:1087900038F8023C28F8022DCAEB08046210504653
:1087A0000021FFF70DFF032CF0DCBDE8F88FBDE8DA
:1087B000F88FBDE8F88F00BFF0B591B00446FFF721
:1087C00073FE0146206805F07FFC064672B604EB96
:1087D00080131C1D03F1440E6F4620686168A26877
:1087E000E3683D460FC5103474452F46F5D162B697
:1087F0000A22684610A9FFF741FF684608A9FFF75B
:10880000ABFE0FAF07A88588041D30F8023FAB42CE
:1088100034D902462380114632F8023D0C469D426F
:10882000F8D3B8420D80EED10DF12E000DF10E03FC
:10883000002233F8021F83420A44FAD112499208F7
:1088400001EBC6039C885888DC80988031F836405C
:1088500090B25C8021F8362059889A880844DB88D9
:108860001044184441F048F94FF07A5141F098F91A
:1088700042F0D6F941F096FB11B0F0BD2146B84266
:108880000D80C0D1D0E700BFB40200102DE9F04741
:108890000F4605462C782E462046013544F0A6FFAB
:1088A0000028F7D12D2C334661D02B2C04BF5C78E7
:1088B0002E464FF00108A4F13002092A23465AD867
:1088C000721C0020147800EB8000A4F1300103EB4F
:1088D0004000092916462346A0F1300002F10102AA
:1088E000F0D941F005F981462E2C08D007B13E6041
:1088F000B8F1000F38D109F10040BDE8F087727877
:10890000701CA2F13003092B38D80023B11C184683
:108910004FF0010A072B0E4603F1010301F101019B
:1089200008DC00EB800002EB40000AEB8A0A3038DA
:108930004FEA4A0A3278A2F13004092CEAD940F011
:1089400079FC044650460D4640F074FC02460B4646
:108950002046294640F00EFE40F0C4FF014648463E
:1089600041F016F88146C1E74846BDE8F0872E463B
:108970005C7880469FE74FF00009B5E70021064686
:10898000EDE700BF012070474FF0FF30704700BF98
:108990000120704710B5054B0446036040683BF06A
:1089A0003BFB034B2046236010BD00BF0083050046
:1089B000108A0500064B10B50446036040683BF082
:1089C0002BFB044B2046236002F076FE204610BDB0
:1089D00000830500108A050038B540680D460A4935
:1089E00044F064FB044670B1284645F000FB0121C9
:1089F00002462346284644F0ADFE0546204644F094
:108A0000B3F8284638BD38BDF082050010B582B0F5
:108A1000047841780023022268468DF800408DF8E2
:108A200001108DF802308DF804308DF80320FBF72B
:108A300051FF02B010BD00BF10B5C1F3421301F0E9
:108A40001F01044603704170FFF7E0FF204610BD90
:108A500041780122007802FA01F1FBF76FBB00BFF9
:108A600010B543780C460121007899401CB9FBF7FA
:108A700081FB204610BDFBF773FB204610BD00BFF5
:108A8000014B0360704700BF2883050010B5034BFE
:108A90000446036002F010FE204610BD2883050046
:108AA000F0B50B6887B01A780C46232A71D053F8BA
:108AB0000C3C022B6DD908460022474902233FF0A7
:108AC000B4FE461C054664D023681B5C232B60D093
:108AD0000223204640492A463FF072FE431C0746C7
:108AE00053D03D4920463A4602233FF09EFE0646BB
:108AF0000130216850D08B5D232B4DD051F80C2CC8
:108B00007B1B95424ED82A46214602A840F078F9B0
:108B100002A904A801F034FC14203FF0A3FB054691
:108B200002F0FCFFBDF81010BDF81220BDF81430A3
:108B30000120A874A981EA812B82721C052320469A
:108B400026493FF03DFE421C226818BFC6EB0003D9
:108B500052F80C2C08BF0346964223D821463246D1
:108B600003A840F04DF9284603A93FF0C4FD039B3C
:108B70001B4CA3F10C00A04217D1029BA3F10C00E7
:108B8000A0421DD1284607B0F0BD2168154844F029
:108B900087FF002007B0F0BD134844F081FF00209C
:108BA00007B0F0BD114840F0FCF953F8042C511EF9
:108BB000002A43F8041CE0DC01A93FF0BFFEDCE71B
:108BC00053F8042C511E002A43F8041CDADC03A9D4
:108BD0003FF0B4FED6E700BF48830500A883050038
:108BE0005C0A00104C830500B083050090830500EB
:108BF00038B51546FFF754FF044618B128462146FC
:108C000000F0A0FA204638BDF0B583B014460F46F8
:108C100001AA19491E46054640F036F92146384654
:108C2000FFF73EFF044660B1828933889A420BD039
:108C30002368124AA3F10C00904212D1204602F0A0
:108C40003BFD284603B0F0BDC28973889A42EFD13C
:108C5000B388028A9A42EBD12846214640F093F825
:108C6000E6E753F8042C511E002A43F8041CE5DC07
:108C700001A93FF063FEE1E70CE905005C0A001082
:108C8000704700BF704700BF704700BF704700BF0C
:108C9000704700BF704700BF704700BF704700BFFC
:108CA000704700BF704700BF10B5034B0446036018
:108CB00003F03AF8204610BDE883050010B5054BD7
:108CC0000446036003F030F8204602F0F5FC20462D
:108CD00010BD00BFE883050010B5044603F034F86A
:108CE000201DFFF747F806480023FF214FF0FF3211
:108CF0002060E160226123766361204610BD00BFE1
:108D0000E8830500002905DBC3689942A8BF19461E
:108D10000161704700210161704700BF036981F361
:108D20000801002BC16004DB9942B8BF0B46036108
:108D30007047002303617047C0687047837A4FF023
:108D4000FF3202619A070CD503F001038B42037ACC
:108D50004FF0010202FA03F2436801D09A617047B2
:108D6000DA617047026930B4FF2A034624D8002A2A
:108D70002FD0FF2A40D044696FF0FF05B4F5007F83
:108D8000B4BF20464FF400701C7EA842B8BF2846EE
:108D90005861A4B902447F2A5A612ADC9A7A900762
:108DA0000AD502F00102A2421A7A4FF0010000FA3D
:108DB00002F25B6819D09A61084630BC7047A2F590
:108DC000807210440028D8BF00245861D8BF1C7698
:108DD000E4E7827A9507EFD512F0010F027A4FF09F
:108DE000010000FA02F25B68E5D130BC0846DA61A6
:108DF000704701241C76D1E7827A9407DCD512F003
:108E0000010F027A4FF0010000FA02F25B68D2D043
:108E1000EBE700BF024900220160C260704700BF5B
:108E20002084050010B5044A002304460260C36094
:108E300002F042FC204610BD20840500F0B587B04A
:108E40009DF81440104F04F0FE04104EADF80800D9
:108E5000ADF80A10ADF80C20386801AA6FF3410490
:108E600005211D4604938DF81440019601F02AF95E
:108E70009DF8142012F0010003D0930744BF049B17
:108E80002B6007B0F0BD00BFE40200102084050095
:108E900070B586B09DF814500D4E0E4C05F0FE05D1
:108EA000ADF80800ADF80A10ADF80C20306845F0B8
:108EB0000205062101AA04938DF81450019401F0D3
:108EC00001F99DF8140000F0010006B070BD00BF6C
:108ED000E40200102084050008B5D0F844020368BD
:108EE0009B68984708BD00BF08B5D0F844020368E6
:108EF0009B69984708BD00BF08B5D0F844020368D5
:108F00001B68984708BD00BF08B5D0F84402036845
:108F10005B68984708BD00BF08B5D0F844020368F5
:108F20001B6A984708BD00BF08B5D0F84402036823
:108F3000DB68984708BD00BF38B50446154604F005
:108F4000B9F8034BC4F844522360204638BD00BF33
:108F50003084050010B50021044690F840020DF061
:108F600081FE94F8400204F110010DF07BFE002018
:108F700010BD00BF0022026042608260704700BFE7
:108F80002DE9F04190E86000B54282B080461CD0E7
:108F9000154F55F8044B3CB12368A3F10C02BA42BB
:108FA00015D1204602F088FBAE42F2D1D8F800007D
:108FB0000023C8F80030C8F80430C8F8083008B1F9
:108FC00002F07AFB02B0BDE8F0812846F0E753F8E2
:108FD000041C481E002943F8040CE2DC104601A9D9
:108FE0003FF0ACFCDDE700BF5C0A001010B50446A2
:108FF000FFF7C6FF206808B102F05EFB204610BDF7
:1090000010B5436882B053F8044D436044B12368FF
:109010000A4AA3F10C00904204D1204602F04CFB16
:1090200002B010BD53F8042C511E002A43F8041C52
:10903000F3DC01A93FF082FCEFE700BF5C0A0010FF
:10904000F8B590E85000B4420F4602D10DE0A642B8
:109050000BD054F8045B384605F10C01062244F0AD
:1090600039FC0028F3D12846F8BD00252846F8BD74
:109070002DE9F04F90E820024D458BB00F4624D0EB
:10908000012600E0464655F8044BD7F800A0E389D6
:10909000B4F80CB00093238A06F10108019322680A
:1090A0000292A37C0393E37C0493A06840F0E4F86D
:1090B000CDE9060162685B460892DAF80840384656
:1090C00003493246A047A945DCD10BB0BDE8F08F7B
:1090D00068840500F8B5426803680446D31A9B10FB
:1090E0000F4605D05A00934226D96FF0030600E0E0
:1090F000042630463FF0B6F8054694E809001B1AEE
:109100009B109A003968AF1807D045F8231094E8EF
:1091100009001B1A9B109A00AF1823B1014628467C
:1091200044F0F0FB2068043708B102F0C5FA2E4481
:10913000A66084E8A000F8BDB2F1804FD5D2DE0071
:10914000D7E700BF2DE9F04790E8A00084B0BD420A
:109150008146019124D08A4601F10C0801E0AF421A
:109160001ED02E68404606F10C0106222C4604351E
:1091700044F0B0FB0028F2D156B13368184AA3F18D
:109180000C00904220D1304602F096FADDF804A09F
:10919000C4F800A0134844F037FD04B0BDE8F087E0
:1091A000D9F808309F420AD0019B17B13B60D9F82B
:1091B00004700437C9F8047004B0BDE8F08748466D
:1091C00001A9FFF787FFE8E753F8042C511E002A96
:1091D00043F8041CD7DC03A93FF0B0FBD3E700BF82
:1091E0005C0A0010C4840500F8B5426803680446B0
:1091F000D31A5B100F4605D05A00934221D96FF065
:10920000010600E0022630463FF02CF8054694E8BF
:1092100009001B1A5B1039885A00AF1818BF25F8CF
:10922000131043B9023708B102F046FA2E44A66083
:1092300084E8A000F8BD0146284644F063FB20689E
:10924000F0E7B2F1004FDAD29E00DCE72DE9F04101
:1092500090E89000BC4282B0884602D114E0A74258
:1092600012D054F8045B2E8A9642F8D1AE89464556
:10927000F5D1596898688E1C814208D0E88901B1FF
:109280000880A7425E60ECD102B0BDE8F0811846CC
:1092900005F10E0101920093FFF7A6FF009B019AD2
:1092A000DDE700BF38B5094B094D044603600246AF
:1092B0000721286800F066FF28682246082100F090
:1092C00061FF204602F030FD204638BDF8840500DD
:1092D000E402001010B50446FFF7E4FF204602F058
:1092E000EBF9204610BD00BF012919D041B1CB07D1
:1092F00015D490F83830022202FA03F319420ED046
:10930000837E9A070BD513F0010F037E4FF0010205
:1093100002FA03F2436901D19A617047DA6170473A
:10932000837E9A07FBD5027E13F0010F01FA02F14A
:10933000436914BF9961D961704700BF01B170479B
:10934000837E9A070AD513F0010F037E4FF00102C6
:1093500002FA03F243690CBF9A61DA61038F6FF37B
:1093600049230387704700BF2DE9F0411E4604469C
:109370001746884602F0E8FC344B254645F8043B86
:1093800098E8030085E8030004F10C0397E8030064
:1093900083E8030004F1140396E8030083E8030064
:1093A000B3799F0703D57079317902F0AFFD0023BF
:1093B000E362228FA17E63F34922228794F8392049
:1093C0000025234E42F0040222484FF07E5763F3FB
:1093D000C30265638D07236384F8392027626662C0
:1093E000A06207D5237E01229A406369C80754BF53
:1093F0009A61DA61A37A99070AD513F0010F237AEB
:109400004FF0010202FA03F2636814BF9A61DA6155
:10941000A37C9A070AD513F0010F237C4FF00102B9
:1094200002FA03F2E36814BF9A61DA61238F2046DF
:109430006FF308232387072102F08CFC20460821C4
:1094400002F088FC2046BDE8F08100BFF8840500EA
:10945000000048420000C07F10B504460162084683
:10946000616B40F09DFB41F0ADFB2063E06210BDFD
:1094700010B5044641630846216A40F091FB41F073
:10948000A1FB2063E06210BD41630263C2627047CA
:10949000036B41631A440263704700BF10B5044672
:1094A0000846216A40F07CFB41F08CFB236BC01A1C
:1094B00010BD00BF38B5837E04469A070D460FD510
:1094C0004269017E506903F00103C84000F00100C9
:1094D000984205D0002B47D0012303FA01F1916196
:1094E00094F8393003F00103AB4215D0238FA27CEE
:1094F00065F30823900723870BD5237C02F0010234
:10950000AA424FF0010202FA03F2E36814BF9A6123
:10951000DA6101203DF0E4FEA37A99070AD513F041
:10952000010F237A4FF0010202FA03F263680CBFC5
:109530009A61DA6103203DF0D3FEA37A9A070AD537
:1095400013F0010F237A4FF0010202FA03F263686D
:1095500014BF9A61DA61E26A002D0CBF01234FF05B
:10956000FF331344E36238BD012303FA01F1D161F3
:10957000B6E700BFF8B5046900F10806B4420F462B
:109580004FF000050DD02069394603685B699847A4
:109590008542B8BF054620463EF012FFB042044661
:1095A000F1D12846F8BD00BFF8B5324B044603633D
:1095B00000F1B00100F14403002243F80C2C43F801
:1095C000082C43F8042C0C338B42F6D194F8A430C9
:1095D000294A03F0D50343F040036FF3C71384F81F
:1095E000A4301C2014603EF03DFE0021054606F02C
:1095F00017FD4FF416512846256006F04FFD102048
:109600003EF030FE054601F00DFE28466561012161
:1096100001F080FD206810B103685B689847002561
:1096200025601C203EF01EFE1449034600F108028E
:109630000160026142610572C56085611049636025
:10964000012204F130003FF025FA0E4A4FF2FF03E9
:10965000D1680B4043F0BF6343F40033D3603BF069
:1096600033FF032800F24F81DFE810F0350141019C
:1096700029010E00680A0010E40200103085050080
:109680005085050000ED00E0A54B1C21186801F095
:10969000F3FE03210646354606F0C2FC2660002D87
:1096A00000F033810022134660694CF6DF1101F0AF
:1096B00063FD002102F01EFB02F006FB94F8A430CB
:1096C00080F00100002260F3000384F8A430606998
:1096D000134648F2AE0101F04FFD002102F00AFBF3
:1096E00002F0F2FA94F8A430002260F3820384F8C6
:1096F000A4306069134643F6662101F03DFD94F8FD
:10970000A4102026C1F3800102F0F4FA02F0DCFA82
:1097100094F8A430002260F3451384F8A430606903
:10972000134645F68B3101F027FD012102F0E2FAE4
:1097300002F0CAFA236894F8A420196860F30412AE
:1097400084F8A42018468A68904728203EF08AFDB5
:10975000054602F093F82B6865629B682846984797
:109760003C203EF07FFD054602F014FDA5624FF45B
:10977000C2703EF077FD0746FEF77EFE694A4FF263
:10978000FF01D068684B014041F0BF614FF0100C01
:109790004FF0080E282541F400311820E762D1600F
:1097A00083F801C383F802E383F8036383F8046357
:1097B00082F8220083F8165383F8185393F8052390
:1097C00045F29E51D20818BF83F80553564B93F8C3
:1097D0000623D2081CBF282283F80623524B93F895
:1097E0000723D2081CBF282283F807234E4B93F887
:1097F0000823D2081CBF282283F80823002213461E
:10980000606901F0B9FC494902F074FA02F0B6F956
:1098100040F0C8FB0022134660634AF25D51606964
:1098200001F0AAFC012102F065FA02F0A7F9054651
:10983000606B40F05DF9A66A0146304602F06CFCB0
:109840002946A06A02F086FC2C203EF00BFD05465E
:109850000BF080F92B68A5619B6828469847182073
:109860003EF000FD054606F03BFA2B68A5609B68BC
:10987000284698474FF4BA703EF0F4FC054609F0CC
:10988000C7FB2B68E5609B682846984704203EF09C
:10989000E9FC054602F058FA254B28462B60256264
:1098A0002BF05AF818203EF0DDFC054606F0ECFDE2
:1098B000256101203EF0D6FCE0612046F8BD184B42
:1098C0001C21186801F0D8FD02210646354606F035
:1098D000A7FB2660E3E6124B1C21186801F0CCFDC3
:1098E00000210646354606F09BFB2660D7E60C4B6A
:1098F0001C21186801F0C0FD01210646354606F01E
:109900008FFB2660CBE62568C9E6054B1C2118684D
:1099100001F0B2FD2946064606F082FB2660C1E64C
:10992000FC02001000ED00E000E100E0A086010074
:1099300020FA05002DE9F04FA04BBDB006AF036043
:10994000804689464FF44C4044F68A51002207F184
:109950002F03FFF773FA08B987F82F00002107F1EA
:10996000D80343F8A81D0A4643F61930FFF766FAF4
:109970004046934901223FF07BF999F8A4309E07B5
:1099800000F18A8197F82F20002A40F0AF811D074F
:1099900040F1078140468B4904223FF069F9D9F82C
:1099A0000C40C7F81CD094F870B104F1F8014FEAEC
:1099B0008B0202F10A0303F4FF63ADEB030D0DF11B
:1099C000180A504643F095FF94F83430DAF8005006
:1099D000DB0740F172817C49284640F095F93FF061
:1099E0004BFCDAF80430C7E90401184676493B62BB
:1099F00040F08AF93FF040FCDAF80830C7E900018E
:109A0000714918467B6240F07FF9D7E90423CDE91C
:109A10000023D7E90023CDE902233FF02DFC07F115
:109A20005806CDE90401694A8021304644F0C0F966
:109A300067490446062240463FF01AF9802C34BF9D
:109A40002246802231463FF013F9BBF1030FC8BF15
:109A5000032417DDDAF80C003FF00EFC5D4ACDE977
:109A600000018021304644F0A3F90134802834BF3E
:109A700002468022314640463FF0FAF8A3450AF1FB
:109A8000040AE7DC7B6A07F1400AFB6407F14C0B30
:109A90003B6A5046D9F80C105A463B657D6506F086
:109AA000F9FFD9F80C30B86C93F83430DC0740F18A
:109AB000F980454940F028F93FF0DEFB04460D46A9
:109AC000786C414940F020F93FF0D6FB02460B4646
:109AD000386C3D49BA60FB6040F016F9FB68BA6823
:109AE000CDE90223CDE900453FF0C6FB374ACDE979
:109AF00004018021304644F05BF9374904460622D0
:109B000040463FF0B5F8802C34BF224680223146D3
:109B10003FF0AEF8D9F80C40204607F083F894F8EF
:109B20003430D90702D5284940F0EEF83FF0A4FBC5
:109B3000CDE90001D9F80C302848D3F8381140F0AD
:109B4000E3F83FF099FB264ACDE902018021304637
:109B500044F02EF93146802834BF02468022404628
:109B60003FF086F83B6B002B00F05C82FB699D4662
:109B700099F8A440C4F38004002C63D053464EF6F9
:109B80008F7049F678210022FFF758F970BB4046E4
:109B9000144902223FF06CF84046DC37BD46BDE870
:109BA000F08FD9F818000BF013F8002800F02C8281
:109BB00040460D4904223FF05BF8F0E6680A0010C9
:109BC00054850500688505003333CB417C8505004D
:109BD0009085050098850500A08505000080BB459F
:109BE000E48505001086050070850500396C07F1D5
:109BF000540091E80C000831FA643B653FF0B7F877
:109C0000FA6C3B6D202100923046354A44F0D0F882
:109C10003146202834BF0246202240463FF028F833
:109C20007B6D304AA3F10C009042B0D053F8042C65
:109C3000511E002A43F8041CA9DC07F134013EF050
:109C40007DFEA4E75B4622464AF616404BF2D3114E
:109C5000FC643C657C65FFF7F1F8002840F09C81CE
:109C60003D6DFA6CAA4200F0F381DFF878B014463B
:109C700002F11009A31A59F803301434A3F10C00AF
:109C8000584540F0E981AC42F4D1F86C00283FF42B
:109C900075AF01F011FD71E74046134905223EF012
:109CA000E7FF7CE63FF0E8FA0446786C0D463FF0AB
:109CB000E3FA02460B46386C12E728463FF0DCFA1E
:109CC000DAF80430C7E9040118463B623FF0D4FAE1
:109CD000DAF80830C7E900017B62184695E600BF54
:109CE000048605005C0A00105885050040469F491F
:109CF00004223EF0BDFFD9F80C0007F1340106F054
:109D00009DFED9F80C00C3693BB1036A07F1340129
:109D1000143001229847D9F80C0090F83430786B51
:109D2000DC0740F1168192493FF0EEFF3FF0A4FAC4
:109D300004460D46B86B8E493FF0E6FF3FF09CFAB3
:109D400082468B46F86B8A493FF0DEFFCDE900453D
:109D5000CDE902AB3FF090FA07F15806CDE90401D6
:109D6000844A8021304644F023F883490446062281
:109D700040463EF07DFF3146802C34BF2246802293
:109D80003EF076FFD9F80C1091F87031032B23DDEB
:109D900003240B469B6853F824500134E86A3FF0D3
:109DA000ABFE296A3FF0B0FF3FF066FA734ACDE997
:109DB00000018021304643F0FBFF3146802834BF4C
:109DC0000246802240463EF053FFD9F80C3093F80B
:109DD0007021A242DEDC19467B6BFD6BBC6B07F188
:109DE000400A07F14C0B50465A467B65FD643C65C2
:109DF00006F050FED9F80C30B86C93F83430D9071F
:109E000040F19C805A493FF07FFF3FF035FA04460D
:109E10000D46786C56493FF077FF3FF02DFA024629
:109E20000B46386C5249BA60FB603FF06DFFFB682F
:109E3000BA68CDE90223CDE900453FF01DFA4D4A4D
:109E4000CDE904018021304643F0B2FF4C4904467D
:109E5000062240463EF00CFF802C34BF2246802272
:109E600031463EF005FFD9F818304649586A3FF0B0
:109E700097FED9F80C40054694F83430DA0703D53C
:109E80003B493FF041FF0546204606F0CBFE94F8E3
:109E90003430DB0768D536493FF036FF04462846A4
:109EA0003FF0EAF9CDE9000120463FF0E5F9CDE9C0
:109EB0000201D9F80C303448D3F838113FF024FFB0
:109EC0003FF0DAF9314ACDE904018021304643F010
:109ED0006FFF3146802834BF0246802240463EF064
:109EE000C7FE386B002800F0958018F0A9FF3FF0FE
:109EF000C3F9274ACDE900018021304643F058FFDD
:109F00003146802834BF0246802240463EF0B0FEF3
:109F1000D9F80C30D3F840013FF0AEF91D4ACDE935
:109F200000013046802143F043FF3146802834BF92
:109F30000246802240463EF09BFE19E63FF09CF927
:109F40000446786C0D463FF097F902460B46386C94
:109F50006FE73FF091F90446B86B0D463FF08CF97E
:109F600082468B46F86BF1E6044698E7608505006B
:109F70003333CB417C85050090850500988505002D
:109F8000A0850500000070420080BB45A885050043
:109F9000C0850500CC850500D7F84C903D6DA945DE
:109FA00058D009F1100CC7F820A009F114047D6203
:109FB000CA46E346C9EB0A0354F8140C5BF8035095
:109FC0003FF05AF9CDE9000154F8100C3FF054F974
:109FD0002B46CDE90201284A2021304643F0E8FE15
:109FE0003146202834BF0246202240463EF040FE43
:109FF000796A0AF1140A514504F11404DAD1D7F848
:10A0000020A0FA6C3D6D2DE640461C4903223EF02F
:10A010002FFE70E6D9F80C30D3F840013FF02CF950
:10A02000174A7CE7D9F80C30D3F840013FF024F907
:10A03000134ACDE900013046802143F0B9FE314694
:10A04000802834BF0246802240463EF011FE8DE556
:10A0500010461BE62A4605E653F8041C01F1FF3EB4
:10A06000002943F804EC3FF70EAE3146BA603EF0EB
:10A0700065FCBA6807E600BFF48505007885050031
:10A08000D885050008B50B6808469B68984708BD49
:10A0900090F8A43010B543F002030446806984F8B8
:10A0A000A4300AF081FFE2689368D068834207D049
:10A0B00053F8042B118F98426FF349211187F7D180
:10A0C00010BD00BF2DE9F04F072983B08B468246B3
:10A0D00090463CD0012301930BEB4B0292000AF116
:10A0E0003801881846688C58B4421CD0244F07EBBE
:10A0F000CB02556805F001096D1006E0284457F8B9
:10A100003B2041469047A6420DD054F8040BB9F1CC
:10A11000000FF3D0415957F83B2028448A58414654
:10A120009047A642F1D1BBF1070F02D003B0BDE8C2
:10A13000F08F9AF8A4309B0702D5019B002BF5D134
:10A14000DAF80C0003B0BDE8F04F06F087BF90F8D6
:10A15000A410D2F1010238BF002262F3410180F85D
:10A16000A41032B9C9B2080744BF62F3C3018AF828
:10A17000A410DAF818000AF02BFD0190ACE700BF3C
:10A180009889050001EB410138B538308B00C518BE
:10A190006C68C058A0420DD00368934218BF031DDD
:10A1A00003D108E00168914205D0A342184603F1AB
:10A1B0000403F7D138BD011D8C4206D0631A9A10F2
:10A1C00003D0920043F09EFB6C68043C6C6038BD89
:10A1D00070B50C46064609B90AE02C463046E168DF
:10A1E000FFF7F6FFA568204601F066FA002DF4D1CE
:10A1F00070BD00BF054B10B5044640F8043BE16854
:10A20000FFF7E6FF024B2046236010BD30850500B6
:10A21000108A0500074B10B5044640F8043BE1687E
:10A22000FFF7D6FF044B2046236001F045FA204695
:10A2300010BD00BF30850500108A0500F8B54268E2
:10A2400003680446D31A9B100F4605D05A00934268
:10A2500026D96FF0030600E0042630463EF002F8EF
:10A26000054694E809001B1A9B109A003968AF183C
:10A2700007D045F8231094E809001B1A9B109A0098
:10A28000AF1823B10146284643F03CFB2068043751
:10A2900008B101F011FA2E44A66084E8A000F8BDD0
:10A2A000B2F1804FD5D2DE00D7E700BF00B501EB99
:10A2B0004101383000EB81004368816883B08B42F4
:10A2C000019207D00BB11A6043680433436003B0B6
:10A2D0005DF804FB01A9FFF7B1FFF8E770B405686A
:10A2E0002878F8B10024104E2146084480FB06234C
:10A2F000C217C118C2EBE111C1EB0121411A0C4494
:10A3000084FB0623E2172344C2EBE313C3EB0323CE
:10A3100015F8010FE31A89B29CB20028E5D141EA91
:10A32000042080B270BC70478180808070B4027855
:10A330000AB30024114E21468D1885FB0623EA1727
:10A34000E918C2EBE111C1EB0121691A0C4484FB4D
:10A350000623E2172344C2EBE313C3EB032310F8F5
:10A36000012FE31A89B29CB2002AE5D141EA042404
:10A37000A0B270BC70471046FBE700BF81808080B0
:10A380002DE9F04F0B68002753F80C3C87B0884646
:10A390000190078047808780002B63D04E4CBA46DF
:10A3A000012340464D4952463EF00AFA4C4B0546C1
:10A3B0000493431C5DD0D8F80020CAEB050352F883
:10A3C0000C2C924579D805AE5246304641463EF0B7
:10A3D00017FD04A831463EF08EF9059BDFF8089181
:10A3E000A3F10C0048455DD1DDF810C09CF80030A9
:10A3F00043B34FF0000B5946604601EB030A8AFB5A
:10A4000004230AEB03014FEAEA73C3EBE111C1EB4A
:10A410000121C1EB0A018B448BFB04230BEB0302EC
:10A420004FEAEB73C3EBE212C2EB022210F8013FDA
:10A43000C2EB0B0289B21FFA82FB002BDDD141EA8D
:10A440000B218BB2019AACF10C00D3536A1C1CD0C7
:10A45000484505F1010A33D1D8F8003053F80C3CD7
:10A460009A4502D307B0BDE8F08F0237062FF9D026
:10A4700096E7D8F8003053F80C3C53451DD305AE91
:10A480005246304641462B46A1E74845EAD05CF8A3
:10A49000043C5A1E002B4CF8042CE3DC31463EF001
:10A4A0004DFADFE753F8042C511E002A43F8041C30
:10A4B0009ADC03A93EF042FA96E70A483EF071FDA5
:10A4C0005CF8043C5A1E002B4CF8042CC4DC3146CA
:10A4D0003EF034FAC0E700BF818080807C2C05000C
:10A4E000680A0010908305005C0A0010202804D040
:10A4F000B0F109035842584170470120704700BF2E
:10A50000F0B50F4E83B006600C68054654F80C7C1D
:10A510002744BC4201D10FE02E6814F8010B45F02E
:10A5200055F8C0B256F80C1C0022009001232846B2
:10A530003EF082FAA742EFD1284603B0F0BD00BF3B
:10A54000680A001070B584B00C4602AA1C49064681
:10A5500003A83EF099FC03990022204651F80C3CD8
:10A560003EF063F9421C18BF00250FD001460122BE
:10A57000144B009520463EF0A9FC0399204651F863
:10A580000C3C00223EF051F9431CEFD10E4B039AD4
:10A590002168A3F10C05A2F10C00A84231602360F0
:10A5A00002D1304604B070BD52F8043C591E002B55
:10A5B00042F8041CF5DC02A93EF0C0F9F1E700BF47
:10A5C000148605000CE90500680A001070B50C46F9
:10A5D000012384B005462149204600223EF0F0F8D0
:10A5E000431C06461ED00022334602A821463EF0F8
:10A5F00007FC2368721C53F80C3C9A4220D8214671
:10A6000003A83EF0FDFB204603A93EF074F8039B2F
:10A61000134AA3F10C00904215D1029B28462B60EF
:10A6200004B070BD214603A83EF0A1FB20460D49B1
:10A6300000223EF02FFA039B28462B6004B070BD29
:10A6400009483EF0AEFC53F8042C511E002A43F892
:10A65000041CE2DC01A93EF071F9DEE7C08B0500C5
:10A660005C0A00100CE905009083050030B50D462A
:10A67000012383B004461149284600223EF0A0F889
:10A68000431C0FD02B68421C53F80C1C4B1C8A42F5
:10A69000C0EB03030ED8294620463EF0B1FB20460E
:10A6A00003B030BD2046064901AA3EF0EDFB20462E
:10A6B00003B030BD03483EF074FC00BFC08B050002
:10A6C0000CE905009083050010B50549006842F0CB
:10A6D000EDFC044642F048FA201C18BF012010BDD2
:10A6E000D415060010B590B14FF0804401220E4BF6
:10A6F0002261186800093FF0FBF93FF053FC032189
:10A70000AA225523606021702272237210BDBFF30C
:10A710004F8F064A064BD16801F4E0610B43D360CA
:10A72000BFF34F8FFEE700BF9801001000ED00E07F
:10A730000400FA05F0B5A14D85B02B680C4607461C
:10A7400003F1300102A83EF012FB236853F80C2CF1
:10A75000002A00F09A8053F8042C002A03DB2046DC
:10A760003EF052F923681A782F2A00F0CB80944DDE
:10A7700000220323214603A83EF042FB03A891498F
:10A780003EF06CF8039B0646A3F10C02AA4240F08F
:10A79000C780002E37D1236853F80C3C022B40F2BF
:10A7A000CC804FF0FF332146032203A83EF028FB64
:10A7B000204603A93DF09FFF039BA3F10C00A84294
:10A7C00040F0BE8080494FF0FF32012302A83EF0E6
:10A7D00011F802A90346002203A83EF011FB02A8CB
:10A7E00003A93DF088FF039BA3F10C00A842BFD052
:10A7F00053F8042C511E002A43F8041CB8DC01A9AC
:10A800003EF09CF8B4E700220223214603A83EF064
:10A81000F7FA03A86D493EF021F8039B0646A3F121
:10A820000C02AA4240F0BA80002E35D0029B53F8A9
:10A83000042C53F80C1C002A01F1FF3603DB02A89C
:10A840003EF0E2F8029B9B5D02A92F2B60D003A88B
:10A850003EF08DFA2F22012103A83EF04FFA03A803
:10A8600021463EF0DCF95A4A03683B600260039BD4
:10A87000A3F10C00A84240F08580029BA3F10C00DC
:10A88000A84269D1384605B0F0BD29683846303154
:10A890003EF06DFA4A4DF0E7236853F80C3C012B6B
:10A8A0004BD94FF0FF332146022203A83EF0A8FA0D
:10A8B000204603A93DF01FFF039BA3F10C00A84213
:10A8C00055D141494FF0FF32012302A83DF092FFDC
:10A8D00002A90346002203A83EF092FA02A803A9A7
:10A8E0003DF009FF039BA3F10C00A8429ED053F852
:10A8F000042C511E002A43F8041C97DC01A93EF0E9
:10A900001DF893E7324A3B60A2F10C052260B4E7E0
:10A9100038463EF02CFA384621463EF080F9ACE746
:10A9200053F8041C481E002943F8040C3FF731AFCC
:10A93000104601A93EF002F82BE726483EF031FB15
:10A9400053F8042C511E002A43F8041C3FF73AAF79
:10A9500001A93DF0F3FF35E753F8042C511E002AFE
:10A9600043F8041C8EDC03A93DF0E8FF8AE753F8A6
:10A97000042C511E002A43F8041CA2DC01A93DF05E
:10A98000DDFF9EE753F8042C511E002A43F8041CF7
:10A990003FF773AF01A93DF0D1FF6EE753F8041CF8
:10A9A000481E002943F8040C3FF73EAF104601A9AA
:10A9B0003DF0C4FF002E7FF439AF6DE7E4020010D4
:10A9C0005C0A00103486050050850500D49E050001
:10A9D000680A0010908305002DE9F04191E810010C
:10A9E000444582B0074616461FD002B30834002003
:10A9F00001E0864216D914F8082C451C3A5454F844
:10AA0000040C3EF039FC07EB050E731BCDE9000189
:10AA1000084A7046194643F0CBF9A045284404F192
:10AA20000804E6D102B0BDE8F0810020FAE7104644
:10AA3000F8E700BF3886050030B585B00D4603AA9B
:10AA4000174904463EF020FA052D23680CDC343506
:10AA5000EDB253F80C1C20460095002201233DF076
:10AA6000EBFF204605B030BD392253F80C1C2046C0
:10AA70000092012300223DF0DFFF20460949012218
:10AA80003EF0F6F82B350368EDB253F80C1C0022AB
:10AA9000009501233DF0D0FF204605B030BD00BF3A
:10AAA000408605007C2C050070B505463CF064F836
:10AAB000074E044602E03068FFF704FB3CF05CF808
:10AAC000001BA8424FF003014FF00002F3D370BD0A
:10AAD000E40200104FF47A7303FB00F0FFF7E4BFC9
:10AAE000F8B5426803680446D31A9B100F4605D098
:10AAF0005A00934221D96FF0030600E00426304645
:10AB00003DF0B0FB054694E809001B1A9B1039681C
:10AB10009A00AF1818BF45F8231043B9043708B19D
:10AB200000F0CAFD2E44A66084E8A000F8BD0146EE
:10AB3000284642F0E7FE2068F0E7B2F1804FDAD213
:10AB4000DE00DCE7F8B5426803680446D31A9B10C0
:10AB50000F4605D05A00934221D96FF0030600E05A
:10AB6000042630463DF07EFB054694E809001B1A9A
:10AB70009B1039689A00AF1818BF45F8231043B9E5
:10AB8000043708B100F098FD2E44A66084E8A000C8
:10AB9000F8BD0146284642F0B5FE2068F0E7B2F164
:10ABA000804FDAD2DE00DCE72DE9F0474268036827
:10ABB00082B0C3EB02095FEAA90907460E4648D0F6
:10ABC0004FEA4903994555D96FF0030948463DF0CE
:10ABD00049FB97E83000291B891000EB8103804670
:10ABE00000F1040A23B13368254A40F8213032606D
:10ABF000AC4231D0231DC3EB050C4FEA9C0C04F191
:10AC000008061F4806EB8C06424622B153F8041C86
:10AC1000116043F8040C0433B34202F10402F4D18E
:10AC200008EB8C0C174E0CF1080A54F8043BA3F106
:10AC30000C02B24212D1A542F7D1386808B100F037
:10AC40003BFD08EB0903BB6087E8000502B0BDE8E7
:10AC5000F0874FF00409B9E72046EFE753F8041CEA
:10AC6000481E002943F8040CE5DC104601A93DF01C
:10AC700065FEE0E7B3F1804FA6D24FEAC909A5E728
:10AC8000680A00105C0A00102DE9F04FDFF80C8113
:10AC9000002385B082460F461646036043608360FA
:10ACA000A8F10C093B78B3424FD0002B4DD07B1C50
:10ACB00000E024B11D4613F8014BB442F9D1AF4274
:10ACC00054D0002F3CD0C7EB050B5846002101AAF9
:10ACD0003DF0E4FDBBF1010F044600F10C0328D167
:10ACE0003A7822734C452C4F44D1DAF80420DAF834
:10ACF000081003938A4233D01AB11360274BCDF862
:10AD00000C800432CAF80420A3F10C00B84238D1F8
:10AD10002B786F1C002BC5D1504605B0BDE8F08FD5
:10AD20002846294601AA3DF0B9FDAB46044600F18C
:10AD30000C03184639465A4642F0DBFD0346D1E77C
:10AD4000002DEDD016483EF026F9DAF80420DAF8A6
:10AD50000810124B8A423D460393A3F10C07CBD156
:10AD6000504603A9FFF720FF039BCDE70B4BA3F150
:10AD70000C07BAE70022C4F800B0A26003F80B2069
:10AD8000B3E753F8042C511E002A43F8041CBFDC1F
:10AD900002A93DF0D3FDBBE75C0A0010680A001071
:10ADA00044860500F0B585B004462C2201A8FFF7C3
:10ADB0006BFF019D029E0023B54223606360A36088
:10ADC00029D055F8040B002143F0E2FF6368A26824
:10ADD000009093421AD01A1D03B118606260AE420F
:10ADE000EFD10198029E86420AD0114F054655F8D0
:10ADF000043BA3F10C00B8420FD1AE42F7D1019849
:10AE000008B100F059FC204605B0F0BD2046694667
:10AE1000FFF766FEE3E72846F2E753F8042C511EDD
:10AE2000002A43F8041CE8DC69463DF087FDE4E7AE
:10AE30005C0A0010F0B585B00446174601A82C2224
:10AE4000FFF722FF019D029E0023B542236063604D
:10AE5000A3602AD0002155F8040B3A4644F032F89A
:10AE60006368A16800908B421AD0191D03B1186065
:10AE70006160AE42EED10198029E86420AD0114F27
:10AE8000054655F8043BA3F10C00B8420FD1AE4281
:10AE9000F7D1019808B100F00FFC204605B0F0BDD5
:10AEA00020466946FFF74EFEE3E72846F2E753F8EF
:10AEB000042C511E002A43F8041CE8DC69463DF0CE
:10AEC0003DFDE4E75C0A001010B50B4682B049680E
:10AED000024618686B4603C30B46D90707D55B10BB
:10AEE000D4580099D0186158884702B010BD02EBC1
:10AEF00063000099884702B010BD00BF036E90F850
:10AF000064109A7990070ED502F0010281F00101D8
:10AF10008A421A794FF0010101FA02F21B6801D04E
:10AF20009A617047DA61704770B5856E82B00446E9
:10AF3000002128463EF0DCFF30BB144A144E00923C
:10AF400001906A466061A46103CAE662E061216221
:10AF5000284610493EF024FE3FF024F801462046E2
:10AF60003CF0C0FA236E94F864109A7990070BD5E0
:10AF700002F001028A421A794FF0010101FA02F24D
:10AF80001B6814BF9A61DA6102B070BDFDAE0000AB
:10AF9000C9AE000000247449F8B50D4600270446E8
:10AFA00039462846E66E3EF0A3FF60B93046294692
:10AFB0003EF0F6FDA06628464FF07E513EF0ACFF15
:10AFC00000B1A666F8BDA766F5E700BF70B50E49EB
:10AFD000044682B0C06E3EF0E3FD3EF0E3FF0B4B53
:10AFE0000022054600930A4E01926B4603CBE064B3
:10AFF000216504F130002946A4646264E66502B06C
:10B00000BDE870403CF06EBA0024744929AF0000DE
:10B01000C9AE0000F8B50446194E17460D463CF07F
:10B0200007FD2046002140F8146B3CF025FA154B33
:10B03000204640F8303B3CF0FBFC266304F1440022
:10B0400000213CF019FA2566AB799A070DD503F07B
:10B05000010387F0010293422B794FF0010202FABB
:10B0600003F22B6814BF9A61DA61074A0023204675
:10B0700084F86470E266A366FFF7A8FF2046F8BD77
:10B0800040320600403306000AD7A33C10B5044600
:10B0900008463EF031FD06493EF036FEE0662046A9
:10B0A000FFF794FF2046BDE81040FFF78FBF00BFB9
:10B0B00000007A4410B503680A4A0446A3F10C0064
:10B0C000904282B002D1204602B010BD53F8042C49
:10B0D000511E002A43F8041CF5DC01A93DF02EFCAA
:10B0E000F1E700BF5C0A00100B460068114647F20A
:10B0F0006932FEF7ABB800BF38B5046805462CB11D
:10B100002046FDF773FF204600F0D6FA00232B609F
:10B1100038BD00BFF8B50C460546FFF7EDFF0C2023
:10B120003DF0A0F80746FDF725FF2F606CB16C6875
:10B13000AE68B44209D0394600E0296854F8040BDF
:10B1400003689B689847A642F7D1F8BD10B504681C
:10B150004CB12046FDF774FF00B110BD044800F06B
:10B16000F3FC0348F9E7034842F04EFD204610BDCA
:10B17000E80200107086050000B583B0ADF800103D
:10B180006946ADF80220ADF80430FFF7DFFF03B0E9
:10B190005DF804FBF8B5426803680446D31A9B10B7
:10B1A0000F4605D05A00934226D96FF0030600E0FF
:10B1B000042630463DF056F8054694E809001B1A6F
:10B1C0009B109A003968AF1807D045F8231094E80F
:10B1D00009001B1A9B109A00AF1823B1014628469C
:10B1E00042F090FB2068043708B100F065FA2E4465
:10B1F000A66084E8A000F8BDB2F1804FD5D2DE0091
:10B20000D7E700BF38B5436884680246A34206D03A
:10B2100009680BB1196043680433536038BDFFF708
:10B22000B9FF38BD2DE9F0410023064684B04360E4
:10B230008360C360054646F8043B10203DF012F8D9
:10B2400004AC07466E4902F0FFFD44F8047D304629
:10B250002146FFF7D7FF01AA6A4920463DF014FEB8
:10B260002046FFF731FA039B674FA3F10C02BA4265
:10B27000804640F0B7802046B8F1000F5ED06149AB
:10B2800001AA3DF001FE10203CF0ECFF21465F4A90
:10B29000804602F0B7F8039BA3F10C00B84277D1C7
:10B2A000B8F1000F05D030462146CDF80C80FFF7ED
:10B2B000A9FF01AA564920463DF0E6FD2046FFF7CA
:10B2C00003FA039B8046A3F10C02BA4249D1B8F1BC
:10B2D000000F1ED04E4901AA20463DF0D5FD10209A
:10B2E0003CF0C0FF21464B4A804602F08BF8039B9E
:10B2F000A3F10C00B84240D1B8F1000F05D03046A0
:10B300002146CDF80C80FFF77DFF284604B0BDE84C
:10B31000F08101AA404920463DF0B6FD2046FFF7E6
:10B32000D3F9039B8046A3F10C02BA424BD1B8F18A
:10B33000000FEAD001AA20463749CEE701AA3749D3
:10B340003DF0A2FD2046FFF7BFF9039B8046A3F125
:10B350000C02BA4227D1B8F1000FAAD020462F49DB
:10B360008EE753F8041C481E002943F8040CAEDC99
:10B37000104602A93DF0E2FAA9E753F8042C511E49
:10B38000002A43F8041CB7DC02A93DF0D7FAB3E762
:10B3900053F8042C511E002A43F8041C80DC02A937
:10B3A0003DF0CCFA7CE753F8041C481E002943F812
:10B3B000040CD0DC104602A93DF0C0FAB8F1000F31
:10B3C0003FF477AFCAE753F8041C481E002943F83E
:10B3D000040CACDC104602A93DF0B0FAB8F1000F45
:10B3E00093D0A7E753F8041C481E002943F8040C27
:10B3F0003FF741AF104602A93DF0A0FA3BE700BF7E
:10B40000AC860500B48605005C0A0010C486050001
:10B41000E0860500D4820500EC860500CC86050098
:10B4200010B5054C204600F079FB20460349044A3C
:10B43000BDE810403CF03BBFE8020010B5B0000092
:10B44000C80000100022026042608260C260704743
:10B45000F0B4084C002725684FEA122C41600281A5
:10B460008F70CF7081F801C00A7005602060F0BC59
:10B47000704700BF040300108B0718BF21F00301C1
:10B480002DE9F00118BF0431456801F1040C1FFAE1
:10B490008CFC2B4610E093F801809A7841EA082151
:10B4A00041EA024141EA046161450A461EDA018926
:10B4B00013446A18934215D2DA781978D70902F042
:10B4C0007F041646E7D05E789C7841EA062141EA7F
:10B4D000044102F07F0241EA0262018913446A18C2
:10B4E0009342E9D30020BDE8F001704746F08006A2
:10B4F0008C45DE7027DA03EB0C02D478CCEB01012B
:10B5000067F3C71404F08004C1F306652543C1F353
:10B510000726C1F3074403F80C10D57056709470D9
:10B52000DC782CF0004C04F0800400214FEA1C254C
:10B5300083F800C05D70DC70997044680189121B4B
:10B540008A4200D300BEBDE8F001181D704700BF5D
:10B550002DE9F00311F8013C11F8035C11F8044CDB
:10B560006FF3C71311F8022C01F8013C44EA0524DB
:10B5700044EA024203F07F034668048942EA036317
:10B580000F1FFA183519AA426CD2D5785FEAD51C7C
:10B590006BD033787578B278F47843EA052343EAC0
:10B5A000024304F07F0443EA0464324616E004894F
:10B5B0001A46A54206EB040C54D21D7893F801906C
:10B5C00093F80280DC7845EA092545EA084504F04D
:10B5D0007F0455EA046445D0634543D21319951B93
:10B5E000BB422544E3D1D378DE09C3F3C01539D17A
:10B5F00011F8046C11F8039C11F8028C11F801CCBD
:10B6000046EA092646EA08460CF07F0C46EA0C6634
:10B61000344423F07F08C4F3066CC4F30726C4F354
:10B6200007432B432C4348EA0C0C2E4382F803C0FB
:10B6300056709370147011F8043C11F8032C11F833
:10B64000024C11F8011C43EA0222436842EA044218
:10B6500001F07F0142EA0161FB1A02890B44934227
:10B6600000D900BEBDE8F0037047961BB44200D27B
:10B6700000BEFE5C92F801C0947846EA0C2205F008
:10B680007F0542EA044242EA056211F8015C134474
:10B69000C3F3066225F07F051543C3F30724C3F304
:10B6A000074201F8043C01F8015C01F8034C01F881
:10B6B000022C46686DE700BF084B01461B684BB182
:10B6C0005A689142FAD3188902449142F6D2184638
:10B6D000FFF73EBF084638F09FBC00BF04030010D0
:10B6E0002DE9F04F0A68446880469568084683B0A3
:10B6F0000F462346B8F8082024494FF00009A84710
:10B70000DFF898B0D8F80460CA4602E0042D33D9B7
:10B710002C44E2783B68D2091D4A9D6808BF5A460E
:10B72000009260782378A178E27843EA002343EA24
:10B73000014302F07F0243EA02620192A31B154912
:10B7400022463846A84721786578E378A27841EA0E
:10B750000525D8F8046045EA024503F07F0245EA72
:10B760000265DB09C6EB0402B8F808302A4408BFBA
:10B77000A9449A42AA44C9D3396852468C684B46B8
:10B7800038460549A04703B0BDE8F08F0C87050097
:10B79000FC8605002C8705005087050004870500FE
:10B7A0004368F0B405891C46002002E0042A14D93D
:10B7B0001344D9785F78CA091A789E7842EA07223A
:10B7C00001F07F0142EA064242EA0162C4EB030152
:10B7D000114408BF8018A942E8D3F0BC704700BFED
:10B7E000032100F0B7BA00BF10B5064B044640680D
:10B7F000236008B1FFF760FF204600F095FA20466D
:10B8000010BD00BF7887050038B5104D04462B6881
:10B8100093F8A430DB0708D50D4B0E4819884A1C55
:10B82000C1F300311A80FDF71BF972B6636A53B198
:10B83000636A013B636262B6042128680022BDE8A6
:10B840003840FEF73FBC62B638BD00BFE4020010CE
:10B850000C030010A802001010B5074B0446406806
:10B86000236008B1FFF728FF204600F05DFA20466C
:10B87000FFF722FF204610BD78870500F0B585B0A0
:10B88000044600F061FA294A002304F118052260F9
:10B890006360A360E3602846FCF76CFA244B2549FB
:10B8A00001AA03A81C603DF0EFFA284603A9FCF7A3
:10B8B00049FC83799B0707D5037901229A400368E5
:10B8C000196821EA02021A60FCF752FB039B1A4A2C
:10B8D000A3F10C0090421ED11849194BD1F8C46055
:10B8E00003250022174846F48006C1F8C4605D6154
:10B8F0005A600168144E8908A6FB010605202061E4
:10B90000B6080127204666619E615D605F60216226
:10B91000626205B0F0BD53F8042C511E002A43F8B2
:10B92000041CD9DC02A93DF009F8D5E778870500A9
:10B9300008030010A88705005C0A001000C00F4033
:10B940000000094098010010CDCCCCCC0349044B39
:10B950000120082248601A60704700BF00000940BB
:10B9600000E100E0074A30B41268074B9208B2FBCE
:10B97000F1F103250124416199615D605C6002621F
:10B9800030BC70479801001000000940F8B54468C9
:10B9900085680646AC42416902D112E0A54210D04A
:10B9A00054F8043B5A69521A002A5A61F6DA1869A7
:10B9B0001F6802445A61BFB10020B847A5427169AF
:10B9C000EED1336A591A002931621BDBB37F9A0723
:10B9D00008D5B169327F496921FA02F25340DB0789
:10B9E00000D5F8BD00BEF8BD5A68002AD6D09F68C1
:10B9F000D86887B1C10710D402EB60000021B847B6
:10BA00007169CBE7074A736A1268013301EB92014F
:10BA100031627362DAE7C307C0D54010135810448F
:10BA2000DF59EBE798010010054B1A68D20703D5E0
:10BA30001A6842F001021A60024B1868FFF7A6BFAD
:10BA40000000094008030010F8F73ABF08B50321C9
:10BA500000F080F9BDE80840F8F732BF10B5034B9D
:10BA60000446036000F060F9204610BDB887050069
:10BA700010B5054B0446036000F056F92046FFF769
:10BA80001BFE204610BD00BFB887050070B51546E7
:10BA90000E46044600F058F90A4B291C18BF012134
:10BAA00023600020F8F7D6FE3046F8F7EBFEF8F7F3
:10BAB00007FF2DB9044B01210822196083F80023E8
:10BAC000204670BDB887050000E100E008B50E4BC8
:10BAD0001B6893F8A430DB070FD500210B48FCF757
:10BAE000BFFF01210A48FCF7BBFF00210948FCF712
:10BAF000B7FF09480121FCF7B3FFF8F7D9FEF8F7C3
:10BB0000DFFE00BE08BD00BFE4020010A40200106A
:10BB1000A6020010A8020010AA02001010B50849E1
:10BB2000002200230446016083608274C274828113
:10BB3000C2810282426003493CF0ACFF204610BD46
:10BB4000680A00100CE9050000220021816082745F
:10BB5000C2748281C2810282426001493CF09ABF74
:10BB60000CE90500837C10B5044613B9024842F085
:10BB70004BF8204610BD00BFE8870500F0B5837C78
:10BB800087B004460BB9C37C03BB0023214605A83C
:10BB900003933DF0ECF804A805A9FEF7D3FC059B40
:10BBA0001C4DA3F10C00A84228D1049E03A93046E5
:10BBB00043F0EEF8039B0746B3420AD9049BA3F176
:10BBC0000C02AA420ED1384607B0F0BD806807B01B
:10BBD000F0BD208A2168A289E38900900E4841F0D7
:10BBE0005FFFEBE753F8041C481E002943F8040CE0
:10BBF000E9DC104605A93CF0A1FEE4E753F8042C6B
:10BC0000511E002A43F8041CCFDC02A93CF096FE2A
:10BC1000CBE700BF5C0A001040880500F0B5837CCC
:10BC200087B004460BB9C37C0BBB0023214605A893
:10BC300003933DF09CF804A805A9FEF783FC059B3F
:10BC40001C4DA3F10C00A84229D1049E03A9304643
:10BC50000A2243F037F9039B0746B3420AD9049BF3
:10BC6000A3F10C02AA420ED1384607B0F0BD4068DD
:10BC700007B0F0BD208A2168A289E38900900E48B0
:10BC800041F00EFFEBE753F8041C481E002943F86F
:10BC9000040CE9DC104605A93CF050FEE4E753F83B
:10BCA000042C511E002A43F8041CCEDC02A93CF0EF
:10BCB00045FECAE75C0A0010D088050010B50446AE
:10BCC0003DF055F8204610BD08B5837C0BB9C37C08
:10BCD00043B90749002203233CF072FD013018BF2D
:10BCE000012008BD4068003018BF012008BD00BF1A
:10BCF0005C89050010B50123044641600846E374E1
:10BD00003DF0FAFEA060204610BD00BF0122816018
:10BD1000C2747047837C10B504461BB90123C374F9
:10BD20003DF031F8204610BD014B0360704700BF65
:10BD30006889050010B5034B04460360FFF7BCFC9F
:10BD4000204610BD68890500014B0360704700BFA5
:10BD500068890500024B02461868FEF7A7BA00BFC3
:10BD6000E4020010014B0360704700BF108A050019
:10BD70000EB4002003B07047014B0360704700BF52
:10BD8000108A050010B5034B04460360FFF794FCCE
:10BD9000204610BD108A050010B5034B0446036011
:10BDA000FFF78AFC204610BD108A0500084642F0C5
:10BDB0001EB900BF0EB42DE9F04392B019AC54F88F
:10BDC000049B02AE234605464A4630464021019474
:10BDD00044F00EFD471C3F2F04460ADC2B68314619
:10BDE0005B6928469847204612B0BDE8F04303B08F
:10BDF000704738463CF034FA39464A46019B804643
:10BE000044F0F6FC2B6841465B6928469847B045EC
:10BE1000E9D0B8F1000FE6D040463CF04DFAE2E739
:10BE200010B4054B054C18461C600549054A5DF8E1
:10BE3000044B3CF03CBA00BF10030010E889050039
:10BE400079BD0000C8000010F0B4104BDFF854C0FA
:10BE50000F4F104E00225CF80200B9581C6941EAED
:10BE6000000524EA05041C615C699861B450043241
:10BE7000142AD96103F12003EDD107490748084B83
:10BE8000052208601A60F0BC704700BF00C009209E
:10BE900028030010140300103C03001080C0092088
:10BEA0005403001040030010F0B4114ADFF858C0EA
:10BEB000104F114E00235CF80340F9581569F058F3
:10BEC0002143043325EA010501EA0004142B21EA89
:10BED000000115619461D16102F12002EBD10749A3
:10BEE0000748084B052208601A60F0BC704700BF85
:10BEF00000C0092040030010140300103C03001090
:10BF000080C00920540300102803001004280AD818
:10BF10001F2908D8012202FA01F1034B53F820200F
:10BF20000A4343F8202070474003001004280AD831
:10BF30001F2908D8012202FA01F1034B53F82020EF
:10BF40000A4343F82020704728030010022994BFB9
:10BF500050F82100004870470000C07F2DE9F84FDD
:10BF6000164603460022D1F80490D6F808A043F8FC
:10BF7000042B42605A6004460D46484651463DF047
:10BF80000FFED5F8088077688346394640463DF075
:10BF900007FE014658463DF0F9FC36682060314600
:10BFA00040463DF0FDFD2D688046294650463DF057
:10BFB000F7FD014640463DF0E9FC29466060384601
:10BFC0003DF0EEFD3146054648463DF0E9FD0146AF
:10BFD00028463DF0DBFCA0602046BDE8F88F00BF9E
:10BFE00070B504460D46006809683DF0D9FD6968E2
:10BFF000064660683DF0D4FD014630463DF0C8FC81
:10C00000A9680646A0683DF0CBFD014630463DF0EC
:10C01000BFFC70BD0346806870B501465D681E6850
:10C020003DF0BEFD2946044628463DF0B9FD3146A7
:10C03000054630463DF0B4FD014628463DF0A8FCDB
:10C04000014620463DF0A4FC70BD00BF70B503461C
:10C050000446002043F8040B58600D4660600868F1
:10C06000116816463DF092FC7168206068683DF0EA
:10C070008DFCB1686060A8683DF088FCA060204637
:10C0800070BD00BF70B503460446002043F8040BA2
:10C0900058600D4660600868114616463DF080FD08
:10C0A0003146206068683DF07BFD31466060A868DD
:10C0B0003DF076FDA060204670BD00BF0346002223
:10C0C00070B543F8042B426004465A6008460D469A
:10C0D000FFF7A0FF3EF0FCFF0646014628683DF052
:10C0E00013FE3146206068683DF00EFE3146606008
:10C0F000A8683DF009FEA060204670BD054B10B455
:10C100000421022400221C6019605DF8044B426384
:10C11000704700BF00E100E038B50D4B04462161D7
:10C1200018680D463DF0E4FC4FF07A513DF038FDC3
:10C1300029463DF0E9FD3EF0E1FC3DF033FF4FF0D4
:10C140004023032101226061986159605A6038BD23
:10C150009801001038B50C4B0D4618683DF0C8FC2E
:10C160004FF07A513DF01CFD0849044628463DF049
:10C17000CBFD014620463DF013FD3EF0BFFC3DF0F7
:10C1800011FF034B986138BD9801001000247449D9
:10C1900000800040F8B5194F194E0025194A4FF09C
:10C1A00040230321C5624563386085609E61596103
:10C1B0005D60D2F8C410144F03F5804341F00401D0
:10C1C00005260446C2F8C4109F6110495E615D6097
:10C1D000FFF7A2FF20460E49FFF7BCFF94F8383066
:10C1E000E56265F3440384F8383094F83830256309
:10C1F00065F3000384F838302046F8BD580300107A
:10C200008096980000C00F4040420F000050C34786
:10C210000000C84230B490F83850C5F34305FDB172
:10C220000023012402E00133AB4219DA04FA03F1DE
:10C23000C26A1142F7D000F1180252F82320917A15
:10C2400011F0020FEFD011F0010F117A526804FAC9
:10C2500001F103F1010314BF9161D161AB42E5DB50
:10C260000023C36230BC7047044B054A196810684C
:10C2700041F001011960FFF7CDBF00BF0080004011
:10C28000580300102DE9F041066B002E53D090F8B2
:10C290003810C1F34301002947D00023F46C9C46B9
:10C2A000012703E00133DBB28B4236DAC3EBC30272
:10C2B00004EBC202926A002AF4D003F01F0807FAC6
:10C2C00008F800EB83029269B56C92F812C018EA84
:10C2D000050F0CBF4FF000084FF001081CF0020FD3
:10C2E0000CF001050BD092F810C0454507FA0CF58B
:10C2F000D2F80CC014BFCCF81850CCF81C50158FD5
:10C30000013368F308251587158FDBB245F40075F6
:10C310008B424FF0010C1587C8DB00234363BCF14F
:10C32000000F03D00120BDE8F0814163034B1B687F
:10C33000986908F01DFE0020BDE8F081E4020010BD
:10C340002DE9F04F90F838300646D80785B0904D6B
:10C3500040F1DC80296891F8A4000391C0F340000B
:10C36000002858D196F83880C8F34308B8F1000F78
:10C3700000F0FD80D6F830B0D6F834A0DBF84C9051
:10C380000746029522E0DDE90023012A73F100034C
:10C390004DDBDCE90245DDE90023121943EB05031F
:10C3A0004FF0FF346FF0404594429D41CCE90223A9
:10C3B00044DB06EB80039B6993F8393013F0020FDE
:10C3C00018BF01270130C0B240457BDAC0EBC00C7A
:10C3D00009EBCC0CDCF82830002BF3D0DCF8301063
:10C3E000DCE90045DCE90423121943EB0503514560
:10C3F000CDE90023CCE90023C5D1DBF83C10514541
:10C40000DBF8401000F099805145BCD1DCE90645CD
:10C41000CCE90445B7E796F8382000236FF3000213
:10C4200086F838207363336305B0BDE8F08F0022CF
:10C430000023CCE9002300224FF08043003243F177
:10C440004043DCF82C10CCE9022306EB80039C6906
:10C450000131CCF82C10A37A9A0708D513F0010FFC
:10C46000227A63687ED1012505FA02F29A6194F876
:10C470003930E26A13F0010F0CBF01234FF0FF3394
:10C480001344E36294F839200428C2F340027CD8B4
:10C49000012300F01F0103FA01F1F36A0B43F36279
:10C4A0003AB1DCF82C20DCF828309A4201D023463F
:10C4B00082E70025CCF82850228F23466FF34922CB
:10C4C000228779E7029DF36A0AF10102726323B1C0
:10C4D000304B0321012259605A60002FA4D10399E7
:10C4E0007763886908F044FD2B6806F1300198698C
:10C4F00008F0C4FC00283ED196F83830376367F363
:10C50000000386F8383005B0BDE8F08F2B6806F1DF
:10C510003001986908F0B2FC002885D03046FFF75A
:10C52000B1FE96F8383060F3000386F8383096F89C
:10C530003830D9073FF50EAF76E7DBF844400022EC
:10C540000023A142CCE90423BFF45EAF5145CCF8EF
:10C5500030103FF45BAFDCE90845CDE90045CCE99C
:10C56000004510E7012101FA02F2DA617FE7474650
:10C57000D6F834A0A7E73046FFF784FE96F83830A7
:10C5800060F3000386F838304EE703483CF009FDBD
:10C59000E402001000800040308A05004FF0402384
:10C5A0001968034A41F0010119601068FFF7C8BE1D
:10C5B0005803001010B490F83820C2F34304631CF1
:10C5C00003F00F0300EB840463F3440280F8382087
:10C5D000581EA1615DF8044B704700BF826808B522
:10C5E00012B1C368984708BD3CF0DEFC08B5034BA8
:10C5F000186883680BB1FFF7F1FF08BD58030010FE
:10C6000070B4074E074D084C08490022C664056502
:10C610004465816502704264826470BC704700BFEB
:10C620000123456789ABCDEFFEDCBA987654321012
:10C63000F0B48AB10C460023A5786678CF5C2D044F
:10C6400045EA0625E6783D4345EA0665C5500433CC
:10C650009A4204F10404EFD8F0BC704730B4A2B1A0
:10C66000034600240D680433055551F8045B043477
:10C670002D0A03F8035C31F8025CA24203F8025C65
:10C6800011F8015C03F8015CECD830BC704700BFC6
:10C690002DE9F04F91B0044640226846266D656D45
:10C6A000A76DD4F84C80FFF7C3FFDDF800E0E24B44
:10C6B00005EA0602F04427EA060C43444CEA020C61
:10C6C0009C44019A06EB7C6CDC4B25EA0C000CEADE
:10C6D00006013A44134440EA0107029A1F440CEB56
:10C6E0003757D74B26EA070007EA0C012A441344C0
:10C6F00040EA01051D44039907EBF535D14B05EAE6
:10C7000007022CEA05000E44334410431844049AEF
:10C71000CD4B05EBB020134427EA000100EA0502E7
:10C720009C441143059E6144C84B00EB7161334446
:10C7300025EA010201EA00061F4432433A44C44E8E
:10C74000069F01EB325220EA020C3E4402EA010746
:10C7500035444CEA07032B44BE4F079D02EBF333ED
:10C7600021EA030C2F4403EA020538444CEA05068B
:10C77000089F0644B84D03EBB62606EA03003D4485
:10C7800022EA0607294447EA000C8C44B348099979
:10C7900006EB7C6C23EA0C0508440CEA06012943ED
:10C7A00002440A9D0A440CEB3257A5F5244226EABE
:10C7B000070007EA0C014F3A134440EA01051D4403
:10C7C0000B98A74A07EBF5352CEA050105EA0703A4
:10C7D0000244164441EA030030440C99A14B05EB96
:10C7E000B02027EA000800EA05020B449C4448EA0E
:10C7F000020161440D9A9C4B00EB716125EA01082E
:10C80000134401EA000C48EA0C0C1F44674401EB96
:10C810003752964B0E9F6FEA020909EA00083B4423
:10C8200002EA010C48EA0C0C1D4405EB0C0302EB78
:10C83000F3330F9DDFF860C26FEA030808EA010BCB
:10C84000AC4403EA020A4BEA0A0A6044019E5044DF
:10C85000DFF848C203EBB02000EA020AB44403EA5E
:10C8600009094AEA09096144069E4944DFF830B2E1
:10C8700000EBF16101EA030CB34400EA08084CEA5A
:10C8800008085A440B9E4244DFF818C201EBF252EA
:10C8900002EA0009B44421EA000849EA08086344AE
:10C8A0004344DFF804C202EBB34303EA0109F44452
:10C8B00022EA010849EA08086044059E4044DFF87E
:10C8C000ECC103EB303000EA020923EA0208B44469
:10C8D000614449EA080B0A9E8B44654900EBFB6BF7
:10C8E0000BEA0308314420EA030C48EA0C0C0A4422
:10C8F000624460490BEBF25A0AEA000C29442BEA25
:10C9000000024CEA02020B44134404995A4A0AEB0F
:10C91000B3490A442AEA0B0309EA0B010B4310440A
:10C920001844099A554B09EB303808EA0A011344B8
:10C9300029EA0A020A439B449344514A08EBFB6CE0
:10C940000CEA09013A4428EA09030B439244039E86
:10C950009A444C4B0CEBFA5000EA080A33442CEA98
:10C9600008024AEA020299449144474B089A00EBB4
:10C97000B94101EA0C0A134420EA0C094AEA090900
:10C9800098440D9EC844414B01EB383202EA00093D
:10C9900021EA000833449C4449EA0803029E6344A8
:10C9A000DFF80C8102EBF36303EA0109B04422EAE9
:10C9B000010C49EA0C0C4044079E6044DFF8F4C0C7
:10C9C00003EBF05000EA0209B44423EA020849EA02
:10C9D000080861440C9E4144DFF8DCC000EBB14123
:10C9E00001EA030920EA0308B444624449EA080C56
:10C9F0009444059A01EB3C3CA2F5B82AAAF2BE6A1F
:10CA000081EA0002089E534482EA0C0A204A5344F9
:10CA10000CEB337332448CEA01080B9E88EA03085E
:10CA200010441C4A404403EB7050324483EA0C0823
:10CA300088EA0008114441E078A46AD756B7C7E8ED
:10CA4000DB702024EECEBDC1AF0F7CF52AC6874730
:10CA5000134630A8019546FDD8988069AFF7448BFE
:10CA6000BED75C892211906B937198FD8E4379A695
:10CA70005314440281E6A1D8C8FBD3E7E6CDE121F7
:10CA8000D60737C3870DD5F4ED145A4505E9E3A958
:10CA900081F6718722619D6D2108B44962251EF6D9
:10CAA00040B340C0515A5E26AAC7B6E95D102FD6E2
:10CAB000F8A3EFFCD9026F678A4C2A8DA44A41443F
:10CAC00000EB31413A4480EA030A019E8AEA010AF6
:10CAD0009444A04AD44401EB7C2C81EA00083244FF
:10CAE00088EA0C08049E1A449B4B42440CEB3272B9
:10CAF0008CEA0108334488EA0208079E03449748F9
:10CB0000434402EB7353304482EA0C080A9E88EADD
:10CB1000030801449248414403EB3141304483EA25
:10CB200002090D9E89EA010984448E48CC4401EB38
:10CB30007C28304481EA030989EA080902448A48CA
:10CB40004A4408EB327C704488EA010282EA0C0213
:10CB5000034413448548039A0CEB735310448CEA46
:10CB60000802069E014482EA0300814A084403EB5E
:10CB70003040324483EA0C09099E89EA0009904456
:10CB80007C4AC84400EB7821324480EA03080C9EBA
:10CB900088EA01089444784AC44401EB3C7C81EA69
:10CBA0000008324488EA0C081A44744B42440CEBE7
:10CBB00072528CEA01082B44029E88EA0208034460
:10CBC0006F48434402EB3343304482EA0C0888EA5E
:10CBD0000308014441446B4803EB7121704461EA4E
:10CBE000020E84448EEA030E079EE644664801EB7B
:10CBF000BE6E30446EEA030C8CEA010C02446244BF
:10CC000062480EEBB252384462EA010787EA0E0727
:10CC100003443B445E48059F02EB7343384463EA98
:10CC20000E07574001440C9E39445A4803EBF1214A
:10CC3000304461EA02065E408644039FB64456488B
:10CC400001EBBE6E6EEA0306384402444E400A9879
:10CC500016440EEBB656A0F5801766EA0102A7F659
:10CC6000833782EA0E023B4413444C48019A06EB98
:10CC70007343104463EA0E02014482EA060008444A
:10CC8000474F089903EBF0200F4460EA06025A4030
:10CC9000BE449644434900EBBE6E29446EEA030548
:10CCA00045400E442E44404A069D0EEBB6562A449B
:10CCB00066EA000181EA0E0113440D9F0B443B4AD2
:10CCC00006EB73433A4463EA0E0110447140014499
:10CCD000374A049803EBF121024461EA0600584008
:10CCE00072440B9D0244334801EBB262284462EA6D
:10CCF00003054D400644029F2E442F4802EBB656D2
:10CD0000384466EA0105554003442B442B48099DED
:10CD100006EB734363EA020E2844276D8EEA060E83
:10CD2000014471441F44606DE56C07EBF127A16D70
:10CD300003442A440E44E264684627656365A66599
:10CD40000021402240F0F9FD11B0BDE8F08F00BF96
:10CD50000C38E5FD44EABEA4A9CFDE4B604BBBF620
:10CD600070BCBFBEC67E9B28FA27A1EA8530EFD4EF
:10CD7000051D880439D0D4D9E599DBE6F87CA21FDB
:10CD80006556ACC4442229F497FF2A43A72394ABE9
:10CD900039A093FCC3595B6592CC0C8FD15D84851F
:10CDA0004F7EA86FE0E62CFE144301A3A111084EAC
:10CDB000827E53F735F23ABDBBD2D72A91D386EBA8
:10CDC0002DE9F843446C1746D20013199A42436484
:10CDD000836CC4F3C50488BF0133C4F1400603EB80
:10CDE0005773B74205468846836409D20444601CE1
:10CDF000002408EB04013A1BBDE8F84340F079BD7C
:10CE000020443246013005F1010940F072FDC4F1C1
:10CE1000800449462846FFF73BFCA74202D212E0B5
:10CE200026461C4608EB06012846FFF731FC04F1B4
:10CE300040039F42F4D2484608EB04013A1BBDE888
:10CE4000F84340F056BD48463446D2E730B5037843
:10CE500083B00446B3BB00F1440529466846082266
:10CE6000FFF7FCFB626C2046C2F3C502372A94BF71
:10CE7000C2F13802C2F178021449FFF7A1FF20463F
:10CE800069460822FFF79CFF04F15C0004F14C01A5
:10CE90001022FFF7E3FB00214022601C40F04DFD13
:10CEA0000022AB1C84F844206A7003F8012B03F8BD
:10CEB000012B03F8012B03F8012B03F8012B0121AF
:10CEC0001A702170204603B030BD00BFD0000010A2
:10CED000F0B50B788BB00746C3B10D4601AC09AE77
:10CEE000204695F85C200D49023440F093FFB4428F
:10CEF00005F10105F4D1002301A938466A468DF8F1
:10CF000024303BF0C1FF38460BB0F0BD044901AA04
:10CF10003BF0BAFF38460BB0F0BD00BF3C8A0500BD
:10CF20000CE9050000207047002070470020704782
:10CF3000F8B50C4B00240C4D06460360274655F807
:10CF4000043BB34207D00134042CF8D130463AF008
:10CF50001DFB3046F8BDE0B2002145F8047C09F025
:10CF600081FEF0E7508A05005C03001010B504460E
:10CF7000FFF7DEFF2046FEF79FFB204610BD00BFF7
:10CF800030B5D0F84052ADF2A46D0B46144686A8D9
:10CF90002A46204940F03EFFA50730D414F0010F87
:10CFA0000CBF01220222A00505D561054CBF42F04D
:10CFB000080242F0100286A996A809F06BFE28BB71
:10CFC00023071ED40DF27C4496A94FF40972204623
:10CFD00040F08FFC4FF40A703BF044F90DF591617D
:10CFE00005464FF40672684640F083FC94E80E0054
:10CFF000284600F0F3F828460DF2A46D30BD032258
:10D00000D1E796A899990AF013F9DBE700200DF211
:10D01000A46D30BD888A050008B508460AF036FAC6
:10D02000003018BF0120404208BD00BF08B50846C7
:10D0300011460AF095FB003018BF0120404208BDA0
:10D0400008B500214FF4007290F840020AF028FC65
:10D05000003018BF0120404208BD00BF10B59AB093
:10D06000D0F840220B460AA80A4940F0D3FE0AA98C
:10D0700001A80AF0A3F950B94FF498703BF0F2F808
:10D0800001A9044600F026F920461AB010BD002080
:10D090001AB010BD888A050008B508460AF056FA8D
:10D0A000003018BF0120404208BD00BF40F2E73009
:10D0B000704700BFF8B506460F463AF07FFA104BAE
:10D0C000104C3360002354F8045F65B10133042B26
:10D0D000F9D10D4B3A461B680C49D8683FF0F0FF78
:10D0E00001203AF00FF90A4AC6F84032D8B206F1E8
:10D0F000100142F8236009F0B5FD3046F8BD00BFCD
:10D10000508A05005803001000020010908A0500A4
:10D110005C030010002070470069704738B5044672
:10D1200004300AF07DF805461CB1236820461B6ACE
:10D130009847284638BD00BF00B583B0043001AB26
:10D1400009F030FF18B9019803B05DF804FB4FF007
:10D15000FF30F9E700B583B0043001AB09F056FEAB
:10D1600018B9019803B05DF804FB4FF0FF30F9E700
:10D17000022A10B5044609D0012A04BFC368C918A1
:10D18000201D0AF055F820B9E06810BD0369194464
:10D19000F6E74FF0FF3010BD08B5043009F0ECFFA2
:10D1A000003018BF0120404208BD00BF10B5034B3E
:10D1B000044603603AF07AFA204610BDD08A050092
:10D1C00010B5054B044603603AF070FA2046FEF7AE
:10D1D00073FA204610BD00BFD08A050084B070B538
:10D1E00006460948354645F8040B05AC84E80E00B0
:10D1F000284621464FF4097240F07BFB3046BDE8DB
:10D20000704004B0704700BFD08A05004FF0FF3077
:10D21000704700BF704700BF014B0360704700BFFD
:10D22000008B050008B510B103689B699847002082
:10D2300008BD00BF00234381704700BF408970478D
:10D2400041817047014B0360704700BF008B0500B0
:10D2500010B5034B04460360FEF72EFA204610BDBE
:10D26000008B050010B5034B04460360FEF724FA5B
:10D27000204610BD008B050010B5154A88B0044645
:10D280004FF4807304306946069207930AF0CEF893
:10D29000D0B99DF8090098B106990B7893B90D2281
:10D2A0000DF1090104F12803184640F022FB9DF816
:10D2B0000810009AC1F3001184F82C11C4F8282139
:10D2C00008B010BD079AEDE7002008B010BD00BF00
:10D2D0006C030010074B70B4044644F8043B0D4641
:10D2E00006460FCD0FC40FCD0FC42B683046236008
:10D2F00070BC7047288B05008088431A58425841FB
:10D30000704700BF10B583680C4A04460C49A3F16E
:10D310000C00904282B0216004D10A4B2046236069
:10D3200002B010BD53F8042C511E002A43F8041C0F
:10D33000F3DC01A93BF002FBEFE700BF5C0A001041
:10D34000508B05002883050010B583680D4A0446FC
:10D350000D49A3F10C00904282B0216007D10B4B24
:10D3600020462360FEF7A8F9204602B010BD53F80E
:10D37000042C511E002A43F8041CF0DC01A93BF0E8
:10D38000DDFAECE75C0A0010508B050028830500ED
:10D3900070B584B000F10801044602A83BF0E7FC38
:10D3A00002A903A83BF0E3FC03A8FDF78DF9039B5A
:10D3B000134DA3F10C02AA4206460AD10EB1012375
:10D3C0002373029BA3F10C00A8420ED1207B04B072
:10D3D00070BD53F8041C481E002943F8040CEDDC12
:10D3E000104601A93BF0AAFAE8E753F8042C511EB5
:10D3F000002A43F8041CE9DC03A93BF09FFAE5E7A7
:10D400005C0A001038B5094B094D04460560A3605D
:10D4100010460D46FCF78AFF2946A08004F108005B
:10D420003BF0B1FC00232373204638BD680A00108E
:10D43000508B0500F0B5A3B007460E46144601A870
:10D440001A4683211D463FF023FD30B340F0CFFD47
:10D4500022AB184410F8853C0A2B07D08CB928461B
:10D460003FF09AFC0A2801D00130F8D101A840F021
:10D47000BEFD01A9024630463BF00CFB012023B063
:10D48000F0BD01A8232140F077FD0028E7D1214617
:10D49000BA68034840F004FBE1E723B0F0BD00BFE9
:10D4A000708B050030B50B7B83B00D46044673B915
:10D4B0000846FFF76DFF50B9094840F0A5FB20462C
:10D4C000084901AA3BF0E0FC204603B030BD05F15D
:10D4D000080120463BF04BFC204603B030BD00BFA6
:10D4E000908B05000CE905002DE9F043037B8BB020
:10D4F000054688469146002B76D008A84146FCF7A1
:10D500003FFF07A82946FFF7CDFF07987D493FF069
:10D51000CDFD079B7C4E0446A3F10C00B04240F0C9
:10D52000E480A3899A062BD4784F05A92046049756
:10D530003FF044FC04A9284600222346FFF77AFF67
:10D5400006A9002859D020463FF038FC2B6807A8D0
:10D55000D3F81CC004AA08AB2946E0470798034645
:10D5600053F80C2DB34240F09880002A55D1049B0B
:10D57000A3F10C00B04240F0A080A3899B06D4D553
:10D5800020463FF0F1FA07A82946FFF78BFF0798DE
:10D590005F493FF08BFD079B0446A3F10C00B042AE
:10D5A00040F0978021460A203FF0C0FD2146D8F880
:10D5B00000003FF019FE234609220121554840F0A2
:10D5C000C9F82146D9F800003FF00EFE234601219C
:10D5D0001122514840F0BEF820463FF0C5FA012420
:10D5E00020460BB0BDE8F083FFF7D2FE04460028CA
:10D5F00083D120460BB0BDE8F083049BA3F10C005F
:10D60000B042BDD053F8042C511E002A43F8041C2C
:10D61000B6DC07A93BF092F9B2E7D8F80020D9F8B8
:10D62000003052F80C0C059953F80C2C069B024460
:10D630005B1A0332043B9342204612D23FF094FA25
:10D640000024049BA3F10C00B042C9D053F8042C71
:10D65000511E002A43F8041CC2DC07A93BF06EF9F6
:10D66000BEE700223FF0E0FE2146D8F800003FF080
:10D67000BBFD214620203FF059FD2146D9F800008E
:10D680003FF0B2FD234601210222244840F062F817
:10D6900020463FF069FA0124D3E750F8041C01F159
:10D6A000FF3E002940F804EC3FF75FAF184603A99E
:10D6B00001923BF043F9019A57E753F8042C511EAD
:10D6C000002A43F8041C3FF758AF07A93BF036F98E
:10D6D00053E753F8042C511E002A43F8041C3FF76B
:10D6E00061AF06A93BF02AF95CE753F8042C511E00
:10D6F000002A43F8041C3FF714AF06A93BF01EF9BB
:10D700000FE700BFB08B05005C0A0010680A00102C
:10D71000F0820500B88B0500C48B0500B48B0500B2
:10D720002DE9F04784B00C469146434903AA0546CB
:10D730003BF0AAFB237B002B48D003A82146FFF730
:10D74000B1FE03983D493FF0B1FC039B3C4E80463F
:10D75000A3F10C00B04263D1B8F80C309A062ED475
:10D76000DFF8E0A019E0276803A8FF69B84728465A
:10D7700003A93AF0C0FF0399A1F10C00B0422ED1E9
:10D780002B6853F80C3CABB9029BA3F10C00B042E0
:10D7900030D1B8F80C309B0611D402A900224346C0
:10D7A0002046CDF808A0FFF745FE02AA4B462146C9
:10D7B0000028D8D1029BA3F10C00B04225D14046ED
:10D7C0003FF0D2F9284604B0BDE8F0872046FFF7C5
:10D7D000DFFD0028B1D1284604B0BDE8F08751F83C
:10D7E000043C5A1E002B41F8042CC9DC01A93BF073
:10D7F000A5F8C5E753F8042C511E002A43F8041C71
:10D80000C7DC03A93BF09AF8C3E753F8042C511E78
:10D81000002A43F8041CD2DC03A93BF08FF8CEE7C2
:10D8200053F8042C511E002A43F8041C94DC02A96E
:10D830003BF084F890E700BF0CE90500D415060022
:10D840005C0A0010680A0010F8B504460846154640
:10D850000E4640F0CCFB0A4B074623602B6820465F
:10D8600053F80C1C39443BF0BAF931463A4620468D
:10D870003BF0FEF9204629463BF0D1F92046F8BDA1
:10D88000680A00102DE9F04F89B093460546894695
:10D8900007A8114605AA3BF0F7FA07A8FCF714FF02
:10D8A000079BDFF8F882A3F10C024245044640F0E2
:10D8B000378114B909B0BDE8F08F5846B1493FF03F
:10D8C000F5FB01260746DFF8D8A205E0049BA3F18B
:10D8D0000C00404540F03181BB899B0600F103817B
:10D8E00008AC44F810AD3246214628463B46013686
:10D8F000FFF7A0FD002800F0E7802B6821469B6918
:10D9000028464A4698470028E0D082894AF6E6131E
:10D910009A42DBD107AA016805A83BF0B5FA484650
:10D92000FBF76EFB05A907A83BF021FA07A8FCF757
:10D93000CBFE079B0446A3F10C02424540F0158143
:10D94000002C40F08480059B53F8042C002A03DB54
:10D9500005A83BF059F8059B1B782F2B0ED007A884
:10D96000894905AAFFF770FF05A807A93AF0C3FE89
:10D97000079BA3F10C00404540F03C8106AC5946A2
:10D9800007AA20463BF080FA2F214FF0FF322046B5
:10D990003AF001FF21460346002207A83BF030FA87
:10D9A000204607A93AF0A7FE079BA3F10C004045CB
:10D9B00040F0CF80214607A83BF0D9F905A907A878
:10D9C0003BF02DF907A8FCF77FFE079B8446A3F1E7
:10D9D0000C02424540F02881BCF1000F16D105AA87
:10D9E00007A86A49FFF730FF07A8FCF76DFE079B01
:10D9F0000446A3F10C02424540F0E38007A8002C46
:10DA00007CD0624905AAFFF71FFF07E0214607A85F
:10DA10003BF0ADF907A805A93BF001F905A807A956
:10DA20003AF069FE079BA3F10C00404540F0D68018
:10DA3000069BA3F10C00404509D053F8042C511E5D
:10DA4000002A43F8041C02DC07A93AF077FF05A975
:10DA500007A83BF08CF907A8FCF736FE079B0446A5
:10DA6000A3F10C02424540F0D280002C41D0059930
:10DA7000474840F015F807A938463FF09FF941495B
:10DA80003A4605983FF0C0FC28464946059AFFF7FC
:10DA9000F9FE3C4958463A463FF0B6FC384607A9DD
:10DAA0003FF068FD059BA3F10C0040453FF40EAF2D
:10DAB00053F8042C511E002A43F8041C3FF706AF0C
:10DAC00007A93AF03BFF01E7049BA3F10C00404596
:10DAD00009D053F8042C511E002A43F8041C02DC20
:10DAE00007A93AF02BFF38463FF03EF809B0BDE8F1
:10DAF000F08F059927483FF0D3FFD3E705AA2649C1
:10DB0000FFF7A2FE07A8FCF7DFFD079B0446A3F181
:10DB10000C02424546D1002C8AD007A81E4971E765
:10DB200053F8041C481E002943F8040C3FF7C1AE0B
:10DB3000104606A93AF002FFBBE653F8042C511E2A
:10DB4000002A43F8041C3FF7C7AE07A93AF0F6FED7
:10DB5000C2E653F8042C511E002A43F8041C3FF778
:10DB600029AF03A93AF0EAFE24E753F8041C481E43
:10DB7000002943F8040C3FF7E3AE104606A93AF03B
:10DB8000DDFEDDE6D415060050850500D88B0500C6
:10DB9000E48B0500008C0500DC8B05005C0A00109E
:10DBA000680A001053F8041C481E002943F8040CAE
:10DBB000B1DC104603A93AF0C1FE002C3FF438AFA7
:10DBC000ABE753F8041C481E002943F8040C3FF748
:10DBD00015AF104603A93AF0B1FE0FE753F8042C35
:10DBE000511E002A43F8041C3FF722AF03A93AF064
:10DBF000A5FE1DE753F8042C06AC511E002A43F87D
:10DC0000041C3FF7BCAE21463AF098FEB7E653F845
:10DC1000041C481E002943F8040C3FF726AF1046A9
:10DC200006A93AF08BFE20E753F8041C481E002991
:10DC300043F8040C3FF7D0AE104603A9CDF804C05A
:10DC40003AF07CFEDDF804C0BCF1000F3FF4C7AE33
:10DC5000DCE600BF30B5037B83B004460D4683B1DC
:10DC600001A82146FFF71EFC2046019A2946FFF72E
:10DC700009FE019B0B4AA3F10C00904207D103B0AF
:10DC800030BDFFF785FB0028EAD103B030BD53F863
:10DC9000042C511E002A43F8041CF0DC69463AF0BB
:10DCA0004DFEECE75C0A00108088431A5842584148
:10DCB000704700BF00207047014B0360704700BFF2
:10DCC0002883050010B5034B04460360FDF7F4FC00
:10DCD000204610BD288305002DE9F0438668C568FD
:10DCE00083B0AE42074688462AD2AE42DFF86C9037
:10DCF00023D23378741C0A2B08BF012204D106E01A
:10DD000014F8013B0A2B01D0AC42F9D1A21B3146D9
:10DD10006B4601A83BF0CDF83B6838469B6901A9EA
:10DD200042469847019BA3F10C0048450BD1FD6882
:10DD3000AC4205D22646AE42DBD334460022E6E7AB
:10DD400003B0BDE8F08353F8042C511E002A43F8B9
:10DD5000041CECDC69463AF0F1FDE8E75C0A0010CF
:10DD60002DE9F04784B00F469246354903AA804614
:10DD70003BF08AF8B968FE68B14247D2B142DFF899
:10DD8000C49031D20B784C1C0A2B08BF012204D15D
:10DD900006E014F8015B0A2D01D0B442F9D1621AF1
:10DDA00003AB02A83BF085F83B6803A8DD69394660
:10DDB000534602AAA847404603A93AF09CFC039B9D
:10DDC000A3F10C00484525D1D8F8003053F80C3C9D
:10DDD0006BB9029BA3F10C00484526D1FE68B44202
:10DDE00014D22146B142CDD30C460022D8E7029B83
:10DDF000A3F10C00484509D053F8042C511E002A09
:10DE000043F8041C02DC03A93AF098FD404604B034
:10DE1000BDE8F08753F8042C511E002A43F8041C77
:10DE2000D2DC01A93AF08AFDCEE753F8042C511E4A
:10DE3000002A43F8041CD1DC03A93AF07FFDCDE7AA
:10DE40000CE905005C0A0010064B10B5044603609F
:10DE50000846FCF76BFA044A044BA080A260E3601A
:10DE6000204610BD388C05007E21060029230600BF
:10DE70005D4BF0B5D3F884E05C4DD3F88440D3F823
:10DE80000471D3F8C4601FFA8EFE0EFB055546F4EC
:10DE90008056C3F8C460D3F8A861240C013407F19C
:10DEA000010C95FBF4F426F0407E561E83B0054627
:10DEB0008F0194FBFCF4C3F8A8E1072E7AD8DFE8C1
:10DEC00006F07169793D79797904474BD3F8A81147
:10DED00041F04071C3F8A81194FBF2F494FBF7F100
:10DEE000FF2936DC002976D04E1E360246F4001695
:10DEF0003F4F94FBF1F1B942296035DC3D4B0022E4
:10DF00001E601868114620F0FF0018606A642B46F6
:10DF10000722013A501C19621964A3F10403F8D1D5
:10DF2000354B162035491D6039F086F8314B2846AF
:10DF3000DA6822F48072DA6003B0F0BD2A4B94FBF9
:10DF4000F2F4D3F8A811C3F8A81194FBF7F1FF2954
:10DF5000C8DD2B483FF0A4FD254FFF2194FBF1F1D4
:10DF6000B942284E2960C9DD89112748274A3FF068
:10DF700097FDBC4236DD3A460123013394FBF3F1B1
:10DF80009142FADC0029B8BF3F31891120483FF0A7
:10DF900087FDB3E7144BD3F8A81141F00071C3F823
:10DFA000A81199E7104BD3F8A81141F08071C3F87C
:10DFB000A81191E71146174801923FF071FD1648EC
:10DFC0003FF022FE084B019AD3F8A81141F080716E
:10DFD000C3F8A81180E711483FF016FE4FF4001671
:10DFE000012185E72146CDE700C00F4000366E01D4
:10DFF000405DC600004003406C040010BDE000001E
:10E00000DC8C050000FE2000648D050075190300FE
:10E01000A88D0500808C0500C88C0500308D05009A
:10E02000254940F201120B6B70B51A4004460AB143
:10E030000A69426040F202221A4012B11E4A526935
:10E04000A26040F204421A4012B11B4A9269E26097
:10E0500040F608021A4012B1174AD269226141F211
:10E0600010021A4012B1144A126A626142F220028E
:10E070001A4012B1104A526AA26144F240021A4098
:10E0800012B10D4A926AE26148F280021A4012B15E
:10E09000094BDB6A2362084B5E68C6F3026604EB39
:10E0A00086056B6A0BB168689847636C13B130469C
:10E0B0006968984770BD00BF00400340014B186875
:10E0C000FFF7AEBF6C040010034B0B44272B9ABF25
:10E0D000024AD05600207047E83FF6DF588C050012
:10E0E000904B0B44272B33D88F490120C95600FA97
:10E0F00001F1D00730D5272B00F2F880DFE813F0CC
:10E10000680086009800F600F600F600F600F600BB
:10E11000F600F600F600F600F600F600F600F6004F
:10E12000F600F600F600F600F600F600F600F6003F
:10E13000F600F600F600F600F600F600F600F6002F
:10E14000F600F600F600F600F600F600AA00BC00A5
:10E15000D0074FF00101CED4272B00F2D980DFE8A1
:10E1600013F09D00A700B100D700D700D700D7005B
:10E17000D700D700D700D700D700D700D700D700E7
:10E18000D700D700D700D700D700D700D700D700D7
:10E19000D700D700D700D700D700D700D700D700C7
:10E1A000D700D700D700D700D700D700D700BB00D3
:10E1B00028005E4BDA6822F04042DA60DA6C22F026
:10E1C0004042DA645A4B1A6822EA0101196070472A
:10E1D000564B5A6822F440325A605A6842F48032F0
:10E1E0005A605A6C22F440325A645A6C42F400323B
:10E1F0005A644F4B1A68D20303D41A6822F0FF0204
:10E200001A604B4B1A68114319607047474B5A68A4
:10E2100022F440225A605A6842F480225A605A6CB2
:10E2200022F440225A645A6C42F400225A64E0E715
:10E230003E4B5A6822F440125A605A6842F48012E7
:10E240005A605A6C22F440125A645A6C42F400121A
:10E250005A64CEE7354BDA6822F04052DA60DA6869
:10E2600042F04052DA60DA6C22F04052DA64DA6C42
:10E2700042F00052DA64BCE72C4BDA6822F04042EC
:10E28000DA60DA6842F04042DA60DA6C22F040424A
:10E29000DA64DA6C42F00042DA64AAE7234B5A6887
:10E2A00022F440325A605A6C22F440325A6489E7B0
:10E2B0001E4B5A6822F440225A605A6C22F44022C3
:10E2C0005A647FE7194B5A6822F440125A605A6C1C
:10E2D00022F440125A6475E7144BDA6822F0405277
:10E2E000DA60DA6C22F04052DA646BE70F4B5A685E
:10E2F00022F440425A605A6842F480425A605A6C92
:10E3000022F440425A645A6C42F400425A6470E764
:10E31000064B5A6822F440425A605A6C22F440423A
:10E320005A644FE7E83FF6DF588C050000C0024012
:10E330000040034008B50D4BC9071A6803D422F406
:10E3400080321A6008BD12F0E06F05D1074B1A68E1
:10E3500042F480321A6008BD05491A680B68C2F39E
:10E360000262D86803493EF0ABFEEFE7004003408D
:10E3700000020010188E0500174B10B40B44272B19
:10E3800017D816480121C356012A01FA03F1144B8C
:10E3900014D0DA6822EA0101D960DB6813F0FF0FBC
:10E3A00004D1104B4FF48002C3F880205DF8044B79
:10E3B0007047012A4FF00101094BEAD1DC68094A94
:10E3C00024F48074DC60DC684FF480002143D96061
:10E3D0005DF8044B10607047E83FF6DF588C05008D
:10E3E0000040034000E100E041647047002930B480
:10E3F00019DD0E4C03464518002013F8012B82EA64
:10E40000000101F00F0154F82110AB4281EA101015
:10E4100080EA121202F00F0254F8222082EA101051
:10E42000EBD130BC70470020FBE700BF548E0500E5
:10E430000020704704300321FDF78CBCA0F10400DC
:10E44000FFF7F8BF08B5836C13B1013B836403B1D8
:10E4500008BD80680BF0F6FAFEE700BFA0F10400EB
:10E46000FFF7F0BF10B5064B044603F1080228334E
:10E47000226040F8043FFDF757FC204610BD00BF66
:10E48000F88E0500A0F10400FFF7ECBF10B5074BB4
:10E49000044603F108022833226040F8043FFDF7E8
:10E4A00043FC2046FDF708F9204610BDF88E050014
:10E4B000A0F10400EAE700BF70B50C460546C97834
:10E4C00022891B483FF0ECFAE378062B2ED8DFE8D0
:10E4D00003F0042D2D0F0D250D0080230020AB64CB
:10E4E0000121F6F7B7F91348F6F7CCF9012070BD12
:10E4F000002301224FF4FA70A5F8400085F83F3060
:10E5000085F8423085F8433085F8443005F13F0600
:10E51000062122751046E660216170BD01200023AE
:10E5200005F8433F2075E560206170BD002070BD97
:10E53000D08E050090D003002DE9F047344B0446FF
:10E5400088B040F8043B8846FDF7FEFBDFF8C8E0E2
:10E55000304BDEF80000DEF80410764603F10802C6
:10E5600004F10C07283384E80C0103C756F80C0F9C
:10E5700001AD7168B268F3689EF808E00FC53069B4
:10E580007169B2694FF0FE0C00264FF004090123B7
:10E590004FF0090A87F800E084F81AC0E376237781
:10E5A000C4F8214084F815A084F81690E675267604
:10E5B00066766677A677E67784F8206007C50DEB68
:10E5C00009050FCDC4F82500C4F8291003CD2D8806
:10E5D000C4F82D20C4F83130C4F83500C4F839101F
:10E5E000A4F83D5004F11501404600F0E9F904F1AA
:10E5F000250704F10C01A06800F0C6F93946A068AF
:10E6000000F09CFA60772046A66408B0BDE8F08769
:10E61000A08E0500F88E0500A88E0500704700BF8B
:10E62000704700BF704700BF704700BF01207047B0
:10E6300070B5002482B00B460D4616460094214664
:10E6400005220BF001FA00280ADD074B294653F892
:10E6500020303246986803689B68984702B070BDC6
:10E66000204602B070BD00BF70040010A0F1080089
:10E67000FFF7DEBF70B5002482B00B460D4616468C
:10E680000094214605220BF0DFF900280ADD074B34
:10E69000294653F82030324698680368DB6898476B
:10E6A00002B070BD204602B070BD00BF7004001003
:10E6B000A0F10800FFF7DEBFF0B5002583B00B46E0
:10E6C00000952946022206460BF0BEF900282BDDF4
:10E6D0001749441C51F824201AB35378022B20D038
:10E6E00001EB84042F4614E0052B0CD1304655B9BC
:10E6F000D378917803F00303012B0CBF022300238E
:10E7000092880BF0B7FE54F8042F52B15378022BC5
:10E7100007D0042BE8D15772D57854F8042F002A7B
:10E72000F4D1012003B0F0BD284603B0F0BD00BF16
:10E7300070040010F0B5CEB283B000921746334695
:10E740000021042205460BF07FF9041E30DD002174
:10E7500033460091284604220BF076F9002827DD85
:10E76000154951F820305F7251F824205378042B5A
:10E770001ED0022B1CD001EB840406E054F8042FB9
:10E780005378042B14D0022B12D0052BF6D1D3785A
:10E79000917803F00303012B0CBF0223002392881E
:10E7A00028460BF067FE54F8042F5378042BEAD167
:10E7B000002003B0F0BD00BF7004001008B50AF0DF
:10E7C0005BFF002008BD00BF08B519B90BF03AF98E
:10E7D000012008BD0BF034F9012008BD10B503215C
:10E7E00004469C30FDF7B6FA2046BDE810400BF019
:10E7F00027B900BFA0F19C00FFF7F0BF0BF0CCBE23
:10E80000A0F19C00FFF7FABF30B54B7883B0013B15
:10E81000012B0C4602D9002003B030BD8B78012BB0
:10E8200019D0022BF7D18B790021052200910BF032
:10E830000BF905463AF00EFD002200233BF000F8EC
:10E840000028E8D0104B214653F82530986803681B
:10E850001B689847E0E78B790021042200910BF0B8
:10E86000F3F805463AF0F6FC002200233AF0E8FF00
:10E870000028D1D0044B214653F82530D8680368CE
:10E880001B689847C8E700BF70040010A0F108009B
:10E89000FFF7BABFF0B50C46497883B001390129BA
:10E8A00016461D4602D9002003B0F0BDA378012B07
:10E8B0001BD0022BF7D10021A379052200910BF088
:10E8C000C3F807463AF0C6FC002200233AF0B8FF2E
:10E8D0000028E8D0124B214653F82730324698687A
:10E8E0002B4604686468A047DDE70021A379042271
:10E8F00000910BF0A9F807463AF0ACFC0022002387
:10E900003AF09EFF0028CED0054B214653F8273021
:10E910003246D8682B4604686468A047C3E700BF46
:10E9200070040010A0F10800FFF7B4BFF0B585B087
:10E9300004216A46124D0746ADF104060BF008FCAF
:10E9400003A87368A5F110042A4603F00F010929F2
:10E9500094BF3031373122F80219A2424FEA131323
:10E96000F3D146F8043F864205F11005E9D1054987
:10E9700038460AF093FE38460BF0C0FD05B0F0BDF6
:10E9800030010010700400100A4B002002E001303A
:10E9900030280CD053F8042F002AF8D1064A074B30
:10E9A00042F8201009785A880A445A8070474FF07C
:10E9B000FF3070476C040010700400101401001048
:10E9C000002230B41348144606E05D780132042D6D
:10E9D00008BF1C46302A19D050F8043F002BF4D150
:10E9E0000D4B187934B1E478CD78A5421CBF00F105
:10E9F000FF30C0B2094D441C887045F822101C71CC
:10EA000009785A8830BC0A445A8070474FF0FF306A
:10EA100030BC70476C04001014010010700400102A
:10EA2000002270B417491446134607E04678042EB6
:10EA300008BF044608BF2B46302A1DD051F8040FEA
:10EA4000D5B201320028F1D1B4B1ABB12F2B11D81E
:10EA50000D4C54F823201AB912E054F823204AB17F
:10EA600051780133052908BF0130DBB208BFC0B2BD
:10EA7000302BF2D170BC70474FF0FF3070BC704744
:10EA80001046F7E76C04001070040010F8B5274E2C
:10EA90000F46A6F1C003002205E06578042D08BFEB
:10EAA0002246B3423AD053F8044F002CF5D1002A45
:10EAB00034D0FFF7B5FFF9781D4AC1F1010601E036
:10EAC000302C16D052F8043FE5B2013493B15D7892
:10EAD000052DF5D1DD788D42F2D19B78BD7803F01C
:10EAE0000F0C6B401B06EBD46645B8BF6646302C56
:10EAF000E8D12546022914D003360F2E0EDCF6B2DB
:10EB0000BB780C4A23F07F031E430B4BBE7042F8C8
:10EB100025705A8839780A445A80F8BD4FF0FF3082
:10EB2000F8BD0E2EE8D10F26EAE700BF2C05001035
:10EB30006C04001070040010140100104B7810B425
:10EB4000032B15D100230D4C184607E052780133F2
:10EB5000032A04BF0130C0B2302B09D054F8042F6F
:10EB6000002AF3D1064A5DF8044B42F8231070479F
:10EB70004FF0FF305DF8044B704700BF6C0400108D
:10EB800070040010F8B504460BF096F804F19C00F0
:10EB9000FDF7DAF8194A1A481A4E1B4D02F18001A6
:10EBA00002F15C0E02F16807034684E80440C4F8F1
:10EBB0009C10A76000F1BC0143F8046F05600022BF
:10EBC00043F8042F8B42FBD120461049FFF7B6FFD4
:10EBD00020460F49FFF7B2FF0E49A8732046FFF702
:10EBE000ADFF0D49E8732046FFF7A8FF0B492874D5
:10EBF0002046FFF7A3FFB0712046F8BD708F0500D7
:10EC000070040010140100106401001010010010C5
:10EC1000508F050034900500200100102090050061
:10EC200010B5064B04464068236008B13DF09CFFD8
:10EC3000034A002384E80C00204610BD60900500C4
:10EC4000108A050010B5084B04464068236008B1DF
:10EC50003DF08AFF054A0023204684E80C00FCF7BB
:10EC60002BFD204610BD00BF60900500108A0500F6
:10EC700070B544680D4654B108463FF0B8F92346D4
:10EC8000024601212846BDE870403EF063BD2046A3
:10EC900070BD00BF0121FDF75DB800BF10B58368EE
:10ECA0000C4A04460C49A3F10C00904282B021604A
:10ECB00005D12046FDF738F8204602B010BD53F8C4
:10ECC000042C511E002A43F8041CF2DC01A939F07F
:10ECD00035FEEEE75C0A0010C094050010B58368AD
:10ECE0000E4A04460E49A3F10C00904282B0216006
:10ECF00008D12046FDF718F82046FCF7DDFC204639
:10ED000002B010BD53F8042C511E002A43F8041C15
:10ED1000EFDC01A939F012FEEBE700BF5C0A00103E
:10ED2000C09405002DE9F04F51F8043B9BB0054617
:10ED30000DA80C933AF01BF80DA908A83AF017F8A3
:10ED4000089C54F80C3C002B6FD0DFF8CC8254F8B0
:10ED5000043C002B03DB08A839F056FE089C2678FB
:10ED6000242E00F0DB8130463EF034FD07460028BB
:10ED700040F0D481472E6FD04D2E6DD0542E6BD0E5
:10ED8000532E69D04E2E00F000823B2E00F0908072
:10ED9000282E00F08D800A2E00F08A800D2E00F0C3
:10EDA000878008A891490022042339F009FD044610
:10EDB000C8B1202E15D00C988D490368DFF85CB2DD
:10EDC0009B689847089BA3F10C00584540F0738658
:10EDD0000D9BA3F10C00584540F03E861BB0BDE8EA
:10EDE000F08F411CE7D0089B53F8042C002A03DB6A
:10EDF00008A839F009FE089B1B5D462B11D014AC06
:10EE0000204606217B4A2B7D3EF0D2FF20463FF074
:10EE1000EEF822460346002108A839F073FE089C4C
:10EE200095E7CDF8508014ACF0E70C987249036870
:10EE3000DFF8E8B19B689847089CA4F10C0058459E
:10EE4000C6D054F8043C5A1E002B44F8042CBFDCF6
:10EE500014A939F073FDBBE76B68002703F10108C3
:10EE600008A866490022022339F0AAFC441C11D0EC
:10EE7000034608A9002214A839F0C2FF08A814A963
:10EE800039F039FC149BDFF894B1A3F10C0058451C
:10EE900040F091866A6801320FB990450BD00C980A
:10EEA00057490368DFF874B19B689847089B8AE765
:10EEB0000C98514981E700274E2E0597514F08BF06
:10EEC000C5F80480089B53F80C2C002A00F04385F9
:10EED0006B7DD80704D52A690C9B9A4200F06285A5
:10EEE00002224949134608A839F06AFCDFF830A12C
:10EEF000411C0646CDF824A000F0B28214AC334683
:10EF000008A9002220460DF1240939F079FF48466E
:10EF1000214639F0F0FB149BAAF10C0BA3F10C0075
:10EF2000584540F0EE85089B53F80C3C9E4200F299
:10EF3000E5854FF0FF33324608A9204639F060FFDF
:10EF400008A8214639F0D7FB149BA3F10C005845C3
:10EF500040F03E86182039F085F9DFF8C8800C9A19
:10EF60000123494606461FF0BFFCD8F80000347A5A
:10EF700090F8A4309A0757D5A307316822D540F2FC
:10EF8000E73399421ED107210122FBF79BF80C9829
:10EF90001E4903689B6898470C98174903689B684B
:10EFA00098472EB130461FF099FB3046FCF784FBA2
:10EFB000DFF868B0099BA3F10C00584540F0858547
:10EFC000089C3AE7124B53F8042F91422CD0BB42D5
:10EFD000F9D190F8A4305B0740F10F820C980D49ED
:10EFE00003689B689847002EDCD1E1E79494050004
:10EFF000A49405009C94050004F90500EC9005001C
:10F000008C940500B4900500F0900500F490050084
:10F010007C9005003C910500473120005C0A0010FF
:10F02000680A0010E4020010610709D57368352BE7
:10F0300000F02282012B00F0E981032B40F2E881ED
:10F04000337A9B0772D53368752B00F0CC8300F2BE
:10F050000B811E2B00F0F18100F22282022B00F0C6
:10F06000A7821C2B62D12EB130461FF037FB3046F1
:10F07000FCF722FB099B05F1080653F80C3C032B17
:10F0800040F23C85494604224FF0FF330EA839F088
:10F09000B7FE0021B84A04230EA839F033FD0268F8
:10F0A0001AAC034644F8182D3046C3F800A0214698
:10F0B00039F021FB149BDFF8E0B2A3F10C005845B6
:10F0C00040F06C850E9BA3F10C00584540F059852B
:10F0D000A868AA493DF0EAFFE860002800F09D8496
:10F0E0000C986A7D036842F001029B68A4496A7526
:10F0F000AA6898470C9B2B61099BA3F10C0058450B
:10F100003FF4E0AE53F8042C511E002A43F8041CCF
:10F110003FF7D8AE14A939F011FCD3E6DFF87CB282
:10F120008BE640F2F512934200F0E682D8F8000038
:10F13000DFF868B202213246FAF7C4FF337AD90603
:10F1400000F12E81059ABAB9DB0700F18583326997
:10F1500052F80C3C002B40F08583D8F8003093F82F
:10F16000A430DC0600F16682580700F163820C9837
:10F17000844903689B689847002EBDD030461FF035
:10F18000ADFA3046FCF798FAB6E714AC3B4608A94E
:10F190000C9A20461FF0A8FB3A46314620461FF045
:10F1A000F1FA3A4680462A2120461FF0EBFA9DF8F4
:10F1B000583007469A0703D5149B6E2B00F0BC838A
:10F1C000714908A80022012339F0FAFA411C00F025
:10F1D000B181034608A900220EA839F011FE08A843
:10F1E0000EA939F088FA0E9BDFF8B0B1A3F10C003C
:10F1F000584540F09384089A13782A2B00F04183F5
:10F2000052F80C1C49B15018002101E0824204D090
:10F21000594012F8013F2A2BF8D1CF1B00220F23AF
:10F2200008A85A4939F001FB421C089B00F05C8297
:10F2300053F80C3C984200F2618402464FF0FF33D1
:10F2400008A90EA839F0DCFD08A80EA939F053FA78
:10F250000E9BDFF848B1A3F10C00584540F06B84D9
:10F2600020461FF03BFAFBE5B3F5FB7F00F0D280B0
:10F2700040F26281B3F5FC7F00F03E82C0F08982EB
:10F28000B3F57A7F7FF452AF099B53F80C3C042B03
:10F2900040F2348414AC4FF0FF3349460522204637
:10F2A00039F0AEFD204608A939F0B9FC0368DFF853
:10F2B000E8B00A93C0F800A0149BA3F10C005845D5
:10F2C00018D000F051BC0A9B53F80C3C002B00F006
:10F2D00015844FF0FF330AA90122204639F090FD32
:10F2E0000AA8214639F007FA149BA3F10C005845EF
:10F2F00040F03A840A9B53F8042C002A03DB0AA846
:10F3000039F082FB0A9B1878FBF7F0F80028DAD175
:10F310002EB130461FF0E2F93046FCF7CDF90A9BDA
:10F3200053F80C3C002B40F0AE8219490BAA204642
:10F3300039F0AAFD174821460C9A27F0CFFC149B00
:10F34000A3F10C00584540F075840C980D490368F2
:10F350009B6898470A9BA3F10C0058453FF42AAEDE
:10F3600053F8042C511E002A43F8041C3FF722AE28
:10F37000214639F0E3FA1DE6C0810500A0810500B1
:10F380006891050004F90500D8900500DC9005009F
:10F390000CE90500349305005C0A00105C0A0010BB
:10F3A000D8F800300C9893F8A4305A07036848BF87
:10F3B000A4499B6858BFA449984732690C9852F8F1
:10F3C0000C3C002B00F0B1800368A0499B68984773
:10F3D0003369002153F80C2C06F110000B4639F06C
:10F3E000C7FA0C989A4903689B689847D8F80000B8
:10F3F00007210022FAF766FEBEE60C9895490368DD
:10F400009B689847002E7FF4CDADD1E5059AF2B107
:10F410002B7515E6904838F057FA2EB130461FF09C
:10F420005DF93046FCF748F90C988C4903688A4A24
:10F430009B689847DFF86CB25EE6D8F8000090F859
:10F44000A4305C0700F1B480DFF858B272E60C9883
:10F45000834903689B689847012273680592ECE52D
:10F460000DF1240908A9484639F08DFC08A87D490A
:10F47000002239F00FFB6DE5089B53F80C3C002B84
:10F4800040F012812B7D032B00F2D6827360C2689C
:10F4900092F8341041F0080182F834102B75CFE552
:10F4A000702B00F08E81732B7FF440AE2EB130466E
:10F4B0001FF014F93046FCF7FFF80C9C14A82368E1
:10F4C0009D68F7F7B5FF064614A8F7F7B5FF664A3B
:10F4D0000346664910680522A1FB0070800CD8F82D
:10F4E00000108DE8050091F8A4103246C1F38001A8
:10F4F000029120465E49A8470C985E4903689B68C4
:10F5000098470C985C4903689B689847D8F8003086
:10F5100093F8A430580600F122820C9857490368EA
:10F52000DFF880B19B68984744E5036854499B68BD
:10F53000984756E7002771E6B3F5FA7F7FF4F1ADFF
:10F54000D8F800300121986905F002FC72B64D4CE4
:10F550004D49414814943DF0A9FD4C49159014A81B
:10F56000FCF728FC1598149408B13DF0FDFA08202A
:10F5700038F078FE464B0446236037483EF01CFDC9
:10F58000022160603246D8F80000F460FAF79AFD74
:10F59000F06810B103685B6898472EB130461FF0E1
:10F5A0009DF83046FCF788F862B63A490C983DE77A
:10F5B0004FF0010A14AC0AAA374985F814A0204676
:10F5C0000DF1380939F060FC534621464846334A6C
:10F5D0001FF08AF9149BDFF8CCB0A3F10C0058455A
:10F5E00040F059830DF12C0AD8F8000002214A4658
:10F5F000FAF768FD2A4907AA504639F045FC01236D
:10F6000020465146254A1FF06FF90B9BA3F10C00D1
:10F61000584540F0348302212246D8F80000FAF71A
:10F6200051FD20461FF05AF848461FF057F8D8F809
:10F6300000007FE5089B53F80C3C002B7FF49CAD49
:10F6400095E500BF10940500189405005CF90500CD
:10F650002C9405005091050070820500A4930500CC
:10F6600004F905000CE905009801001083DE1B4336
:10F67000F0910500F8920500049305002C93050015
:10F680002094050060900500A081050054930500BA
:10F6900000830500709305009C9105001003001085
:10F6A000A09105005C0A00102EB130461FF016F83C
:10F6B0003046FCF701F8182038F0D4FD012308A9E2
:10F6C0000C9A06461FF010F9002208A8A74939F045
:10F6D000E1F9337A5A0740F1AF817368012B00F2E8
:10F6E000AB81D8F80000D2E6002153F80C2C08A812
:10F6F0000B4639F03DF9B3E514AC4946204639F0E4
:10F7000036FB0DF1380908A9204639F088FA484639
:10F710002146FAF7ABFF149BDFF880B2A3F10C008F
:10F72000584540F094820E9B53F80C1C002940F081
:10F73000DE8048468E49132239F0ACF933688D4A91
:10F740008D4840F2F515AB4214BF054615464946B3
:10F75000204639F00CFB284621460C9A27F0BEFAC9
:10F76000149BA3F10C00584540F04B820E9BA3F173
:10F770000C00584540F0EC812EB130461EF0AEFF33
:10F780003046FBF799FF0C987C4903689B689847C3
:10F7900010E477487A493DF089FC002800F0378171
:10F7A0003DF0E2F90C9877490368714A9B689847E5
:10F7B000337AD8F8000043F001033372DFF8DCB18C
:10F7C000B8E4D8F8000007210022FAF77BFCD8F84B
:10F7D00000306D49586803689B689847002E7FF495
:10F7E000E1ABFFF7E5BB099B53F80C3C032B40F260
:10F7F000858114AC4FF0FF3349460422204639F08E
:10F80000FFFA204608A939F00AFA0368DFF890B138
:10F810000E93C0F800A0149BA3F10C00584540F0D3
:10F82000228243F6122044F2404100220EABF9F747
:10F830002FFB2EB130461EF051FF3046FBF73CFF48
:10F840000C984E4903689B6898470E9BA3F10C00E7
:10F8500058453FF4AFAB83E50C984C4903689B686F
:10F86000984774E40C984A4903689B689847336941
:10F87000002153F80C2C06F110000B4639F078F8F3
:10F880007AE40021C9E40BA80AA9FAF739FE0BA90A
:10F890000EA8FAF79BFE0E9D0BA9204639F067FAD9
:10F8A00028460C9A214627F019FA149B0546A3F125
:10F8B0000C025A4540F0B181002D00F0B6800E9B3D
:10F8C000A3F10C00584540F00D810B9BA3F10C00F7
:10F8D00058453FF43AAD53F8042C511E002A43F822
:10F8E000041C3FF732AD214639F028F82DE51431DC
:10F8F0002046CDF850A039F072F91422254920464F
:10F9000039F0B6F94946204639F089F9484621468A
:10F9100038F0F1FE149BA3F10C0058453FF40EAFF4
:10F9200053F8042C511E002A43F8041C3FF706AF7D
:10F930000BA939F003F801E70C9810490368C5F8E2
:10F9400004809B68984720461EF0C8FEDFF84CB044
:10F95000089CFFF772BADFF844B0FFF734BA0C988E
:10F960000D4903689B689847D7E500BF0CE905007F
:10F9700070820500B8900500C890050004F90500E4
:10F98000D4150600D8930500A491050004EB0500EA
:10F99000489405008C930500109305005C0A001044
:10F9A0005C0A0010032308A9002214A839F028FAE1
:10F9B00014A8C04938F052FF149BDFF820B3044666
:10F9C000A3F10C00584540F01081002C59D0EB6891
:10F9D000002B4ED0B84908A839F084F90898EB6894
:10F9E000012150F80C2C3DF0B5FE089B53F80C3C5F
:10F9F00098420C983ED00368B0499B689847E868E5
:10FA00003DF0B2F80023EB60089BFFF7DCB90C98DF
:10FA1000AB4903689B689847CAE60C98A9490368F4
:10FA2000AA689B689847FFF765BB0C98A6490368CE
:10FA30000E9A9B68984742E72EB130461EF04EFE64
:10FA40003046FBF739FE0C98A0490368DFF88CB20A
:10FA50009B689847FFF7AEBA53F8042C511E002A52
:10FA600043F8041C3FF7BAA914A938F067FFFFF761
:10FA7000B5B90C98036896499B689847089BFFF7AF
:10FA8000A2B9E8683DF070F86B7DAA6864F30003E2
:10FA90006B7552F80C2C05F1080021462346EC60EA
:10FAA00038F066FF0C982C6103688A499B68984778
:10FAB000089BFFF788B953F8042C511E002A43F81D
:10FAC000041C3FF785A9FFF7C3B953F8042C511E56
:10FAD000002A43F8041C3FF773AA14A938F02EFF3C
:10FAE000FFF76EBA53F8042C511E002A43F8041C89
:10FAF0003FF7EBAE214638F021FFE6E6764839F0D5
:10FB000050FA53F8042C511E002A43F8041C3FF706
:10FB10000AAA0EA938F012FFFFF705BA53F8042C11
:10FB2000511E002A43F8041C3FF765AB0BA938F0BF
:10FB300005FFFFF760BB53F8042C511E002A43F861
:10FB4000041C3FF78DAB0BA938F0F8FEFFF788BB1C
:10FB500053F8042C511E002A43F8041C3FF70CAE46
:10FB6000214638F0EBFE07E653F8042C511E002A1C
:10FB700043F8041C3FF7BEAB0EA938F0DFFEFFF7D9
:10FB8000B9BB53F8042C511E002A43F8041C3FF75C
:10FB90009FAA214638F0D2FEFFF79ABA53F8042CF8
:10FBA000511E002A43F8041C3FF78CAA0BA938F019
:10FBB000C5FEFFF787BA53F8042C511E002A43F8FC
:10FBC000041C3FF767A90EA938F0B8FEFFF762B929
:10FBD00053F8042C511E002A43F8041C3FF7BAA91D
:10FBE0000EA938F0ABFEFFF7B5B953F8042C511E3F
:10FBF000002A43F8041C3FF7E8AE0EA938F09EFE39
:10FC0000E3E653F8042C511E002A43F8041C3FF786
:10FC1000ADAD0BA938F092FEA8E553F8041C481EC0
:10FC2000002943F8040C3FF747AE104607A938F007
:10FC300085FE41E653F8042C511E002A43F8041CAB
:10FC40003FF783AB0EA938F079FEFFF77EBB53F880
:10FC5000042C511E002A43F8041C3FF764AD0BA985
:10FC600038F06CFE5FE553F8042C511E002A43F86F
:10FC7000041C3FF7D6AD0BA938F060FED1E553F870
:10FC8000042C511E002A43F8041C3FF7C4AC0AA9F7
:10FC900038F054FEBFE453F8042C0DF12C0A511E29
:10FCA000002A43F8041C3FF79FAC514638F046FE4B
:10FCB0009AE400BF5094050004EB05006C94050025
:10FCC000F8930500809105003C93050054910500D0
:10FCD00004F9050054940500908305005C0A0010A7
:10FCE00038B50446FCF730F8627D0023064D07481E
:10FCF00063F300024FF0FF312375A0602560627549
:10FD000023616160204638BDC0940500680A001078
:10FD100002694069101A18BF01207047A0F1040061
:10FD2000FFF7F6BF037E184AC3F3C10302F148018F
:10FD3000022B10B50446026041601AD0032B1DD07F
:10FD4000012B124B14BF20224022C3F88020104BFD
:10FD50001868F4F7DBFB0F4BE06800221A6008B16B
:10FD600038F0AAFA0C4B20466360FBF7DDFF204613
:10FD700010BD064B8022C3F88020E8E7034B4FF408
:10FD80008072C3F88020E2E7F894050000E100E00B
:10FD90003405001030050010108A0500A0F10400A1
:10FDA000FFF7C0BF10B50446FFF7BCFF2046FBF7C6
:10FDB00083FC204610BD00BFA0F10400FFF7F2BF96
:10FDC00010B508460C463EF012F9044B0246214697
:10FDD0001868BDE810400123F4F7D2BB34050010C9
:10FDE000A0F10400FFF7ECBF08B5034BC9B21868D7
:10FDF000F4F7C4FB012008BD34050010A0F1040095
:10FE0000FFF7F2BF38B50269436904469A420DD044
:10FE100020692269A3680132B2FBF3F5E16803FBB4
:10FE20001523085C23610A2808D038BD0120FAF7A1
:10FE300051FE226963699A42EAD1F7E7637E013B8A
:10FE4000637638BDA0F10400FFF7DCBF30B5037E58
:10FE500083B0D90704462DD49A0701D403B030BD2E
:10FE6000284D6FF341032376002228680721FAF713
:10FE700029F9226963699A420CD0A268236923692F
:10FE80000133B3FBF2F102FB113323612169636992
:10FE90009942F3D1637E6FF3070363762B6893F87F
:10FEA000A4305B071BD423682046DB6B16499847B8
:10FEB00003B030BD134902686FF30003037609688D
:10FEC00001A8D56BF9F736FD20460199A847019B9B
:10FED0000E4AA3F10C00904208D1237EBCE72368B0
:10FEE0002046DB6B0A49984703B030BD53F8042C19
:10FEF000511E002A43F8041CEFDC694638F01EFD51
:10FF0000EBE700BFE40200107C9505005C0A0010DE
:10FF1000609505002DE9F04F437E85B0044613B986
:10FF200005B0BDE8F08FDFF8F4B004AD45F80CBDC6
:10FF30002846142138F053FEABF10C064FF00008B0
:10FF400028E022692169A3680131B1FBF3F903FBC1
:10FF50001913E16811F802902361B9F10A0F32D048
:10FF6000019B53F80C1C53F8082C01F1010A92452F
:10FF700003D853F8042C002A05DD514638F02FFE33
:10FF8000019B53F80C1C03F80190019BA3F10C0298
:10FF9000B24239D12269636928469A42D1D1637E3F
:10FFA0006FF307036376019BA3F10C00B042B7D057
:10FFB00053F8042C511E002A43F8041CB0DC02A99B
:10FFC00038F0BCFCACE7637E2946013B637603A8AE
:10FFD000CDF80CB038F0D7FE0F4B0434186802AAE5
:10FFE00001210294FAF76EF8039BA3F10C00B042D2
:10FFF000D9D053F8042C511E002A43F8041CD2DC3B
:020000021000EC
:10000000694638F09BFCCEE743F8048C43F80CAC0F
:1000100003F80A80BEE700BFE4020010680A00107F
:1000200038B504460D46FBF78FFE154B4FF4807034
:1000300003F1480223606260A06038F011F90023E8
:100040002361E0606361032D06D8DFE805F0151138
:100050000D020C4B0C4A1A60237E0C4A65F3C40354
:1000600023761460204638BD064B094A1A60F3E730
:10007000044B084A1A60EFE7024B074A1A60EBE7A5
:10008000F89405003405001000C009403005001048
:10009000008009400000014000C000402DE9F0430D
:1000A000037E87B0C3F3C103013B022B074688469A
:1000B00057D83E4A3E4912F823203E4802F1010932
:1000C00011F8231010F823305FFA89F906AE06F80C
:1000D000103D002530468DF80920374C8DF80A1068
:1000E0008DF80C508DF80B50F4F7F4FB30468DF87A
:1000F0000990F4F7EFFB04A8F4F736FA04A9206896
:10010000CDF81080F4F76AF801A8F4F7DDFA01A938
:100110002068F4F7BDFA20680121F4F7DDFA2068C1
:1001200029460122F4F78CFA20682A460221F4F7C6
:1001300087FA20682A460121F4F782FA3B7EC3F34E
:10014000C103022B28D0032B1BD0012B0FD005207D
:100150001A4936F071FF1A4B20221A6007B0BDE829
:10016000F0834FF00309002302220121AEE70620AD
:10017000124936F061FF124B40221A6007B0BDE809
:10018000F08308200D4936F057FF0D4B4FF4807275
:100190001A6007B0BDE8F0830720084936F04CFF2D
:1001A000074B80221A6007B0BDE8F083B0950500C8
:1001B000A4950500BC950500340500106D020100F2
:1001C00000E100E03F2910B434D0182939D01929B2
:1001D0003ED00A29037E27D0B1F10D04624262416C
:1001E00062F38203002A037618BF0A2142698368FA
:1001F0000132B2FBF3F403FB14230469A34210D0D1
:100200004269C3680A2999544269836802F101026C
:10021000B2FBF3F403FB1423436102D1437E0133A9
:1002200043765DF8044B70475A07DFD56FF38203BE
:100230000376F6E7037E5DF8044B43F00103037693
:100240007047037E5DF8044B43F00203037670476A
:10025000054B5DF8044B1B6893F8A42042F0800224
:1002600083F8A420704700BFE402001030B5134C9F
:1002700083B02068F4F706FA00F00E03062B17D0BF
:1002800000F00600042801D003B030BD0C4D2068FA
:100290000DF1070101220023F4F798F90028F3D0AB
:1002A00028680028F3D09DF80710FFF78BFFEEE7D2
:1002B0002068F4F7E3F903B030BD00BF3405001047
:1002C00030050010034B0A46014618680123F4F775
:1002D00057B900BF3405001008B5054B186818B1B0
:1002E00003685B6B984708BD4FF0FF3008BD00BF47
:1002F000300500102DE9F84F8C688A4680469346F9
:1003000001F10409BCB1136800E02C4626690127FD
:100310009E428EBFA568E5680027002DF5D15FB924
:10032000B342254616D80023C8F8004088F80430A8
:100330004046BDE8F88F4C46DAF80C50A54209D08B
:10034000204638F050F8DBF8003006692546B34205
:100350000446E8D955B3A94526D0DBF800602B69DF
:100360009E422CBF00260126142037F07BFF044656
:1003700038B1002343608360C360DBF80020037062
:10038000026130462A464B46214638F02EF8DAF80C
:10039000143001221344C8F80040CAF8143088F819
:1003A00004204046BDE8F88F0126DDE72C46BAE779
:1003B00030B51A4D85B02B68044642F6AA2244F2A5
:1003C000ED1158690023FAF7D7FE4FF41651FBF7E9
:1003D00091FCFBF7D3FB39F0BFFD01462046FFF748
:1003E0005DFE237E627E03F0FC036FF307026FF372
:1003F00082036276237620460021FBF7ABFC204681
:100400000321FBF7A7FC2B680434596802A80431C8
:1004100001AA0194FFF76EFF05B030BDE4020010A1
:1004200038B5164D0022296813460446486941F242
:100430009371FAF7A1FE1249FBF768FCFBF79EFBEC
:10044000296800221346E06048694BF66D41FAF7CF
:1004500093FE0C49FBF75AFCFBF790FB296800223E
:1004600013462061486942F2C351FAF785FE002124
:10047000FBF74CFCFBF782FB606138BDE402001027
:10048000CDCC4C3D0000C07F0022034610B503F8E0
:10049000012B0133427003F8012B03F8012B03F801
:1004A000012B03F8012B03F8012B03F8012B03F8B0
:1004B000012B03F8012B03F8012B04461A70FFF7F8
:1004C000AFFF204610BD00BF2A4B2DE9F0471B6847
:1004D00046699F698246BC6807F104082146404688
:1004E00005F002F90546404605F03CF900283ED1EA
:1004F000FB689C4215D095F85030DB0711D531468A
:10050000284604F01FFE21460646404605F0D8F86E
:1005100004462146404605F0E7F8FB680546A3423D
:10052000E9D1284604F044FEBB688146A3421ED0B0
:100530002146404605F0BCF804462146404605F0F9
:10054000D3F84946064604F063FE696A8146726A3A
:10055000284604F051FFBB683546A342E8D1304637
:10056000DAF81420716ABDE8F04704F045BF2E4662
:10057000F5E700BFE40200102DE9F04F8B4E8146F5
:10058000306885B0806901939DF84830043090460A
:100590000F46029305F09CF80446B8F1000F00F0F6
:1005A0008C810025CDF80C904446AA4600954FF06A
:1005B000010B8146B84614E009F148010AF01F0218
:1005C0000BFA02F2086820EA020008600AF1010A48
:1005D000002FB8BF7F42A24549F8057005F1040518
:1005E00023D2326858F80510D26892685059F8F74B
:1005F00055FF07460028DFD06C480123026858F8F1
:100600000510D0683A46806800934059F8F740FFDB
:10061000002F0AF01F0280F27B810BFA02F2D9F858
:1006200048101143C9F84810D0E7009B4C46DDF84C
:100630000C90002B00F041814FF08A41119839F065
:10064000AFFA3AF0EDFA39F0ADFC94F85020029987
:10065000B4F8523061F3041260F30B03D2B2256890
:10066000A4F8523042F00802D9F80C7084F85020F7
:10067000002D00F08380109B04F11401E3622346F7
:1006800003E01A68954238BF154604339942F8D101
:100690000E9B4FF00008656123624146184639F011
:1006A0003BFC002800F00481019B2846E36139F0FF
:1006B0001FFA019939F074FA0E9939F025FBA061FF
:1006C0000F9BD9F81450002B00F0F0803368DFF84E
:1006D000DC809869043005F045F8002868D0D9F826
:1006E00014001099A56301F10048014639F058FA49
:1006F00041460746404639F04BF9216A39F050FA35
:100700000146384639F042F93AF0E2FC07463946EC
:10071000284639F001FC00B13D4665623946E06982
:1007200039F0E6FB94F8503000283AD160F34103E9
:1007300084F8503094F8503043F0010384F850307E
:100740000F9B002B00F0C78019685A689B68C9F896
:100750000010C9F80420C9F808304846FFF7B4FE75
:1007600094F85030326843F00403906984F85030B4
:1007700004F0BAFA012005B0BDE8F08F6368002BE1
:100780007FF479AFA368002B00F09E80D9F8108029
:100790004046414639F0CAFB00287FF46CAF47461B
:1007A00069E743F0020384F85030C3E7E402001025
:1007B000D8F800309B6903F104089968404604F0BA
:1007C0007FFF0146404604F08FFF90F8502003461B
:1007D000120784D538460021D3F81C8039F09CFBE1
:1007E00000283FF47CAF4046002139F095FB0028FB
:1007F0003FF475AF0F9BD9F80000196800F1004075
:1008000039F0CEF90F9B83465968D9F8040039F0C6
:10081000C7F90146584639F0B9F80F9B83469968E5
:10082000D9F8080039F0BCF90146584639F0AEF85D
:100830003A49834639F05CFB00283FF450AFE56944
:100840004046294639F068FB00285FD058463449B5
:1008500039F058FB00283FF442AF59464FF07E5024
:1008600039F094F84FF07C5139F09AF93AF030FCB5
:1008700039468046109839F093F9414639F090F99D
:10088000414607464FF07E5039F080F80146384621
:1008900039F03AFA3AF01CFC07463946284639F056
:1008A0003BFB00283FF41BAF3D4618E7284618E7FE
:1008B000C4F81C80C4F8188002E7204604F0A2FBAC
:1008C000012005B0BDE8F08F94F8503065F3C30304
:1008D00084F85030CFE60F984B4603F8010B0133F4
:1008E00089F8010003F8010B03F8010B03F8010B71
:1008F00003F8010B03F8010B03F8010B03F8010BDC
:1009000003F8010B03F8010B187026E745469DE735
:10091000012309F14801009352E600BF72F97F3FBD
:1009200072F97FBF014B0360704700BFD09505008F
:10093000002070470020704710B5034B0446036049
:10094000FAF7BAFE204610BDD095050030B583B049
:10095000002402AB054643F8044D2146224643F6E7
:100960001930F8F76BFA38B195F8363064F3820332
:1009700085F8363003B030BD95F83620002342F0BC
:10098000040285F83620C5F8403103B030BD00BF01
:100990002DE9F0470446D4F8D830D0F8E800984262
:1009A00027D0D4F8EC30D4F8F420984223D0A0F12A
:1009B0000C0310F80CAC10F80B9C10F80A8C10F813
:1009C000097C50F8086C50F8045CC4F8E83094F8DE
:1009D000343084F8A4A067F3410368F3820369F319
:1009E0000003C4F82451C4F8206184F83430BDE811
:1009F000F087BDE8F08752F8043C93F8ECA193F837
:100A0000ED9193F8EE8193F8EF71D3F8F061D3F89C
:100A1000F451FAF751FED4F8F4301A1FC4F8F42058
:100A200053F8043C03F5FC7103F5F672C4F8EC309E
:100A3000C4F8F010C4F8E820C9E700BFF0B5846836
:100A400087B0266800230546F06A0193029303935A
:100A5000049305930F4639F04FF8316A39F054F991
:100A600066680190F06A39F047F8316A39F04CF95C
:100A7000A4680290E06A39F03FF8216A39F044F93D
:100A80006B68039018683A46C46801A91846A047E5
:100A900007B0F0BD2DE9F04791F8A47001F13808D6
:100AA00007EB4707BF0008EB07090C460546D9F8D6
:100AB00008109068164638F069FFD4F8B01038F086
:100AC00067FFD4F8BC1038F061FFD9F804108246F3
:100AD000706838F05BFFD4F8AC1038F059FFD4F8E8
:100AE000B81038F053FF58F807108146306838F0D6
:100AF0004DFFD4F8A81038F04BFFD4F8B41038F0FC
:100B000045FFC5F804902860C5F808A02846BDE850
:100B1000F08700BF000000002DE9F04F90F8704111
:100B200085B08046002C50D0002602E00136B44249
:100B30004BD9D8F8083053F8267097F839301B078E
:100B4000F4D43D6A796A284639F02AF8224B824665
:100B5000D3F80090D9F8340038F0CAFF83465946DC
:100B6000504639F0CFF90028E0D02946584639F0F0
:100B7000CBF839F0C3FF38F07FFB15A3D3E900238E
:100B800004460D4638F0CCFB02460B46204629466B
:100B900038F012FA38F0A6FE78620546504638F072
:100BA0006BFBD9F804402768CDE90001284638F0EE
:100BB00063FBCDE9020132462046BB6807499847EE
:100BC00098F870410136B442B3D805B0BDE8F08F53
:100BD0007B14AE47E17A843FE40200107096050072
:100BE00090F87011032910DD82680320083202E0BA
:100BF0000130814209DD52F8043F93F8393013F097
:100C0000080FF5D05B07F3D570470020704700BF91
:100C10008B684A680968C0F8B820C0F8BC10C0F8F2
:100C2000B4307047054B1B689B681B7D013B022B52
:100C30008CBFD0F82001D0F824017047E4020010E6
:100C400010B5022982B00C4602D9002002B010BDB6
:100C50004FF44C4044F68A5100220DF10303F8F79B
:100C6000EDF80028F1D09DF80320002AEDD14FF4D3
:100C70004C4048F2150101ABF8F7E0F80028E5D048
:100C800002AB1C4414F8040CE0E700BF10B5846804
:100C900014B1C368984710BD38F086F92DE9F04FBC
:100CA00088469FB093469946074600296AD0042992
:100CB00000F0CF80052900F0968008A9FFF7BEFE5E
:100CC000FB692BB108A907F114000122FFF7DEFF31
:100CD000B8F1010F00F0DB80B8F1020F00F0FB80EB
:100CE000B8F1030F00F02A8100220DF1380A5846AE
:100CF000514637F0BDFF97F87021032A1ADDA8F19D
:100D00000206F6B20C254124B9F1000F05D0BB68EC
:100D10005B5993F839301B0704D4B8F1040F0CD099
:100D2000012E24D9A4F13D03934205F1040504F1F9
:100D30000104E9DB1FB0BDE8F08F7B19D3F8F800A0
:100D400038F09AFA924ACDE90001234650464021F4
:100D50003DF02EF84028024688BF402240F2148120
:100D60005846514637F084FF97F87021DAE7BB68A0
:100D70005B59D86A069338F0BFFE069B196A38F0B3
:100D8000C3FFDDE7D0F8F830D0F80051D0F8FC40D0
:100D90000DF1380A0BA83946524610930E950F9460
:100DA000FFF778FE97F834300D98D90739D438F02A
:100DB00063FA04460C980D4638F05EFA02460B982A
:100DC0000B46CDE90223CDE9004538F055FA714ACA
:100DD000CDE90401504640213CF0EAFF402834BFF1
:100DE0000246402283E7D0F80C0138F045FACDE9FD
:100DF0000001D7F8100138F03FFACDE90201D7F829
:100E0000140138F039FA0DF1380ACDE90401624ACB
:100E1000504640213CF0CCFF402834BF02464022DF
:100E200065E75E4938F070FF38F026FA04460D4653
:100E30000C985A4938F068FF38F01EFA02460B4603
:100E40000B9856490792069338F05EFF069B079A67
:100E5000B7E7D0F8F80038F00FFACDE90001D7F87D
:100E6000FC0038F009FACDE90201D7F8000138F0AA
:100E700003FA0DF1380ACDE90401494A50464021F0
:100E80003CF096FF402834BF024640222FE7089BE3
:100E90000A9D099C0DF1380A52460BA83946109359
:100EA0000E950F94FFF7F6FD97F834300D98DA079A
:100EB0002CD438F0E1F904460C980D4638F0DCF9F2
:100EC00002460B980B46CDE90223CDE9004538F0E8
:100ED000D3F9344A7CE7089838F0CEF9CDE900011F
:100EE000099838F0C9F9CDE902010A9838F0C4F937
:100EF0000DF1380ACDE904012B4A504640213CF05F
:100F000057FF402834BF02464022F0E6234938F01C
:100F1000FBFE38F0B1F904460D460C981F4938F035
:100F2000F3FE38F0A9F902460B460B981B490792CD
:100F3000069338F0E9FE069B079AC4E7BB680DF1FB
:100F4000380A1E689C68F06A5D6838F0D5FD316A21
:100F500038F0DAFE38F090F9EB6AE66ACDE9000184
:100F6000184638F0C9FD296A38F0CEFE38F084F909
:100F7000CDE90201304638F0BFFD216A38F0C4FEE9
:100F800038F07AF9094A23E7002A7FF4E9AEEBE664
:100F90008C970500D49605000C9705003333CB41A0
:100FA000F09605002C9705004C9705006C970500FE
:100FB00070B50546C06986B0C5F8F810C5F80C11C3
:100FC000C5F8FC20C5F81021C5F80031C5F814316A
:100FD00030B105F1140005F1F8010122FFF756FECA
:100FE000686801AE036832469B6805F586719847CC
:100FF0000024AB68315918590434F8F739FA0C2C2D
:10100000F7D106B070BD00BFD0F80C11D0F8102198
:10101000D0F81431FFF7CCBF30B4022A00EB8204C1
:101020000346C4F80C110DDD90F87001824201DB1B
:1010300030BC7047C4F8F8109B6830BC53F82200ED
:10104000F8F716BA30BCFFF7DFBF00BF08B58268FB
:1010500012B1C368984708BD37F0A6FF2DE9F047E5
:1010600090F8703186B00546002B6ED0D0F808900D
:101070004FEA8308002401AF59F80460F06A38F0A1
:101080003BFD316A38F040FE385104344445F3D119
:10109000686805F5867403683946DB682246984718
:1010A00023686668A068E26805F1F801C5F8F830C1
:1010B0004E608860CA6023690B61EB6923B105F15A
:1010C00014000122FFF7E2FD6868214603683A46F2
:1010D0009B6898470024AB68395918590434F8F7CD
:1010E000C7F90C2CF7D195F87031032B2ADDA846EF
:1010F0004FF0030A05F12409AB683E591B594846D5
:1011000093F83920314612070BD5EA6A4AB1FFF746
:101110009DFF0146304638F0F7FDAB6839591B5941
:101120000646C8F81861C8F804611846F8F7A0F92F
:1011300095F870310AF1010A534504F1040408F1ED
:101140000408D9DC06B0BDE8F08701AFA0E700BF16
:10115000F8B506460F4600243D592946284638F082
:10116000E5FE294618B9B3681859F8F781F904342F
:101170000C2CF1D13046BDE8F840FFF76FBF00BF3F
:101180002DE9F04F97B090F8703106AF7A619A0070
:1011900002F10A0303F4FF63ADEB030D06AEADEB02
:1011A000030D06AD044628463CF0A3FBE3692BB1D2
:1011B00004F1140029460022FFF768FD94F8353049
:1011C000590730D54FF00009C846A24620465FFABD
:1011D00088F1FFF735FDE8B1DAF858B158465946BD
:1011E00038F0A4FE38B9584655F8091038F094FE86
:1011F000002840F03C81DAF864B15846594638F08E
:1012000095FE38B9584655F8091038F067FE0028A1
:1012100040F02D8108F10108B8F1030F09F104092C
:101220000AF1040AD2D194F87021002A00F03F811B
:101230004FF0000A0023BB614FEA8208D346C7F88B
:101240001CA004EB0A02D2F80C1155F80A0038F081
:101250009DFB8146A84920F0004046F80A9038F0EE
:101260003DFE28B9BBF1020F40F227810123FB614B
:101270000AF1040AC2450BF1010BE2D1FB69002B14
:1012800000F015814FF0000856F808009A4920F048
:10129000004008F1040838F035FE002840F0548181
:1012A000B8F10C0FF0D10023FB6101233B6194F8EE
:1012B00034309E0640F12A8129686A68AB68F96279
:1012C0003A637B6394F870814FF0000BB8F1030F21
:1012D0002BD904F1240342464FF00C09032607F1F1
:1012E0002C0A9846A36855F8091053F809304AF8B3
:1012F000091093F83930404619070CD5E36A53B109
:10130000FFF7A4FE01465AF8090038F049FC94F8AA
:1013100070214AF809003B690136002B40F0D98062
:10132000B24209F10409DDD890463B69002B40F038
:10133000FC807869F96938F0E7FCD4F83C31BB618E
:10134000B8F1000F57D0A368BC604FEA88090026A7
:1013500007F12C0AFD609B4604465BF806505AF8DC
:101360000600696B38F012FB20F0004840466249E5
:1013700038F0B4FD002839D195F8393021465B07A3
:10138000404633D538F00CFC6B6A0246194687E8B4
:101390000C0038F0C1FD3A687B68114658B1184618
:1013A00038F0B2FC0146786938F0FAFBF9697861E7
:1013B00038F0AAFC0446AD6A2946284638F0B6FD46
:1013C000F96998B9404638F09FFCB96938F0E8FBF4
:1013D0002946804638F0A0FD414638B1284638F00D
:1013E00093FC0146B86938F0DBFBB86104364E4522
:1013F000B3D1FD68BC68414E3368B04607E0F8F7EA
:1014000061FED8F8003093F8A4108A074FD493F8FF
:10141000A4601846C6F3C00603212246002EEED172
:1014200018693B6994F87021002B00F08A803346DC
:1014300094F83560D4F84011D7F81CE00193BB69EB
:10144000C6F3400602930391CDF800E07B69049651
:1014500007F12C01FFF790F848B394F8702104F5D8
:101460008670294692003CF044FA012420E094F86A
:101470003540C4F3C004002C00F0B6801F4E336822
:10148000586893F8A420036852074CBF1C491D49B3
:101490009B689847336808F1580258681A490368EE
:1014A0009B689847306807210022F8F70BFE00245C
:1014B00020464437BD46BDE8F08F4946484638F0DF
:1014C0006FFB0146B86938F063FA0123B861FB612C
:1014D000CEE6A3685AF8090053F80930596B3A6010
:1014E00038F054FA014638F05BFB0146584638F0B4
:1014F0004FFA3A68834613E7ACC52737E402001079
:101500001094050018940500989705006068294616
:10151000036807F12C029B6898473E4B1B6893F8C1
:10152000A43098077FF5CEAEC1E7584639F0D0FD1C
:101530003949F86138F0D2FC0028B8D194F87081AC
:10154000F7E607F1200373E7B86939F0C1FD3249C6
:10155000F86138F0C3FC0028A9D1D7F81CB0D7F83F
:1015600014A08046BD6156F80800594638F0CCFBFF
:1015700004EB0802D2F84891054607F1200E00213D
:101580004EF80850484638F0C7FC08F104082946D0
:1015900090B1504638F004FB20F0004529464846FB
:1015A00038F09CFC294638B1484638F0ADFB01467E
:1015B000504638F0F5FA8246B8F10C0FD3D1D4F882
:1015C000546100213046BD69C7F814A038F0A4FC6E
:1015D00040B13046514638F081FC18B100237E619D
:1015E0003B6164E6386162E60A4E336893F8A420F2
:1015F0005868530703684CBF084909499B689847D6
:10160000336808F158025868064903689B68984790
:101610004EE700BFE4020010ACC527371094050068
:1016200018940500D897050070B5C3690446CBB17E
:10163000143001460322984794F83520002363F3C1
:10164000410284F835200D49E3612362D4F820017A
:1016500038F05AFB04F1F805024629462046FFF708
:101660008FFD00B170BD2046D4F8F810D4F8FC20EE
:10167000D4F80031BDE87040FFF79ABC000070421A
:101680002DE9F84F244C814620680E4690F8A410AE
:1016900098468B0700AF92462ED41046002138F0B2
:1016A00027FC044640BB99F8702109F1F80B920021
:1016B00002F10A0303F4FF63ADEB030D68465946DC
:1016C0006D463CF016F9B8F1000F09D04FEA8808D2
:1016D0002859315938F05CF9285104344445F7D180
:1016E00099F8353052466FF3410389F83530484652
:1016F0002946FFF745FD18B90020BD46BDE8F88F23
:1017000099F870215846920029463CF0F2F80120E1
:10171000BD46BDE8F88F00BFE40200102DE9F04F90
:1017200095B0044600AF0E46D0F82401D4F8381125
:101730003A62FB6338F0E8FA0021B86297F87C500F
:1017400038F0D6FB002840F0218294F8363094F827
:10175000358003F0030303F13E0254F822103A6A85
:10176000C8F301194FEA981852F8230009F13E0214
:1017700008F13E0354F8222054F82330BA63FB6288
:1017800038F004F93B6A834653F82960FB6BB86B69
:1017900053F8299053F82830C7F834907A6B3B639C
:1017A00002F10042BA643B6A3A6B314653F8288032
:1017B00002F1004A38F088FB30B1F86A414638F04F
:1017C00083FB002840F08C81B96B304638F0DEF89E
:1017D000796B38F0DBF8F96A0646404638F0D6F8FF
:1017E000396B38F0D3F880464146B86C38F0D8F9F8
:1017F00031468146504638F0D3F90146484638F024
:10180000C5F831468146B86C38F0CAF941460646FB
:10181000504638F0C5F90146304638F0B9F801466F
:10182000484639F061FA94F83630804603F00303F5
:10183000012B08BF85F001050021002D00F0C081BB
:1018400038F06AFB20B14046A84938F09FF880463E
:1018500094F87061B300023B23F00703ADEB030D76
:10186000032E6D460FDD3B6AD4F80411D86838F0BA
:101870008DF8042E009006D0396A0869D4F8081152
:1018800038F084F80190B96F404638F089F92BF0B0
:10189000004136F013FD9649786438F01FFB0028AC
:1018A00040F06F81D4F8309100214846D4F82C6183
:1018B00038F032FB68B1B86F014638F069F803467A
:1018C000194648467B6038F009FB7B68002840F0E9
:1018D0008F813046874938F001FB08B14FF07C56C4
:1018E0003146786C38F010FA39F008F938F05AFBC4
:1018F00080B20128786240F2788138F0FDF806461F
:101900003146404638F000FA31463864584638F0DF
:10191000FBF994F87021C7F810D0A2F10308FA641B
:101920004FEA880202F10A0323F00703ADEB030D2F
:10193000B8F1000FB8617A64C7F814D013DD4FF026
:10194000000BC146D7F81480FC615C4655F80B00CB
:10195000314638F0D9F901344C4548F80B000BF109
:10196000040BF3DBFC69386C4FF07C5138F018F94C
:10197000396C38F015F901464FF07E5038F006F812
:101980007A6CF86102F1160323F00703ADEB030D47
:10199000FB6C68469A0004F1F8013BF0AAFF94F84A
:1019A0003630002003F0030303F13E0254F82220F6
:1019B0006D467864F8644DF8232001264E490B6883
:1019C00093F8A430C3F34003002B40F00781786CF8
:1019D000D4F8442141B2914280F292805046F96994
:1019E00038F0DEF8396C8346B86C38F0D9F85946CF
:1019F00037F0CEFFF9698346B86C38F0D1F8396C0E
:101A00008046504638F0CCF80146404637F0BEFFDD
:101A10007B6C94F8352003F101095FFA89F9B86409
:101A2000DA46C7F84490C2F30118796BB86B37F007
:101A3000AFFFB96C37F0ACFF396B45F82800F86A96
:101A400037F0A6FF514637F0A3FF94F835B0B969D7
:101A50004FEA9B1B45F82B0094F836B00BF0030BB4
:101A600055F82B0037F094FF45F82B0094F87031AF
:101A7000032B15DD7B69AB46A3F104084FF0030986
:101A8000DBF80C0058F8041F37F082FFCBF80C008D
:101A900094F8703109F101094B450BF1040BEFDCAF
:101AA00029462046BA6AFFF76BFBF96C013600291C
:101AB00008BF0146786AB3B28342F964FFF47EAF8F
:101AC0003B699D46396ABA6A2046FFF759FB0028F0
:101AD000F86C07F1540718BF0120BD46BDE8F08F30
:101AE000002D78D0DFF81480B2E600BFDB0FC940CC
:101AF000BD37863517B7D138E4020010DB0FC9C0F7
:101B000030467B6037F0F8FF396C38F049F8804692
:101B100038F0BAFF8246404639F0A8F894F835E02C
:101B2000FA6BCEF30118834652F828004FEA9E1E46
:101B300000F1004C6046514652F82E90C7F808C09C
:101B400038F02EF8594602464846FA6038F028F830
:101B5000FA680146104637F01BFFD7F808C0B86492
:101B60006146584638F01CF849468346504638F0DE
:101B700017F87B68014658467B6437F007FF8246BA
:101B800053E700205437BD46BDE8F08F337AB86A7A
:101B900043F010033372002138F096F9204B2149AD
:101BA000002806F1100608BF1946304614BF13225C
:101BB0000D2236F06FFF00205437BD46BDE8F08F90
:101BC00038F08CF900283FF443AE4046164937F010
:101BD000DFFE80463CE6DFF8508039E63B690020B6
:101BE0009D465437BD46BDE8F08F0023FB6469E78E
:101BF0001846494637F0CAFE0146484637F0D0FF3E
:101C000039F066FA014637F0C3FED4F82C1181464C
:101C100038F082F900283FF45CAE4E4659E600BF2A
:101C2000209805000C980500DB0FC9402DE9F04114
:101C3000054690F835001446C0F30117820982B0BA
:101C40000E4654F8270054F822101F469DF82080B5
:101C500036F034FBB8F10302534253410090019334
:101C6000284631463A462346FFF758FD02B0BDE804
:101C7000F08100BF2DE9F04F8BB0044600AF0D4658
:101C800018460021BB61BA6038F032F9002840F0F4
:101C9000F480B9680868D4F8F81037F077FEBA68AD
:101CA0008346D4F8FC10506837F070FEBB680646D7
:101CB000D4F80011986837F069FE31468046304606
:101CC00037F06EFF59460646584637F069FF014621
:101CD000304637F05DFE41460646404637F060FF2D
:101CE0000146304637F054FE39F0F2F99A4906467B
:101CF00038F0F4F8002840F0F980386D014638F0EB
:101D000015F90246C8B92B7A590716D56B68012B0D
:101D100013D13B6D3146B8693B623A6037F0F4FF4E
:101D20003A6878624EF289014AF6765007F120034C
:101D3000F7F7AEF8002840F0F38094F83430C3F39E
:101D400000113961002940F0BC805A0640F1D98069
:101D5000D4F834514FF07E51284638F0DDF8002891
:101D600000F0A780B969304637F0CEFF014628461B
:101D700037F016FF38F044FE4FF07E51054638F03C
:101D8000CBF8002800F09D80284638F00BF980B28F
:101D900078617B69012B40F2948094F87021C7F838
:101DA00004D0920002F10A0303F4FF63ADEB030DCC
:101DB000C7F80CD0ADEB030D684604F1F801C7F885
:101DC0001CD03BF096FD94F87031FBB178693B6014
:101DD00037F092FE3B68D7F80C80D7F8089006469B
:101DE0009D004FF0000B9A4604EB0B03D3F8F8105C
:101DF00059F80B0037F0CAFD314637F085FF48F837
:101E00000B000BF1040BAB45EED15346DFF854B198
:101E1000DBF8002092F8A450C5F34005002D40F0F7
:101E200085800126A3B1FB68D7F81C80A3F10409C3
:101E30004FF0000AD8F8000059F8041F37F0A8FD49
:101E400048F8040B94F870310AF1010A9A45F1DB65
:101E50002046F969BA69FFF793F97B690136002DCD
:101E600008BF05469E4268D0DBF8003093F8A430E6
:101E70009B075BD494F87031D4E72B7AB86943F0B0
:101E800010032B72002138F01FF8344B344900281E
:101E900005F1100508BF1946284614BF13220D226C
:101EA00036F0F8FD00233B6138692C37BD46BDE8AC
:101EB000F08FD4F828510021284638F005F8002882
:101EC0003ED00025B968BA692046FFF759F90028C5
:101ED00018BF012594F834303D6138696FF3C303AE
:101EE0002C3784F83430BD46BDE8F08FB968BA6944
:101EF0002046FFF745F9386138692C37BD46BDE803
:101F0000F08F284658211CF007FC00287FF420AFF2
:101F1000284659211CF000FC00287FF419AFD0E7B7
:101F2000B869796A37F03CFEB86106E77B683869C2
:101F30009D462C37BD46BDE8F08F7B689D46C1E7C6
:101F40002946304637F0E0FE38F05AFD38F02AF8DE
:101F500080B278611DE700BFACC527372098050027
:101F60000C980500E40200102DE9F04F8FB0B74B3C
:101F700002AF07F1200804460D46BA600FCB88E88F
:101F80000F00002606F158095FFA89F949462846EC
:101F90001CF0C2FB002840F021810136032EF1D154
:101FA00000234FF000097B61BB61FB614926284695
:101FB00031461CF0B1FB002840F0FF800136F6B23C
:101FC0004C2E09F10409F2D194F8702104F1F803C0
:101FD00092007B6002F10A0303F4FF63ADEB030D93
:101FE0000DF10809484679683BF083FC94F83460A9
:101FF000320700F11C81C6F34006002E00F08480F9
:102000003E6A3046314637F091FF98B994F8A430D3
:10201000304603EB430304EB8303196C37F0B8FC41
:10202000D4F8B01037F0B2FCD4F8BC1037F0B0FCE4
:10203000C9F800007E6A3046314637F077FF98B91C
:1020400094F8A430304603EB430304EB8303D96BCD
:1020500037F09EFCD4F8AC1037F098FCD4F8B810E8
:1020600037F096FCC9F80400BE6A3046314637F0B6
:102070005DFFA0B994F8A43004F1380203EB4303E8
:1020800052F82310304637F083FCD4F8A81037F00C
:102090007DFCD4F8B41037F07BFCC9F80800284662
:1020A00045211CF039FB002846D1694AFA6094F8B2
:1020B0007031032B61DDA0464E464FF0030B09E063
:1020C00094F870210BF1010B5A4508F1040806F150
:1020D000040652DD0BF13E025FFA82FA51462846B1
:1020E0001CF01AFB0028EBD05146002228461CF0B9
:1020F00027FB94F834200146930703D4D8F8040151
:1021000037F046FCF060DBE758F806A05046514631
:1021100037F00CFFA31930B9D3F8F810504637F058
:1021200037FC49F8060004360C2EEDD1284645212F
:102130001CF0F2FA0028B8D02046FEF751FD4521E8
:102140000646002228461CF0FBFA002EF860ACDDA3
:10215000014637F0EBFE0028A7D194F834305B0736
:1021600040F18480F86806F13E0354F8231049F8E2
:10217000260037F00BFCF86099E7284646211CF052
:10218000CBFA90B1BA682846012A4FF046014FF0C9
:10219000000278D01CF0D4FA94F83430D90702D574
:1021A0002C4937F0FDFCC4F82401BA68531E032BF8
:1021B00039D8DFE803F06522515131462846002224
:1021C0001CF0BEFA94F834302249DB0701D537F011
:1021D000E7FC07F1140349F80300EFE649462846F7
:1021E00000221CF0ADFA94F834301A49DB0701D50F
:1021F00037F0D6FC48F82600CFE6D4F82401D4F80E
:10220000381137F081FDFA680346009229462046CE
:102210004A46FFF72FFD30B194F87021786892009C
:1022200049463BF066FB3437BD46BDE8F08F0026DB
:1022300058F806A05046514637F078FE08B949F8DC
:1022400006A004360C2EF3D129E700BFE89505005F
:102250000000C07F3333CB41BB6829460093204642
:1022600007F114024B46FFF7E1FCD4E706F13E0309
:1022700054F82310F86837F08BFB49F8260016E76E
:10228000D4F82001BBE71CF05BFA94F83430DE0789
:1022900002D5034937F084FCC4F82001AFE700BF42
:1022A0003333CB4170B50646006868B1756A74690E
:1022B0000435AC4206D254F8040BF9F7FDF9A542F7
:1022C000F9D83068F9F7F8F9304670BD0E4B10B503
:1022D000044640F8D03BFFF7E5FFE36A23B104F181
:1022E0002400014603229847E36923B104F1140056
:1022F000014603229847A06808B1F9F7DDF92046A6
:10230000F9F712FD204610BD40960500104B10B5A0
:10231000044640F8D03BFFF7C5FFE36A23B104F160
:102320002400014603229847E36923B104F1140015
:10233000014603229847A06808B1F9F7BDF9204685
:10234000F9F7F2FC2046F9F7B7F9204610BD00BFB7
:1023500040960500F8B5426803680446D31A9B10FE
:102360000F4605D05A00934226D96FF0030600E0CD
:102370000426304635F076FF054694E809001B1A1E
:102380009B109A003968AF1807D045F8231094E8DD
:1023900009001B1A9B109A00AF1823B1014628466A
:1023A0003BF0B0FA2068043708B1F9F785F92E44FC
:1023B000A66084E8A000F8BDB2F1804FD5D2DE005F
:1023C000D7E700BF30B5184D83B02B680446986A34
:1023D0000191FAF7EFF894F87031042B06D92B68C5
:1023E0001249586803689B68984700BEE3682269F1
:1023F000934211D0019A13B11A60E368019A043331
:10240000E36094F8703182F8383094F87001431C1E
:1024100084F8703103B030BD04F1080001A9FFF762
:1024200099FF019AEDE700BFE40200103098050023
:102430002DE9F04F044640689DB010B103685B6819
:102440009847304D00222968134648694FF22141D0
:10245000F8F792FE0DF11C0A05AA06462A495046D5
:1024600036F012FD30465146F9F754FC01460DA8EE
:10247000F9F724FC0DA8F7F731FF0D9BDFF89080EA
:102480000646A3F10C00404540F0D5830DF1180934
:10249000079BA3F10C00404540F0E78341F6AE43B3
:1024A0009E4200F027834EF29C539E4200F022830E
:1024B0004EF29D639E4200F0558345F208139E4202
:1024C00028D041F293139E4224D041F60C339E4211
:1024D00020D0B6F5F47F1DD041F2DE139E4200F00D
:1024E000638345F60F539E4200F078834EF6866371
:1024F0009E4200F07D83042035F0B4FE034B036060
:10250000606010E0E40200106498050050FC0500D3
:102510005C0A0010442035F0A5FE2B680646596978
:1025200026F06CF966602B680022586941F6E911C3
:102530001346F8F721FEC149F9F7E8FBF9F71EFB4E
:10254000296800221346C4F8240148694BF6FD01AE
:10255000F8F712FEB949F9F7D9FBF9F70FFB29682B
:1025600000221346C4F82001486947F2E051F8F709
:1025700003FE0021F9F7CAFBF9F700FB29680022E6
:102580001346C4F82801486943F65A71F8F7F4FD78
:102590000021F9F7BBFBF9F7F1FA2968002213468D
:1025A000C4F83401486943F66E41F8F7E5FD0021AF
:1025B000F9F7ACFBF9F7E2FA296800221346C4F8F0
:1025C0002C0148694DF6A361F8F7D6FD9C49F9F74F
:1025D0009DFBF9F7D3FA296800221346C4F83001AD
:1025E000486941F2D231F8F7C7FD0521F9F782FBBE
:1025F000F9F7C4FA37F0B0FC296800221346C4F892
:10260000440148694FF6A751F8F7B6FD8D49F9F72F
:102610007DFBF9F7B3FA8C4937F076FB2968002285
:102620001346C4F84801486940F6A861F8F7A4FDCC
:102630008449F9F76BFBF9F7A1FA834937F064FB9A
:10264000296800221346C4F84C01486941F6A96183
:10265000F8F792FD7D49F9F759FBF9F78FFA7A49B6
:1026600037F052FB296800221346C4F8500148692C
:102670004CF6B951F8F780FD7549F9F747FBF9F7C2
:102680007DFA714937F040FB296800221346C4F8EF
:102690005401486948F25B71F8F76EFD0121F9F7C2
:1026A00029FBF9F711FB94F834302968002260F314
:1026B000861384F834304869134645F6E271F8F71A
:1026C0005BFD0021F9F716FBF9F7FEFA94F83430B8
:1026D0002968002260F3C71384F834304869134630
:1026E00045F6E011F8F748FD2B6893F8A410C1F304
:1026F0008001F9F7FFFAF9F7E7FA94F8353000228C
:1027000060F3000384F8353029681346486942F2C3
:102710007F71F8F731FD4A4606464E490DA836F05E
:10272000B3FB0DA93046F9F7F5FA014604A8F9F70D
:10273000C5FA0D9BA3F10C00404540F0A28204991C
:1027400051F80C3C002B40F0DC812B6800225869CA
:1027500044F6D6311346F8F70FFD3F49F9F7D6FA9C
:10276000F9F70CFA3D4EC4F8400106F1300C0DF1BA
:10277000340E30687168B268F36877460FC7103658
:102780006645BE46F5D130687168B2682B68AEE820
:1027900007000022586946F2EE211346F8F7ECFCD8
:1027A0002649F9F7B3FAF9F7E9F90DAF0097C4F83C
:1027B0003C0100265046F5F7DDFA09A8F5F7DAFAEC
:1027C0000BA8F5F7D7FA4FF0000BDDF800C02B6827
:1027D00000223CF80B1058691346F8F7CDFC02AA0A
:1027E00007461F4905A836F04FFB05A93846F9F7FB
:1027F00091FA01464846F9F761FA0AEB8B0049461F
:10280000F5F7A0FC8179069B8907A3F10C020BF177
:10281000020B09D590F804E00168012000FA0EFED1
:1028200008684EEA00000860424540F0F781059BC9
:10283000A3F10C00404540F0E58113E00000C842E0
:102840000AD7233C00606A470000704200009643AC
:10285000000070C20CE90500CDCC4C3FF895050096
:10286000EC820500BBF1060FAFD19DF822309A072C
:1028700040F132819DF82A309B0740F12D813C20A8
:1028800035F0F0FC5146074609AA0BABF6F76CFD94
:1028900020463946FFF796FDB042834640F04A8114
:1028A0002B6806EB46011CAA02EB8101A7680022F7
:1028B00031F8361C5869134657F82670F8F75CFC57
:1028C000022E0CBFBD49BE494FEA860CCDF804C0AC
:1028D000F9F71CFAF9F752F901463846F6F7BCFD4C
:1028E0000BEB4B0B0DF1700E2B680EEB8B0B0022DC
:1028F000DDF804C0A7683BF8341C5869134657F844
:102900000C70F8F739FCAF49F9F700FAF9F736F926
:10291000AD4937F0F9F92B68D4F808E0DDF804C0C8
:10292000002278623BF8321C586913465EF80C703E
:10293000F8F722FCA549F9F7E9F9F9F71FF9DDF8ED
:1029400000C001360CF10C0C052ECDF800C0B862A9
:102950007FF430AF2046FEF7DFF8A3689B68986AE3
:10296000014637F0E3FA002840F00681606804F180
:10297000F801036852469B6898470026A3685AF8F6
:10298000061098590436F6F773FD0C2EF6D194F81C
:102990007031032B0FD9A368D4F80411D868F6F767
:1029A00067FD94F87031042B05D9A368D4F8081199
:1029B0001869F6F75DFD2B6847F2693241F21D3167
:1029C00058690023F8F7D8FB0021F9F793F9F9F7D4
:1029D0007BF994F8353041F2AA3260F3820384F82F
:1029E00035302B6841F21D3158690023F8F7C4FBDC
:1029F0000121F9F77FF9F9F767F994F8353046F2D4
:102A00001D1260F3C30384F835302B6841F21D3189
:102A100058690023F8F7B0FB6C49F9F777F9F9F733
:102A2000ADF82B6846F21E62C4F8580141F21D3120
:102A300058690023F8F7A0FB6449F9F767F9F9F73B
:102A40009DF82B6846F61F32C4F85C0141F21D3137
:102A500058690023F8F790FB5C49F9F757F9F9F743
:102A60008DF82B6845F61F32C4F8600141F21D3124
:102A700058690023F8F780FB5449F9F747F9F9F74B
:102A80007DF82B6846F22002C4F8640141F21D3142
:102A900058690023F8F770FB4C49F9F737F9F9F753
:102AA0006DF82B6846F22152C4F8680141F21D31DD
:102AB00058690023F8F760FB4449F9F727F9F9F75B
:102AC0005DF8049BC4F86C01A3F10C00404540F094
:102AD000C0801DB0BDE8F08F022E3FF63BAF2B68E3
:102AE0003B49586806F1580203689B68984784F888
:102AF000706127E0042035F0B5FB364B0360606061
:102B000011E50DA8F8F74EF90D980E9B1B1A9B10B6
:102B1000032B05D000283FF418AEF8F7CDFD14E6DE
:102B2000816843680268C4F8A810C4F8B020C4F8EB
:102B3000AC30EFE72B685A465868334601688C681A
:102B40002549A047049BA3F10C004045C1D053F890
:102B5000042C511E002A43F8041CBADC514635F0FF
:102B6000EDFEB6E70C2035F07DFB2B680646596973
:102B700026F0F8F86660D6E42B68002258694EF615
:102B8000C8411346F8F7F8FA1049F9F7BFF8F8F713
:102B9000F5FF0146064637F0C9F900287FF4E6AE96
:102BA000A3689B689E62E1E60C2035F05BFB2B6816
:102BB0000646596927F01CFC6660B4E40000204515
:102BC0000000A0420060EA46000070420000C07FA2
:102BD00070980500F0FA05009C980500282035F053
:102BE00041FB2B680646596926F068FD66609AE449
:102BF0002C2035F037FB2B680646596926F044FA3D
:102C0000666090E453F8042C511E002A43F8041C1B
:102C10003FF728AE494635F091FE23E653F8041CF1
:102C2000481E002943F8040C3FF701AE104603A9E3
:102C300035F084FEFBE553F8042C0DF11809511E04
:102C4000002A43F8041C3FF723AC494635F076FED2
:102C50001EE453F8042C511E002A43F8041C3FF7CD
:102C600038AF494635F06AFE33E753F8042C511E5D
:102C7000002A43F8041C3FF711AC0DA935F05EFEA5
:102C80000CE453F8042C511E002A43F8041C3FF7AF
:102C900056AD514635F052FE51E500BF10B5022148
:102CA0000446F9F757F82046BDE81040FFF7C0BBCF
:102CB0002DE9F84305462A6840682B4B821A92108A
:102CC00003FB02F38846002B45D05A00934244D9B7
:102CD0006FF00306304635F0C5FA6C68D5F800C0D1
:102CE0000746CCEB040323F00303C31800F10C09DF
:102CF0001CBF98E8070083E80700A4451FD063467F
:102D00003A462AB119681160596851609968916012
:102D10000C33A34202F10C02F3D10CF10C09C9EB04
:102D20000303124A9B0802FB03F929F0404909F109
:102D3000010909EB490907EB890909F10C09BCF103
:102D4000000F02D06046F8F7B7FC3E44AE6085E85D
:102D50008002BDE8F8830C26BCE705498A42B7D853
:102D600002EB83039E00B5E7ABAAAAAAABAAAA2AE4
:102D7000555555152DE9F0470023036043608360E6
:102D800005460C20884691F8A49035F06BFA6E68E1
:102D90002F680446F31B23F0030310EB030A09D04A
:102DA0003C4A0021E1504846CAF8042036F0A0FE13
:102DB000CAF80800BE4268D03A4623462BB11168D3
:102DC000196051685960916899600C32964203F11C
:102DD0000C03F3D107F10C03F31A2F4A9B0802FBF3
:102DE00003F323F04043013303EB430304EB830974
:102DF00009F10C0917B13846F8F75EFC08F1380301
:102E000008F1A40704F10C06BB422C60AE60C5F8C3
:102E100004903CD01C464B469E4221D01BB194E806
:102E2000070083E807000C336B600C34A742F3D132
:102E3000B34222D023B108F1A80207CA83E80700F1
:102E40000C336B60B34212D02BB108F1B40898E890
:102E5000070083E807000C336B602846BDE8F08765
:102E600028462146FFF724FF6B68AE68DDE708F1CE
:102E7000B4012846FFF71CFFEFE7284608F1A80138
:102E8000FFF716FF6B68AE68DCE7A146B0E74B467C
:102E9000CEE700BF00001041ABAAAA2A70B50C46CD
:102EA000064609B90AE02C463046E168FFF7F6FF0E
:102EB000A5682046F8F700FC002DF4D170BD00BFD6
:102EC000D0F808C02DE9F843064600F10408BCF12B
:102ED000000F51D00A7847466446237C934223D2A0
:102EE000E468002CF9D13C46F368D6F81490A3426C
:102EF00034D0A74208BF4FF0000912D0204635F069
:102F00005FFA41460546204635F0CBFAF8F7D4FB88
:102F10007369BD4203F1FF332C467361EED1C3EBFD
:102F200009094846BDE8F88304D92746A468002C5F
:102F3000D3D1D8E7A068E36838B1057C95422ABFB1
:102F40000446C06880680028F7D1002BCCD0187CDC
:102F500090428ABF1F46DB689B68F6E7B845C8D138
:102F600061463046FFF79AFF0023C6F80C80C6F88A
:102F70001080B3607361D4E74746B4E72DE9F84F9A
:102F8000224D4FEA510AA5FB0A25AD08EB1C082B80
:102F900038BF0823064643609800894635F062F939
:102FA000736801355B1B4FEA530B00EB8B0707EB94
:102FB0008505AF428046306038BF3C4607D24FF4AB
:102FC000FC7035F04FF944F8040BA542F7D80F4BCD
:102FD0007761A3FB0A2A58F82B202A234FEA9A0A82
:102FE00003FB1A9902F5FC712B1F3161F2607362C9
:102FF00055F8043C09EB490903F5FC7003EB890122
:10300000B260F3613062B161BDE8F88F310CC3305A
:103010002DE9F0438BB08046F8F796FE794B0024FB
:1030200008F1380921466C22C8F80030C8F8084079
:10303000C8F80C40C8F81040C8F81C40C8F82C402C
:1030400048463AF07AFC0023214688F8A44088F8E4
:10305000C040C8F8A830C8F8AC30C8F8B030C8F8DC
:10306000B430C8F8B830C8F8BC30C8F8C430C8F8B4
:10307000C830C8F8CC306846009401940294039498
:10308000049405940694079408940994FFF776FF36
:10309000C8F8D040C8F8D440C8F8D840C8F8DC40D8
:1030A000C8F8E040C8F8E440C8F8E840C8F8EC4088
:1030B000C8F8F040C8F8F440214608F1D000FFF706
:1030C0005DFF009C7CB3D8F8E05008F1D80E02AB4D
:1030D0000FCBD8F8D870D8F8DC600495D8F8E45055
:1030E0008EE80F0005950AAD15E90F00D8F8E850F5
:1030F00008F1E80E0695D8F8EC5002970795D8F835
:10310000F05003960895D8F8F4508EE80F00099512
:10311000D8F8D020C8F8D040D8F8D43001998DE83C
:103120000C00C8F8D4106846FFF7BCF898F83410C3
:1031300098F8352098F836300124022001F0FE017D
:1031400002F0CF0260F3010364F3871241F006013D
:1031500088F8363088F8341088F835200021142299
:1031600008F1F8003AF0E9FB142208F58670002116
:103170003AF0E3FB244AD8F81C5000230024C8F896
:103180003821C8F8BC30C8F8B830C8F8B430C8F82E
:10319000044045B108F1140001460322A847C8F8CD
:1031A0001C40C8F82040D8F82C304BB108F124005E
:1031B0000146032298470023C8F82C30C8F8303065
:1031C0000023484608F1A4018360436040F80C3BAB
:1031D00088424FF00002F7D198F83430002103F014
:1031E000E7036FF345134046C8F8B020C8F8AC2099
:1031F000C8F8A82088F8343088F870110BB0BDE802
:10320000F08300BF40960500000070422DE9F843AE
:1032100090E80C00456A0446A81AA3EBA000012818
:103220000E4615D94FF4FC7035F01CF86860A369A0
:103230001BB196E8070083E80700636A1A1D626203
:103240005B6803F5FC72E361A3612262BDE8F88369
:103250006169C1EB05084FEAA80808F1010808F107
:103260000107B3EB470F31D8002B3FD05B009D1C0B
:10327000B5F1804F45D2A80034F0F4FF636A61696C
:103280000433EF1B5B1A7F089A10814600EB870717
:1032900003D0920038463AF035FB2068F8F70CFA74
:1032A000C4F80090656067613A6808F18043013BAB
:1032B00007EB830502F5FC71E2606562216157F856
:1032C000233003F5FC72E3612262ABE7DF1B7F086A
:1032D00002EB87070435B942C1EB050508D9AA10EE
:1032E000E1D0920038463AF00DFBDCE70325C2E757
:1032F000AD10D8D0AA0007EB8800801A3AF002FB84
:10330000D1E735F045FE00BFF0B50346D0F8F01028
:1033100090F83420D3F8E84090F8A460D0F8205119
:103320000C39D0F8240185B0C2F3400CC2F38007F9
:103330008C42C2F300028DF807C08DF806708DF83C
:1033400005208DF80460029503900CD034B104ADD3
:1033500015E9070084E80700D3F8E8400C34C3F807
:10336000E84005B0F0BD03F1D00001A9FFF74EFF22
:10337000F7E700BF2DE9F04F0D46097A99B0C1F388
:1033800080060446002E00F0D2806A685C2A00F2B3
:10339000BF80DFE812F09202FB00B60295029B01AB
:1033A000BD00BD00BD00BD00BD002F02BD00BD00C1
:1033B000BD00BD00BD00BD001E020D029702AF02A0
:1033C000A802BD00BD00BD00BD00BD00BD00BD0028
:1033D000BD00BD00BD00BD00BD00BD00BD00BD0005
:1033E000BD00BD00BD00BD00BD00BD005D00BD0055
:1033F000BD00BD00BD00BD000502BD00BD00BD009B
:10340000BD00F001F001F001F001F001F001BD009C
:10341000BD00BD00BD00BD00BD00BD00BD00BD00C4
:10342000BD00BD00BD00BD00BD00BD00BD00BD00B4
:10343000BD00BD00BD00BD00BD00BD00BD00BD00A4
:10344000BD00BD00BD00BD00BD00E901E0011401EB
:10345000C1F34213073303F00703012B58D80023AD
:10346000284658211293139314931BF055F9002802
:1034700041F04981284659211BF04EF9002841F0BE
:10348000338128465A211BF047F9002841F05A8120
:10349000DDF85090DDF848A000215046D4F8BC80FB
:1034A000D4F8B870D4F8B46036F00EFD20B94046B8
:1034B000514636F06DFA8046DDF84CA000215046AA
:1034C00036F002FD20B93846514636F061FA07461B
:1034D0004846002136F0F8FC20B93046494636F01F
:1034E00057FA06462B7AC4F8BC805B09022BC4F855
:1034F000B870C4F8B4600BD1D4F83811D4F82001F6
:1035000036F002FC12A9024603232046FEF7B8F863
:1035100094F835306FF3410384F8353094F8343043
:103520006FF3C30384F8343019B0BDE8F08F8F0710
:10353000EED52A68722A00F0348415D8122A00F0D9
:10354000F68340F24382532A00F02F8200F26A820F
:103550001E2A00F0FA85522ADAD190F8343043F06E
:10356000040380F83430D3E7D32A00F0938300F2C9
:103570004582CB2A00F0C78100F2A282782A00F0AF
:10358000D283792AC4D1FDF703FAC1E7022728467E
:1035900053211BF0C1F830B12846532100221BF003
:1035A000CFF8C4F8400194F83530294666F341035A
:1035B0003A4684F835302046FEF7D6FCAEE74B0994
:1035C000DA1D02F00702012A40F2A68228461BF00B
:1035D00021F92B7A5B09002800F09E82042B01F070
:1035E0002680032B00F0BB86D4F80071D4F8FC6071
:1035F000D4F8F8300FA8214612AA12971396149304
:10360000D4F8B080D4F8AC70D4F8A860FDF742FAD2
:10361000284658211BF080F8002840F0A58728464E
:1036200059211BF079F8002840F0CA8728465A2112
:103630001BF072F8002840F0AD872B7AC4F8B080F8
:10364000C4F8AC70C4F8A8605B09002B00F0AD852D
:103650009A077FF469AF28461BF0DCF800287FF753
:1036600063AF94F87031032B7FF75EAF27460326D4
:1036700006F13E085FFA88F84146284600221BF012
:103680005FF8A368814653F82630002193F839305B
:103690004FEA860A1B0702D536F016FC70B1414688
:1036A00028461BF039F8494640B1C7F81891C7F8C9
:1036B0000491A36853F80A00F5F7DAFE94F8703124
:1036C0000136B34207F10407D2DC2DE7284650212A
:1036D0001BF022F8002800F0B482C54B28461B6876
:1036E000502193F8A420C2F38002002A00F09585AF
:1036F00000221BF025F8BF4936F052FA36F052FC92
:103700000646284653211BF007F8002840F0548154
:10371000002E3FF4FDAEB64D01212B68986901F0F3
:1037200017FB33F029FA4FF47A73074603FB06F6CA
:1037300008E02868F6F7C6FC2B6893F8A4309807D1
:103740003FF5F2AE33F018FAC01BB0424FF0030160
:103750002246EED3DCE690F8343003F0FD036FF33D
:10376000820380F83430D3E690F8343043F0060317
:1037700080F83430CCE6363AD2B280F8A4206B68B8
:103780003B2B7FF4C5AE2B7A5B093FF4C1AE1344EB
:10379000DBB2082B40F2DB81082380F8A430B7E6C7
:1037A0000023C0F8BC30C0F8B830C0F8B430AFE681
:1037B00090F8352090F8363002F0CF020220012137
:1037C00060F3871261F3010384F8352084F8363002
:1037D0009EE690F8352090F8363002F0CF020120B6
:1037E000022160F3871261F3010384F8352084F825
:1037F00036308DE628464C211AF08EFF00283FF423
:1038000087AE28464C2100221AF0BCFF022807D0C0
:1038100028464C2100221AF0B5FF14287FF478AE18
:10382000284650211AF078FF00283FF471AE284650
:10383000502100221AF0CAFF002840F08D8594F82C
:10384000A430082B3FF664AE03EB43034FEA830A30
:1038500004F1380B0BEB0A0728464C210022D7F85D
:103860000890D7F804805BF80A601AF08BFF1428E0
:1038700001F0378094F834202846C2F340025821E2
:10388000002A00F09B871AF047FF002841F074805F
:10389000284659211AF040FF002841F08F80284621
:1038A0005A211AF039FF002841F07780C7F80890B4
:1038B000C7F804804BF80A602AE60026012766E66E
:1038C000042764E690F83520012363F3051290F88D
:1038D0003630022161F387126FF3010380F835203F
:1038E00080F8363014E690F834306FF3000380F837
:1038F00034300DE690F8343043F0010380F8343072
:1039000006E6032743E628461AF084FF002840F025
:103910009C8407465826A146A846D8F80C4098F83B
:103920000820236852099D6818BFD9F8083009EBB0
:10393000070116BFDB59D1F84801586A35F09CFCE5
:103940003246CDE90001013620462B49A8475B2EBF
:1039500007F10407E1D198F808304C465B09012BC8
:10396000454640F05F8499F87061032E40F2678409
:10397000032703E00137BE4240F26184A36853F895
:10398000273093F839201207F4D4586A35F074FCC4
:10399000EB6807F13E021E68CDE900011846B668E3
:1039A0001549B04794F87061E4E790F8343066F355
:1039B000820380F83430ABE52846532100221AF008
:1039C000E1FE4FF47A7303FB0066A1E6032A00F0E0
:1039D0003A8140F2A980052A00F09581112A7FF4EE
:1039E00097AD034B082118680122F6F76BFB8FE5B2
:1039F000E402001000007A44E4980500B2F5FA7F72
:103A000000F0388200F2A680DC2A00F0A683B2F52E
:103A1000C87F7FF47DAD994B01211B68986901F047
:103A200097F975E5542A00F000815C2A7FF470ADA7
:103A300090F870610027C6B9AEE3A368D5F80C9082
:103A400053F80830D9F80080186A35F015FCCDE934
:103A500000013246D8F8083048468949984794F81A
:103A600070610137BE4240F39783A3684FEA87082D
:103A700053F8273093F839301A07F2D4022FD4BF05
:103A800007F1580607F13E06F6B2284631461AF00D
:103A900043FE0028D1D0A36831462846002253F8BF
:103AA00008901AF04DFE94F834300146DB0703D538
:103AB000744936F075F801464846F5F7CDFCBCE789
:103AC000CC2A00F09081CD2A7FF422AD28465821DF
:103AD0001AF022FE002840F02E8528465A211AF0BE
:103AE0001BFE002840F01585284653211AF014FECD
:103AF00000283FF40DAD2846532100221AF020FE85
:103B00000021054636F0EAF9002840F07F865B4B3D
:103B10001B681B695D61FBE40022C4F8B020C4F897
:103B2000AC20C4F8A82090E5022A7FF4F1AC534BF6
:103B30001B689869012101F00BF994F83410524A7E
:103B400041F00201002384F83410C4F8382184F8CD
:103B5000A430DDE440F2F7139A4200F08B8140F28A
:103B600099239A427FF4D4AC0DF148084046294687
:103B70001AF04EFF18AE532306F8243D3146404656
:103B8000FFF79EF95523314640468DF83C30FFF74C
:103B900097F9179B002B40F0148440461499FFF7C7
:103BA0007DF913AF00226068159716971492036889
:103BB000414617925B699847C8B1159EBE4216D020
:103BC000B946706935F058FBEB68327C1F68CDE967
:103BD0000001BF6818462D49B8472B7A304643F09C
:103BE00001032B7234F0D9FB48450646E9D128463B
:103BF00053211AF091FD0646002800F05983002257
:103C0000284653211AF09CFDED68C4F8340135F0C4
:103C100033FB2E6802460B46B66828461C49B0475F
:103C200040461499FFF73AF972E4144D01212B68CC
:103C3000986901F08DF8286808210022F6F742FA09
:103C400066E406465DE590F8363058077FF560ACCF
:103C50000A4B01211B68986901F07AF82846532124
:103C60001AF05AFD00283FF453AC2846324653213F
:103C70001AF066FDC4F840014AE400BFE4020010F7
:103C8000DC9805003333CB41000070420C9B0500EB
:103C9000189B0500284653211AF03EFD002840F0ED
:103CA0008083E86894F8356003686C496C4A16F0C4
:103CB000040F08BF0A469B686A499847274658265A
:103CC000D7F85801014636F031F9002840F0328526
:103CD000D7F864010437014636F028F9002840F08F
:103CE0002185A6F15801C9B22046FCF7A9FF00289A
:103CF00000F08C8201365B2EE2D1E8685A490368F5
:103D00009B68984704E490F8363059077FF500AC7B
:103D1000564B01211B68986901F01AF80023C4F87A
:103D20004031FFF7F5BBFFF7EFFAFFF7F1BB28468D
:103D30001AF070FD00287FF778AF94F87071AFB17A
:103D400037464FF00208022ED4BF06F1580106F1A3
:103D50003E01C9B228461AF0DFFC10B108FA06F39A
:103D60001F4394F870310136B342ECDC28464521FC
:103D70001AF0D2FC40B12046FCF732FF002803DDE8
:103D8000022303FA00F00743384D01212B6898699C
:103D900000F0DEFF28683A460821F6F793F9FFF7AE
:103DA000B7BB334E18AC44F8186D012349092246BD
:103DB000FCF774FF214605F1100034F030FF129B30
:103DC0000C3EA3F10C00B0423FF4AEAB53F8042C10
:103DD000511E002A43F8041C3FF7A6AB0FA934F08C
:103DE000ADFDFFF7A1BB284653211AF095FC002832
:103DF00040F07F8394F87061002E3FF489AB002778
:103E000005E094F870610137BE427FF781ABA3688B
:103E10004FEA870853F8273093F839301B07F2D45C
:103E2000022FD4BF07F1580607F13E06F6B2284626
:103E300031461AF071FC0028E3D0314628460022B2
:103E40001AF07EFC0021064636F052F8002840F0B9
:103E50008182A36853F808309E62D2E7D0980500AB
:103E6000C8980500F898050004EB0500E40200106E
:103E7000680A0010E8689D49036800279B68984716
:103E800094F87061F6B1A36853F8273093F839209D
:103E9000100714D4022F186AD4BF07F1580607F18F
:103EA0003E0635F0E9F9EB68F6B232461E68CDE918
:103EB000000118468E49B368984794F8706101373D
:103EC000BE42E0DCE8688B4903689B689847D4F8F9
:103ED0003C0135F0D1F9EE68024637680B46BF6801
:103EE00030468549B84794F87061002736B3A36817
:103EF00053F8273093F8392011071CD4D3F82880C1
:103F0000022FD4BF07F1580907F13E094046414648
:103F10005FFA89F936F00AF868B9404635F0ACF92D
:103F2000EB684A461E68CDE9000118467049B3683F
:103F3000984794F870610137BE42D8DCE8686D4953
:103F400003689B6898476D4BD5F80C901A68D9F8B0
:103F50000030D2F81080D3F808A0D8F80C0035F063
:103F60008BF9D8F810B006460F465846594635F03A
:103F7000DDFF002840F0B583584635F07DF9CDE9E6
:103F80000001D8F8140035F077F932463B46CDE908
:103F9000020148465A49D047D4F8480135F06CF937
:103FA0000646D4F84C010F4635F066F9D5F80C807A
:103FB000D8F80090CDE90001D4F8500135F05CF953
:103FC000CDE90201D4F8540135F056F9CDE90401E8
:103FD00032463B46D9F808604A494046B047E8684F
:103FE0004949036800279B68984794F87061F6B1C7
:103FF000A36853F8273093F83920120714D4022FFE
:10400000586AD4BF07F1580607F13E0635F034F977
:10401000EB68F6B232461E68CDE900011846344915
:10402000B368984794F870610137BE42E0DCE868F5
:104030003049036813AF9B68984700226068149268
:104040001597169703680DF148088DF84C201792C4
:104050005B694146984710B3179B03B3E8682B4947
:1040600003689B689847159EBE4218BFB94611D099
:10407000706935F001F9EB68327C1F68CDE9000109
:10408000BF6818462249B847304634F086F948459B
:104090000646EDD1E868174903689B6898472B6886
:1040A00040F2F712934200F0F68294F83530DB07C5
:1040B00000F18E8194F83430DB093FF4B1ADD4F8CF
:1040C000B0600021304635F0FFFED4F8AC9008B364
:1040D0000021484635F0F8FEE0B1D4F8A8000021F0
:1040E00035F0F2FE00287FF49BAD13E06C990500DB
:1040F000AC99050004EB050084990500E40200106A
:10410000B8990500289A0500709A0500989B05004B
:104110009C9A0500304635F0AFF8064648460F46F3
:1041200035F0AAF8ED68D5F80090CDE90001D4F893
:10413000A80035F0A1F8CDE9020132463B46D9F896
:1041400008602846B649B0476AE5B64B1B6893F845
:10415000A42055077FF5DCA9EBE4284653211AF08B
:10416000DBFA002800F0C0802846532100221AF014
:10417000E7FAAD49054635F0B1FE002840F0F2817E
:104180002846AA4935F0C8FE002800F05284A84805
:10419000C4F83801FFF7BCB92B7A204643F001037D
:1041A0002B72FCF7B9FCFFF7BFB9284645211AF07E
:1041B000B3FA002800F02B822046FCF711FD071E01
:1041C00020DD284645211AF0A7FA002840F0288271
:1041D000002604EB8703C3F80C61C3F8F860A268FB
:1041E000E36A52F82770002B00F0188204F12400D3
:1041F000FCF72CFF0146304635F0D2FC014638462C
:10420000F5F736F92B7A5B09FFF722BAE868894996
:10421000036832469B6898476CE51AF0B3FA064685
:10422000FFF76FBAD9F8540135F026F8D8F80C60CA
:10423000024637680B46BF6830467F49B8472B7A3D
:1042400043F001032B72FFF763B95827284639461C
:104250001AF062FA002870D1043601370C2EFFB232
:10426000F4D12B7A5B09012B4FD194F87061032EA6
:104270005ED90327324602E00137BA4251D9A3681A
:104280004FEA870853F8273093F83930C3F3C00654
:10429000002EF1D107F13E095FFA89F94946284617
:1042A0001AF03AFA002840F0A88194F87021E3E768
:1042B000284655211AF030FA00283FF4B1AC3246B6
:1042C000284655211AF03CFA0023ED68C4F8343131
:1042D000C4F8280134F0D0FF2E6802460B46B668B9
:1042E00028465649B0479BE4D4F83811544835F075
:1042F0000BFD34F0C1FFED6802462E680B46B66830
:1043000028465049B047FFF703B9284653211AF011
:1043100003FA30B12846532100221AF011FAC4F8EA
:1043200054012B7A5B0900F09B81012B7FF4F0A8EC
:104330002046FCF7F1FBFFF7EBB800222846394690
:104340001AF0FEF92B7AA2195B0940F04F81C2F8EE
:10435000480181E73C4E7CE5431EFFF772BA2846D0
:1043600058211AF0D9F9002840F021820027284668
:1043700059211AF0D1F9002840F01282002628466F
:104380005A211AF0C9F9002840F0048200202B7A43
:10439000C4F8B070C4F8AC60C4F8A8005B09FFF7BB
:1043A00054B92846324653211AF010FA451E94F8A3
:1043B00035306842684160F3820384F83530FFF796
:1043C000A7B86068414603681B699847FFF7E5BBDB
:1043D000E8681E4903689B689847EE680FA8336831
:1043E00094F8A4109F68F6F727FB0F9A30461849F7
:1043F000B8470F9B174AA3F10C00904240F02B8363
:1044000004F1A40304F138069E420A933FF452AE2D
:1044100004F1440B01270C940B95CDF8348052E045
:10442000E89B0500E40200100000204100007A44EF
:104430000000C04038990500F0980500409B050039
:104440000080BB45509905000000C07FFC9A050024
:104450005CF905005C0A001075680021284635F0FB
:1044600033FD00283BD15BF80CACA9460B9B0FA891
:10447000DD68791E2B68D3F80880F6F7DDFA204650
:1044800034F0FAFECDE90001484634F0F5FECDE9FE
:104490000201504634F0F0FE0F9ACDE90401069275
:1044A00028463A46AF49C0470F9BAF4AA3F10C00DC
:1044B000904240F0C4820A9B0C36B34207F10107D8
:1044C0000BF10C0B49D0B4680021204635F0FCFC00
:1044D0000028C1D1D6F804905BF80CACC6E75BF8B5
:1044E0000CAC0021504635F0EFFC0028E3D1A94682
:1044F000BCE75321284600221AF022F94FF07E51E2
:10450000064635F0EBFC002840F08381C4F83C619E
:1045100070E45A21284600221AF012F993490646FF
:1045200035F0E6FC002840F07781914B1B681B6951
:104530001E61FFF7D9BA5821284600221AF000F967
:104540000021064635F0CAFC002840F06781884B00
:104550001B681B69DE60FFF7C0BA0C9C0B9DDDF881
:104560003480A7E5834813E65821284600221AF034
:10457000E7F894F83430D90702D57F4935F010FBBD
:10458000119935F003FA0146404635F001FA8046AC
:10459000FFF745B85A21284600221AF0D1F894F8BE
:1045A0003430D90702D5744935F0FAFA0F9935F04D
:1045B000EDF90146304635F0EBF90646FFF73DB818
:1045C0002846592100221AF0BBF894F83430DB0752
:1045D00002D5694935F0E4FA109935F0D7F901466A
:1045E000384635F0D5F90746FFF720B8012B7FF4A0
:1045F00033AEA3689B5958622EE649463246284698
:104600001AF09EF8A36853F8083058624DE6284621
:104610001AF000F900283FF4CFADF3E53146EEE59E
:104620002846452100221AF08BF80646D1E5284697
:1046300058211AF071F8002840F0078128465921C6
:104640001AF06AF8002840F0EB8028465A211AF048
:1046500063F8002840F00E812B7A5B09FEF7F5BF66
:10466000284641211AF058F8002800F01881E8681F
:104670004249036800269B68984706F14107FFB24C
:10468000394628461AF048F808BB0136032EF4D103
:104690002B7A5B0949E6E868394903689B689847C3
:1046A000D4F8340134F0E8FD0646D4F828010F466A
:1046B00034F0E2FDD5F80CE03246DEF80060CDE9DA
:1046C00000013B467046B6682E49B047EDE43946D6
:1046D000284600221AF034F8A36853F826305862AE
:1046E000D3E7002028494AE40022284659211AF03D
:1046F00027F894F83420D70702D51F4935F050FA2F
:104700001390FEF7BEBE0022284658211AF018F872
:1047100094F83420D20702D5174935F041FA1290A7
:10472000FEF7A8BEE8681949036832469B689847B7
:10473000FFF7D7BAE8681649036832469B6898477E
:10474000FFF7C6BA002228465A2119F0F9FF94F85B
:104750003420D60702D5084935F022FA1490814654
:10476000FEF798BEC89B05005C0A0010000080BFE1
:10477000E4020010000016443333CB41649B050073
:10478000A89A0500EC9A05000000F0BF24990500E6
:104790001099050028465A21002219F0D1FFF6E5AC
:1047A00028465921002219F0CBFF0646E7E52846A6
:1047B0005821002219F0C4FF0746D8E5099219F0E4
:1047C000ABFF099A002840F0C5802846592119F00E
:1047D000A3FF002872D128465A2119F09DFF002816
:1047E0003FF464A828465A21002219F0A9FF94F842
:1047F00034300146DD0703D59D4935F0D1F9014636
:10480000304635F0C5F80646FFF750B80025FFF7EB
:104810007EB94FF07E5679E6964E86E6002696E6FD
:10482000954B00221B6828465921DE6819F088FF45
:1048300094F83420D20702D58D4935F0B1F9C6F885
:1048400010013046FCF7E0FBFFE68B4B58211B685C
:1048500000222846DE6819F073FF94F83420D1074F
:1048600002D5834935F09CF9C6F80C013046FCF7B7
:10487000CBFBE3E6804B00221B6828465A21DE680A
:1048800019F05EFF94F83420D70702D5784935F047
:1048900087F9C6F814013046FCF7B6FBDCE628467B
:1048A000422119F039FF00287FF4E1AE2846432168
:1048B00019F032FF00287FF4DAAEE9E659212846E4
:1048C000002219F03DFF94F834300146DB0703D590
:1048D000674935F065F90146404635F059F880469C
:1048E00079E7D4F800C1D4F8FCE0D4F8F8300FA888
:1048F000214612AACDF848C0CDF84CE01493FCF73D
:10490000C9F82846582119F007FF00287CD128460D
:10491000592119F001FF002861D128465A2119F0C8
:10492000FBFE00283EF4C2AF5A210022284619F0AF
:1049300007FF94F83420D10702D54D4935F030F9FE
:104940000F9935F023F80146304635F01FF806463A
:10495000FEF7ACBF5821284619F0F2FE94F8343027
:104960000146DA0703D5424935F01AF901464846AF
:1049700035F00EF8814628E700222846582119F024
:10498000DFFE94F834308146DA077EF581AF38498E
:1049900035F006F98146FEF77BBF5A2128460022F2
:1049A00019F0CEFE94F834300646D9077EF57EAF76
:1049B0002F4935F0F5F80646FEF778BF284659210D
:1049C000002219F0BDFE94F834308046DB077EF5F6
:1049D00066AF274935F0E4F88046FEF760BF002255
:1049E0002846592119F0ACFE94F83420D20702D59C
:1049F0001F4935F0D5F8109934F0C8FF01464046FC
:104A000034F0C4FF804688E758210022284619F078
:104A100097FE94F83420D10702D5154935F0C0F837
:104A2000119934F0B3FF0146484634F0AFFF814698
:104A30006DE72946114835F067F9FFF7A9BB53F830
:104A4000042C511E002A43F8041C3FF734AD0EA974
:104A500033F074FF2FE553F8042C511E002A43F85D
:104A6000041C3FF7CDAC0EA933F068FFC8E400BFCB
:104A70003333CB410000C07FE40200100080BB450F
:104A800038B503210446144DF7F764F92046072191
:104A9000F7F760F92B68002258694EF2952113460A
:104AA000F6F76AFB2021F7F725F9F7F767F835F0F5
:104AB00079FA2968002213462062486944F2E761C6
:104AC000F6F75AFB6421F7F715F9F7F757F835F0C1
:104AD00069FAE06138BD00BFE402001010B5054B73
:104AE000044640F8043B00F0CFFD2046F7F71CF9E0
:104AF000204610BD089C050010B5074B044640F841
:104B0000043B00F0C1FD2046F7F70EF92046F6F70A
:104B1000D3FD204610BD00BF089C050001B17047C1
:104B200090F8283061F3410380F8283090F828305D
:104B300043F0040380F8283090F8283061F3C30371
:104B400080F8283090F8283061F3051380F8283079
:104B5000704700BF10B50446F7F7F6F8134B204630
:104B600040F8043B00F088FD94F8283000226FF3F1
:104B7000000384F8283094F8283062626FF3410310
:104B800084F8283094F8283020466FF3820384F8A4
:104B9000283094F828306FF3051384F8283094F8FF
:104BA00028306FF3C30384F8283010BD089C05003B
:104BB00010B50446084600F005FA201D216A00F0F1
:104BC000D7FD94F8283043F0010384F8283010BD55
:104BD00008B5043000F0C6FDC8B10D4B1B68DA689B
:104BE0009368D1688B420FD01A6892F83900C0F3ED
:104BF000400058B9043305E053F8042B92F83920EB
:104C0000920704D49942F7D1012008BD002008BDC5
:104C1000E4020010F8B5224D04462B680F46DA076F
:104C200015D5204E251D284600F09CFD68BBDFB140
:104C300031F0A2FF306094F828305B0706D494F876
:104C4000283043F0020384F82830F8BDF8BD284628
:104C500033F01CFB0028E4D031F08EFF114E3060A1
:104C6000284633F021FBDDE7284600F06DFD0028E3
:104C7000DED131F081FFE3694FF47A7202FB03F277
:104C80003368C01A9042D3D2F8BD94F828306FF33D
:104C9000410384F8283031F06FFF3060F8BD00BF69
:104CA000380500103C05001010B590F82830044677
:104CB000DB0715D4E26823699A4206D00434204603
:104CC00000F050FD10B100BE10BD10BD204600F038
:104CD00005FD00F097F92046BDE8104000F024BD26
:104CE0000021FFF797FFE5E7F8B5041D07462046CA
:104CF000164D00F029FD68B12868032190F8A460E2
:104D0000B3071CD43A46F5F7DDF9204600F01CFD48
:104D10000028F1D12B680D4E93F8A450C5F340053F
:104D20006DB9204600F0E6FC306808210122F5F755
:104D3000C9F938462946BDE8F840FFF76BBF204661
:104D400000F0C6FCBDE8F84000F05CB9E4020010D9
:104D5000F8B590F8283004466FF300030F4680F84A
:104D60002830051D114E07E02046FFF753FF30683D
:104D700003212246F5F7A6F9284600F0F3FC0121AD
:104D80000028F1D05FB1094D02E02868F5F79AF9E3
:104D90002046FFF71DFF032122460028F5D094F896
:104DA000283043F0010384F82830F8BDE4020010F5
:104DB0002DE9F0470C46074681B990F82830806904
:104DC00061F3051387F82830002851D033F074FAC6
:104DD0004FF00108BC614046BDE8F087041D204645
:104DE00000F0C0FC064600283DD197F82880C8F3A3
:104DF000C008B8F1000F36D01F4BF9681B68204679
:104E0000DB6893F8705100F053FC0146204600F037
:104E10006BFCC5EBC5094FEAC9090446484633F0A7
:104E20001FFA8446F8B195B1D4F84CA00AEB0605F8
:104E30000CEB06040FCD0FC40FCD0FC40FCD0FC464
:104E40003836B14595E8030084E80300EED197F8C1
:104E50002830012262F30513C7F818C087F82830FC
:104E60004046BDE8F0874FF000084046BDE8F087B7
:104E70004FF00108AFE700BFE40200102DE9F04158
:104E800090F82830044618070E4621D494F82830AC
:104E9000590714D52269A3689A4218BF251D08D066
:104EA0002169284600F004FC20612269A3689A4227
:104EB000F6D194F828306FF3820384F828302B4B16
:104EC00000221B68626293F8A470C7F340071FB109
:104ED00000252846BDE8F0812269A3689A42F7D0F0
:104EE00094F82830C3F30113012B22DC94F82850E6
:104EF000C5F34005002DEBD02169201D00F0F4FB27
:104F000090F850305A06E3D490F850305B0700D444
:104F100000BE90F85030C26943F0200380F8503052
:104F200090F850306FF3000380F8503062623060C8
:104F3000CFE72169201D00F0D7FBA169804600F072
:104F4000DBF898F85030D8F81C2043F0200388F89C
:104F5000503098F85030012567F3000388F850303E
:104F600028466262C6F80080BDE8F081E4020010C5
:104F700010B590F828300446C3F30113012B00DD6F
:104F800010BD0169043000F093FB206194F82830D3
:104F9000C3F30113012BF3D194F82830022262F3FA
:104FA000051384F82830EBE790F828306FF34103BD
:104FB00080F8283090F8283043F0040380F8283037
:104FC000704700BF0B4B0C4A1B6810B59B6A1070F2
:104FD000186934F051F902460B4634F0A1F9024643
:104FE0000B460020054934F0C5FA054CC4E9000120
:104FF00010BD00BFE4020010480500100000D043BF
:105000004005001090F8502070B56FF382020446FE
:10501000034680F850200021143043F8041B8342DB
:105020004FF00002F9D194F85030B4F8521003F068
:10503000FE0362F3410384F8503094F85000274D8A
:1050400020F0200084F8500094F85000002362F310
:10505000041084F8500094F85060E06C26F040068C
:1050600062F30B01E5626261E2632264A26462643E
:1050700084F85060A4F85210A361E3612362636274
:10508000A3622363A363164DE8B12D78D5B1E16C1B
:10509000C5EBC50500202031ED00044600220023A9
:1050A0003830A84241E9082341E9062341E90423B5
:1050B00041E90223C1E900238C60CC600C6101F15D
:1050C0003801EDD170BD2B78C3EBC300C00033F0C5
:1050D000C7F8E0640028D8D100BED6E70000C84277
:1050E0004805001010B5002304468364C364FFF72D
:1050F00089FF204610BD00BF2DE9F001104B80460E
:105100001B780F46C3B1C3EBC3034FEAC30C0026A1
:10511000BB191C469B6A63B1D8F84C500FCC354480
:105120000FC50FCC0FC50FCC0FC594E8030085E861
:10513000030038366645EBD1BDE8F001704700BF8B
:1051400048050010F8B5866B456A04460F462846A8
:10515000314634F0B9FE50B994F850309B0704D46E
:105160003046394634F0D8FE18B9666235462846CE
:10517000F8BDE36A3946384603F1004634F010FDC5
:1051800031460546304634F003FC216A34F008FD10
:105190000146284634F0FAFB35F09AFFA56B064627
:1051A000294634F0B9FE00B935466562DFE700BF35
:1051B00070B590F8503004469A0625D490F85030D7
:1051C0009B0702D5C469204670BD406AE36A014668
:1051D00003F1004634F0E4FC31460546304634F035
:1051E000D7FB216A34F0DCFC0146284634F0CEFBC4
:1051F00035F06EFFE4690546214634F08DFE002847
:10520000E1D12C46204670BD846A204670BD00BFA7
:1052100070B5C669044630460D4634F05FFE00B9ED
:105220002E46A56B3046294634F076FE00B9354649
:105230002846616A34F05CFE30B194F85030656203
:105240006FF3000384F850302046BDE87040FFF74C
:10525000AFBF00BF2DE9F04F07468DB0406916463D
:105260000C4634F045FC01464FF07E5034F04CFDC6
:105270005D4B09902046D3E9004533F0FDFF2246FF
:105280002B4634F04DF8CDE90A01304633F0F4FFF7
:105290000B4602462946204634F042F8534BCDE9EE
:1052A00006011B78002B00F096805149013BD1F894
:1052B0000090FA6CDBB207EB83064D4602F1200A40
:1052C000A7F1040BB14637E0CAF81030DDE90A2334
:1052D000CDE90223DDE90023DDE9020134F020F805
:1052E00035F02AFA34F094FEDDE900234AE904019E
:1052F000DDE9060134F014F835F01EFA34F088FECA
:10530000404261EB41014AE90201796B404634F0C9
:1053100047FC314634F0F8FC4FF0BD4134F040FC1E
:1053200033F0AAFF35F008FA34F072FECAE9000142
:10533000CB450AF1380A4ED05BF8043F1846CAF84C
:105340000830002BF4D034F0D3FB099934F028FC5A
:10535000804633F091FFAB6ACDE90001386B1E69DE
:1053600033F08AFFDDE9002333F0DAFFCDE90401F1
:10537000304633F081FF02460B46DDE9040134F08C
:10538000F9F800221B4B33F0CBFF35F0D5F934F0A0
:105390003FFE7A6CFB6B4AE9080100210020541C97
:1053A0004AE906010021CAF80C10CAF81040002B87
:1053B0008AD106983B6C029023B9079901F100410C
:1053C000039187E79A4209D0CAF8103000220023DF
:1053D000CDE902237EE70DB0BDE8F08F002000216B
:1053E000CDE9020176E700BF400500104805001036
:1053F000E40200100000D0432DE9F04F90F8504037
:1054000085B0A3068346174602D505B0BDE8F08FE8
:10541000C5690846294634F077FCDBF81840014698
:10542000204634F0BDFB29460646384634F06CFC75
:105430000146204634F0B4FB8046DBF8140034F01B
:1054400057FBDBF82C10044634F0AAFBDBF82010E5
:1054500034F05AFC41468146404634F0A1FB3146C7
:105460008246304634F09CFB49460546204634F0DF
:1054700097FB29460446504634F08AFA4FF07C5197
:1054800034F08EFB0146204634F082FA35F020FEDF
:10549000DBF818400546214634F03EFD002840F078
:1054A0008C803146CBF83450284634F06FFA4946A8
:1054B000039034F029FC29468246404634F066FACF
:1054C00009F1004134F020FC21468146284634F0A1
:1054D00023FD002840F0B38000222C465949504655
:1054E0000968896A0D690092294634F059FB35F044
:1054F00005FB34F057FD29460190484634F050FB37
:1055000035F0FCFA34F04EFD49460290504634F036
:105510003FFA009A114634F03BFA294634F040FB3A
:1055200035F0ECFA34F03EFD8146019834F0E0FAB3
:10553000294634F0E9FB8246029834F0D9FA29462C
:1055400034F0E2FB00210546504634F0E5FC00282B
:1055500070D05146039834F0D7FB8246284600218C
:1055600034F0DAFC002868D04146204634F00EFAC8
:10557000294634F0C9FB0246029B9BF85040C3EB1E
:105580000901019B44F04004CBF84010CBF83C30BB
:10559000CBF84490CBF83060CBF8287051468BF8AC
:1055A00050405846FFF756FE9BF8502022F040022C
:1055B0008BF8502005B0BDE8F08F3146CBF8344071
:1055C000204634F0E3F94946039034F09DFB214630
:1055D0008246404634F0DAF909F1004134F094FB98
:1055E0008146DBF8140034F083FA21460546304644
:1055F00034F0CEF94FF07C5134F0D2FA514634F009
:10560000CFFA0146284634F0C1F921460546404606
:1056100034F0BEF94FF07C5134F0C2FA494634F010
:10562000BFFA0146284634F0B1F9214634F06CFB4C
:10563000024653E74FF0000A90E700229CE72C4611
:10564000CFE700BFE402001008B5C36CC1EBC10195
:1056500003EBC103D3E9000134F064FA4FF00251C7
:1056600034F09EFA034B1B689B6A196934F098FA70
:1056700008BD00BFE4020010002282604260816821
:1056800002600261C1607047002310B5836043600F
:105690008268016904460360C26019B1034B18684F
:1056A000F5F756FF00232361204610BDFC020010D1
:1056B000006820B1013188428CBF08460020704745
:1056C000006808B109B1481E70470138704700BF33
:1056D00042680369542000FB023070478268036906
:1056E000542000FB023070470369542000FB013056
:1056F000704700BF036806E0013281689A4228BF04
:105700000022914206D14268002BF5D181681A46E9
:105710009142F8D0426823B101329A4234BF134615
:1057200000234360704700BF426883689A4203D0F9
:10573000036882680BB983607047013293428CBF63
:1057400013460023F7E700BF0368426823B1013224
:1057500093428CBF134600238068C31A58425841B5
:10576000704700BF42688068131A5842584170471A
:105770002DE9F8434268836804469A420F4602D0F6
:105780000020BDE8F883C1B972B6426883689A42C6
:1057900003D062B60020BDE8F88300238360036075
:1057A000436062B6016919B11E4B1868F5F7D0FE67
:1057B000002323610120BDE8F883DFF868905421BD
:1057C000D9F8000001FB07F1F5F756FE80460028E6
:1057D000D6D006467D1E3046013DFFF783FC6B1C8C
:1057E00006F15406F7D1216972B66268A3689A423D
:1057F00006D062B6D9F800004146F5F7A9FEBFE72A
:105800000023A360C4F810802760636062B631B1E2
:10581000D9F80000F5F79CFE0120BDE8F8830120CF
:10582000BDE8F883FC02001008B5044B53F82000D3
:1058300003681B6A9847C0B208BD00BF5C03001034
:1058400008B5044B53F8200003685B6A9847C0B260
:1058500008BD00BF5C0300102DE9F843D718BA4219
:10586000144680460D4613D2DFF82C9001E0BC426E
:105870000ED259F828002946026805F50075966A87
:105880002246B04701340028F1D00420BDE8F88357
:105890000020BDE8F88300BF5C0300102DE9F84349
:1058A000D718BA42144680460D4613D2DFF82C9022
:1058B00001E0BC420ED259F828002946026805F5DD
:1058C0000075D66A2246B04701340028F1D0042082
:1058D000BDE8F8830020BDE8F88300BF5C0300103A
:1058E00000B5012983B019D00BD3032903D00420BC
:1058F00003B05DF804FB01230020136003B05DF8E2
:1059000004FB114B53F8200060B103681B6B9847F0
:10591000003018BF012003B05DF804FB0A4B53F8B8
:10592000200018B9032003B05DF804FB03685B6B2B
:1059300001910092984700280199009A02DD1060B9
:105940000020D5E70846D3E75C0300102DE9F041BD
:10595000C56A04468D420E4602D0037973B916B962
:105960000020BDE8F081607804F130013246012367
:10597000FFF772FF20BBE662BDE8F08100F130085E
:10598000414640782A460123FFF788FFC0B9E36902
:10599000226A20711A449542E1D2E778012F01D89A
:1059A000DDE7E3691D44013F2A4660784146012353
:1059B000FFB2FFF773FF012FF3D1002ED0D0D2E753
:1059C0000120BDE8F08100BFF8B503690E4601F182
:1059D0000905002B4DD04469002294F80CC00CF04E
:1059E0000807FFB2A35C0132202B0DD0052B08BFA6
:1059F000E523A3F141011FB119299CBF2033DBB27C
:105A0000082A05F8013BEDD1237A202B1AD029462C
:105A10000CF0100C2E235FFA8CFC01F8043B0135CE
:105A2000E21D12F8013F202BA3F141070AD0BCF17F
:105A3000000F03D0192F9CBF2033DBB205F8013BC8
:105A40008D42EED1E37A3372A37FE27F217F1B0484
:105A500043EA0263627F0B4343EA02233360627EC0
:105A6000237E43EA0223B380E27DA37D43EA02233F
:105A7000F38000242C70B56935B1F36923B1036953
:105A80001BB9002400232B55F8BD028C4FF6FF7381
:105A90009A42F6D0C769388860B9F2E7F369013BEA
:105AA0009C42EED201342B1903F8010C37F8140094
:105AB0000028E7D00021EEF767FF0028EED1E0E7ED
:105AC0002DE9F84F00210546FFF740FF034650B986
:105AD0002B78032B0AD0002168780A46FFF700FFD5
:105AE000031C18BF01231846BDE8F88F6B79002B03
:105AF000F1D005F13001E8620B4605F50C7203F8B0
:105B0000010B93424FF00004F9D12A69EB68C2F30C
:105B1000072B4FEA124A4FEA134C4FEA136E5220FA
:105B20004FEA1269C3F3072885F8182285F819B2DD
:105B300061224FF0410B85F81AA255274FF0720AE7
:105B4000AA2685F81C3285F8300085F8310085F8E2
:105B5000322085F8172285F81B9285F81D8285F87A
:105B60001EC285F81FE285F82E7285F82F6285F82F
:105B700033B085F816B285F814A285F815A26878B6
:105B80006A690123FFF78AFE6C71A4E710B5044629
:105B90000A46407804F130010123FFF75DFE08B1A9
:105BA000032010BD94F82F1294F82E22174B42EACE
:105BB000012212B29A4201D0022010BD94F868303E
:105BC00094F869201B0494F8661043EA026394F881
:105BD00067200B4343EA02220D4B22F07F429A4298
:105BE000EBD094F8842094F8850094F88210120485
:105BF00042EA006294F883000A4342EA002020F05F
:105C00007F40C01A18BF012010BD00BF55AAFFFF7A
